:100000005446495300010000587402004E5268CD16
:100010001017013719011515443159301017020016
:100020001901151544313030101701281901151523
:100030004431594C030000000000000000000000A3
:100040005446435300200000944B0200000000007F
:100050000080011001210000252100004122000044
:10006000292100002B2100002D2100003D2100004E
:100070003D2100003D2100003D2100002F21000016
:10008000312100003D21000033210000115C0000FF
:10009000F75C0000372100003D210000B551001041
:1000A00037210000174000001D4000003D210000E6
:1000B0003D2100004B580000A94F000023400000E4
:1000C000D1550000372100003D2100003D210000F6
:1000D0000000000000000000000000000000000020
:1000E0000000000000000000000000000000000010
:1000F0000000000000000000000000000000000000
:1001000000000000000000000000000000000000EF
:1001100000000000000000000000000000000000DF
:1001200000000000000000000000000000000000CF
:1001300000000000000000000000000000000000BF
:1001400000000000000000000000000000000000AF
:1001500000F003F800F020F8FEE70D480168890878
:100160008900002001C101C101C101C17047000027
:100170001C5E0010FEE7FEE7FEE7FEE7FEE7FEE797
:10018000FEE7FEE7FEE703480047FEE7FEE7000064
:10019000202100003D21000000F002F800F068F886
:1001A0000AA090E8000C82448344AAF10107DA45D2
:1001B00001D100F05DF8AFF2090EBAE80F0013F0BC
:1001C000010F18BFFB1A43F00103184778EA01003A
:1001D000B8EA01000A444FF0000C10F8013B13F09C
:1001E000070408BF10F8014B1D1108BF10F8015B90
:1001F000641E05D010F8016B641E01F8016BF9D183
:1002000013F0080F1EBF10F8014BAD1C0C1B09D1D9
:100210006D1E58BF01F801CBFAD505E014F8016B4B
:1002200001F8016B6D1EF9D59142D6D370470000DD
:10023000103A24BF78C878C1FAD8520724BF30C812
:1002400030C144BF04680C607047000000230024E4
:1002500000250026103A28BF78C1FBD8520728BFD6
:1002600030C148BF0B6070471FB51FBD10B510BD32
:10027000DFF80CD0FFF7F8FF05F080FA1CF0BEFCA9
:100280000080011003B4FFF7F1FF03BC1CF0BEFCBB
:100290001EF0040F0CBFEFF30880EFF309800AF0A3
:1002A000B1BD000008B5002103200B460A460091AD
:1002B0001AF0FCF808BD38B5F74D00246C81AC810C
:1002C000EC811AF0C4F8E861FF20E871F348234696
:1002D0002246046044600472012028726C612C7014
:1002E0000320214600941AF0E1F8012038BD38B50A
:1002F000E94D0228EC7922460DD0052810D0A24203
:1003000008BF38BD002003460246214600901AF07F
:10031000CDF8EC7138BD022914BF01240224EEE7A8
:10032000022914BF64246524E9E738B513460A4658
:100330004FF0010C00240146604600941AF0B6F814
:1003400038BDD549012048707047D3484078704780
:10035000D1490020487070472DE9F041044601273B
:10036000002503F00700CC4E8846012804BF00207A
:10037000F08146D0022844D1F08904280BD200280D
:1003800018BFB06902D11AF0B6F9B06110F8011BBC
:100390002170B0612EE0062808D21AF0AEF9F1897A
:1003A000C1F10501C900C840207023E0082808D227
:1003B0001AF0A7F9F189C1F10701C900C8402070FE
:1003C00018E00C2808D21AF042F8F189C1F10B01AB
:1003D000C900C84020700DE00E2808D21AF039F884
:1003E000F189C1F10D01C900C840207002E0FF2071
:1003F00020700027F089401C80B2F0810E2828BFB1
:10040000012588F800503846BDE8F08130B403F08B
:1004100007000024DFF880C201280BD06046BCF83A
:100420000E304089022B0CD2120242EA1020ACF8A6
:100430000A0010E0ACF80A40ACF80C40ACF80E40F2
:100440000CE01844851EB5F5806F04DADCF81C500A
:10045000284400F8022C581CACF80E000C7030BC7C
:1004600000207047F0B40746002003F007048A4DCF
:100470000646012C04BFEE812E6125D0DFF818C29C
:10048000022CBCF80CC003D013F0070F0DD01BE0FA
:10049000EA890CEB0203B3F5806F15D2E869C05C02
:1004A0003870501CE88101200EE0120242EA1C2242
:1004B000AA812B69012B05D1B2F5806F24BF40F2D0
:1004C000FF32AA815A1C2A610E70F0BC704738B501
:1004D00003F0070000240D4601280AD16E4821468A
:1004E0000B46C4814481848102200A46009419F09D
:1004F000DDFF2C70002038BD30B50C0068A183B042
:1005000009684FF00002029108BF03250AD0217844
:1005100002AB5D5C002D18BF022D41D0012D7ED0B5
:10052000032D0DD10F210170032141704280828083
:10053000C280028142818281817B21F0010181732D
:10054000002D1EBF012D03B030BD05F025F9052893
:100550001CBF03B030BD0AF0ECFC042804BF03B09C
:1005600030BD002D0CBFC020C1208DF80000607888
:100570008DF8010060880123000A8DF80200A07840
:100580008DF80300A0880622000A8DF80400207967
:100590008DF80500694607200DF036FE03B030BD2A
:1005A000617800EB011202F8101C617800EB011178
:1005B00001F80F5C6278618800EB021222F80E1CD1
:1005C0006278A18800EB021222F80C1C6278A179F3
:1005D00000EB021222F80A1C6278217A00EB021268
:1005E00022F8081C6278617A00EB021222F8061CDD
:1005F0006278217B00EB021222F8041CE1790529C4
:10060000617800EB011010F8021C0EBF41F00101EF
:1006100021F0010100F8021C92D132E0FFE761787D
:1006200000EB011303F8101C6378012100EB0313A6
:1006300003F80F1C6378618800EB031323F80E1C8A
:100640006378A18800EB031323F80C1C617800EB9E
:10065000011121F80A2C617800EB011121F8082C16
:10066000617800EB011121F8062C617800EB011193
:1006700021F8042C617800EB011010F8021C21F025
:10068000010100F8021C5BE70349002088707047F5
:10069000014880787047000000840010F88800103E
:1006A000030002017C490120887070477B4A115485
:1006B0007047794800B5C06983B04FF000014078B9
:1006C00010F0020F0AD000918DF8041001230522CA
:1006D000694600200DF0CFFD03B000BD10F0040FFF
:1006E00012D001208DF800008DF801108DF8021055
:1006F0008DF803108DF8041003460522694600208A
:100700000DF0B9FD03B000BD10F0080F12D00220AB
:100710008DF800008DF801108DF802108DF803108F
:100720008DF8041001230522694600200DF0A3FD79
:1007300003B000BD03B001230022632107205DF850
:1007400004EB0DF031BD10B5044615F0DBF80028C0
:1007500018BF10BD226812F0C00F12D04E4812F020
:10076000400F04BF0021017004D0012101704169D4
:10077000491C416101230021BDE8104006200DF015
:1007800013BD012300226321BDE8104007200DF0B6
:100790000BBD70474049002818BF01200872704700
:1007A0003D48007A70473C48C0787047002818BF21
:1007B00001203949C87070473748C07870473649BA
:1007C0000871704734480079002818BF012070472D
:1007D00001460020072904BF31487047082908BF97
:1007E0003048704710B44FF0000C072808BFDFF8FE
:1007F000B0C003D0082808BFDFF8A8C04FF0000041
:10080000ABB1002A9CBF10BC70473CF91030141AE1
:1008100001EB440434F9024C234403EBD3735B1023
:100820002CF81030401C8242EFD810BC7047002AD0
:100830009CBF10BC7047131A01EB430333F8023C12
:100840002CF81030401C8242F5D810BC704712487A
:100850000078002818BF012070470F484069704792
:100860000D4948617047002818BF01200A494871A6
:10087000704709484079002818BF012070470028B8
:1008800018BF012004498871704703488079002807
:1008900018BF01207047000000840010F888001085
:1008A0000A890010028900107047FE48D0F85003F2
:1008B00000F00100704770B5FA4D04000AD001F055
:1008C0003DFB38B9D5F8500310F0010F1CBF0020D4
:1008D000A86005D10120A860002C08BF002000D02E
:1008E0000120286270BDEF48006A002818BF01206F
:1008F0007047C00000F1804000F5A04041637047A0
:10090000C00000F1804000F5A040006B00F4807052
:1009100070471021C00000F1804000F5A040416305
:100920007047E049D1F8402160F30D22C1F8402121
:100930007047DC48D0F84001C0F30520704700F054
:100940000F0202EB42029201C0F3031002EB80108F
:1009500000F1804000F5A0400029D0F8401114BFFC
:1009600041F0010121F00101C0F84011704700F091
:100970000F0101EB41018901C0F3031001EB80106D
:1009800000F1804000F5A040D0F8400100F00100E7
:100990007047C44900230B6202680A6042684A60DB
:1009A00082688A60C268CA60426A0A64826A4A646B
:1009B00002698A614269CA61826B0A66826C0A674F
:1009C000C26C4A67026D8A67426DCA67826DC1F860
:1009D0008020C26DC1F88420026EC1F88820426E6A
:1009E000C1F88C20426FC1F8B020C26FC1F8B820A6
:1009F000C26EC1F8A820D0F89422C1F85023D0F8D4
:100A00009822C1F85423D0F89C22C1F85823D0F87A
:100A1000A022C1F85C23D0F88420C1F8F020D0F8DF
:100A20008820C1F8F420D0F88C20C1F8F820D0F844
:100A30009020C1F8FC2021224A63CA63C2694A623D
:100A4000C26A8A64026BCA64026FC1F8AC20026A8F
:100A5000CA62426B0A65C26B4A66026C8A66426C65
:100A6000CA66826FC1F8B420D0F88020C1F8BC20DB
:100A7000D0F8A422C1F86023D0F8A822C1F86423DA
:100A8000D0F8AC22C1F86823D0F8B022C1F86C23AA
:100A9000D0F8B422C1F87023D0F8B822C1F874237A
:100AA000D0F8BC22C1F87823D0F8C022C1F87C234A
:100AB000D0F88C2222F48032C1F84023D0F8902262
:100AC000C1F84C23D0F89420C1F80021D0F8982028
:100AD000C1F80421D0F89C20C1F80821D0F8A0204A
:100AE000C1F80C21D0F8A420C1F81021D0F8A8201A
:100AF000C1F81421D0F8C820C1F83421D0F8AC20B6
:100B0000C1F81821D0F8B020C1F81C21D0F8B420C9
:100B1000C1F82021D0F8B820C1F82421D0F8BC2099
:100B2000C1F82821D0F8C020C1F82C21D0F8C42069
:100B3000C1F83021D0F8CC20C1F84021D0F8D02025
:100B4000C1F84421D0F8D820C1F84C21D0F8E420D5
:100B5000C1F86021D0F8E820C1F86421D0F8EC2079
:100B6000C1F86821D0F8F020C1F86C21D0F8D42069
:100B7000C1F84821D0F8DC20C1F85021D0F8E0209D
:100B8000C1F85421D0F8F420C1F87021D0F8F82031
:100B9000C1F87421D0F8FC20C1F87821D0F80021E8
:100BA000C1F87C21D0F83C21C1F8C021D0F8402107
:100BB000C1F8C421D0F84421C1F8C821D0F8482197
:100BC000C1F8CC21D0F84C21C1F8D021D0F8502167
:100BD000C1F8D421D0F87021C1F8F421D0F8542103
:100BE000C1F8D821D0F85821C1F8DC21D0F85C2117
:100BF000C1F8E021D0F86021C1F8E421D0F86421E7
:100C0000C1F8E821D0F86821C1F8EC21D0F86C21B6
:100C1000C1F8F021D0F87421C1F80022D0F8782171
:100C2000C1F80422D0F88021C1F80C22D0F88C2120
:100C3000C1F82022D0F89021C1F82422D0F89421C4
:100C4000C1F82822D0F89821C1F82C22D0F8AC2184
:100C5000C1F84022D0F8B021C1F84422D0F8B82120
:100C6000C1F84C22D0F8C421C1F86022D0F8C821C4
:100C7000C1F86422D0F8CC21C1F86822D0F8D02184
:100C8000C1F86C22D0F87C21C1F80822D0F8842168
:100C9000C1F81022D0F88821C1F81422D0F89C2184
:100CA00002E0000000500040C1F83022D0F8A0213E
:100CB000C1F83422D0F8A421C1F83822D0F8A821F4
:100CC000C1F83C22D0F8B421C1F84822D0F8BC21A8
:100CD000C1F85022D0F8C021C1F85422D0F8D42154
:100CE000C1F87022D0F8D821C1F87422D0F8DC21E4
:100CF000C1F87822D0F8E021C1F87C22D0F8E421B4
:100D0000C1F88022D0F8E821C1F88422D0F8EC2183
:100D1000C1F88822D0F8F021C1F88C22D0F8F42153
:100D2000C1F89022D0F8F821C1F89422D0F8182206
:100D3000C1F8B422D0F8FC21C1F89822D0F80022E2
:100D4000C1F89C22D0F80422C1F8A022D0F80822D1
:100D5000C1F8A422D0F80C22C1F8A822D0F81022A1
:100D6000C1F8AC22D0F81422C1F8B022D0F81C226D
:100D7000C1F8C022D0F82022C1F8C422D0F828221D
:100D8000C1F8CC22D0F83422C1F8E022D0F83822C1
:100D9000C1F8E422D0F83C22C1F8E822D0F8402281
:100DA000C1F8EC22D0F85422C1F80023D0F8582220
:100DB000C1F80423D0F86022C1F80C23D0F86C22CB
:100DC000C1F82023D0F87022C1F82423D0F874226F
:100DD000C1F82823D0F87822C1F82C23D0F8242297
:100DE000C1F8C822D0F82C22C1F8D022D0F8302285
:100DF000C1F8D422D0F84422C1F8F022D0F8482219
:100E0000C1F8F422D0F84C22C1F8F822D0F85022D0
:100E1000C1F8FC22D0F85C22C1F80823D0F8642283
:100E2000C1F81023D0F86822C1F81423D0F87C222E
:100E3000C1F83023D0F88022C1F83423D0F88422BE
:100E4000C1F83823D0F88822C1F83C23FD4A126843
:100E500032F0FF0C05D1D1F890C062F3030CC1F859
:100E600090C0F94A5370D0F8943213F0010F1CBFB0
:100E700001235370D1F8503323F00103C1F85033EC
:100E8000D0F8A43213F0010F03D0537843F00203DB
:100E90005370D1F8603323F00103C1F86033D0F808
:100EA000B43213F0010F03D0537843F004035370AE
:100EB000D1F8703323F00103C1F87033D0F8AC02DD
:100EC00010F0010F03D0507840F008005070D1F8B6
:100ED000680320F00100C1F868037047DA48007821
:100EE0007047D94880787047D749C8707047D6484E
:100EF000C0787047D549D1F8542360F30902C1F88E
:100F000054237047D148D0F85403C0F30900704708
:100F1000CD4948607047CD48C06870472DE9F0471B
:100F2000DFF82493054615F4003F99F8010099F87D
:100F3000031000EA010418BF24F0010415F4802F07
:100F400018BF24F0020415F4002F18BF24F0040485
:100F500015F4801F18BF24F00804DFF8F082D8F8D9
:100F6000400320F48030C8F8400314F00F0F65D020
:100F7000D9F80460D8F84803002740F00100C8F809
:100F80004803D8F8480320F00100C8F84803D8F80F
:100F9000400340F48030C8F840034FF0630A0DE08E
:100FA00002F0C7FE5046D8F8481311F0010F01D0E7
:100FB000012703E0011EA0F10100F4DC301EA6F1C0
:100FC000010601DD002FEBD0BFB3D8F8500314F0B9
:100FD000010F0CBF20F0010040F00100C8F85003E1
:100FE000D8F8600314F0020F14BF40F0010020F0A5
:100FF0000100C8F86003D8F8700314F0040F14BFA0
:1010000040F0010020F00100C8F87003D8F8680330
:1010100014F0080F14BF40F0010020F00100C8F8E0
:10102000680389F80240012089F80000D8F84003DD
:1010300040F48030C8F840033AE0FFE7D8F85003A6
:1010400020F00100C8F85003D8F8600320F0010038
:10105000C8F86003D8F8700320F00100C8F87003E6
:10106000D8F8680320F00100C8F86803002089F868
:101070000200ACB1022089F80000D8F8400340F427
:101080008030C8F84003D8F8480340F00100C8F8A1
:101090004803D8F8480320F00100C8F8480307E0E7
:1010A000D8F8401321F48031C8F8401389F80000C3
:1010B000D8F8400115F0020F20F00D0018BF40F0E5
:1010C000010015F0080F18BF40F0040015F0040FE0
:1010D00018BF40F00800C8F8400115F0010F21D0FA
:1010E00001F061F9044601F061F90146D8F80C00FD
:1010F00000280EBF2046084621460028D8F80002E6
:1011000014BF40F0010020F00100C8F80002D8F838
:101110004002002914BF40F0010020F00100C8F88F
:1011200040020BE0D8F8000220F00100C8F80002ED
:10113000D8F8400220F00100C8F8400215F0200F56
:1011400018BF002417D0204601F037F900284FEAD5
:10115000841000F1804000F5A040D0F8C01214BF08
:1011600041F0010121F00101C0F8C012641C022C01
:10117000E9D3BDE8F087D8F8C00220F00100C8F834
:10118000C002D8F8000320F00100C8F80003BDE851
:10119000F0872DE9F003024602F00F01002001EB79
:1011A00041018C01C2F3031104EB811101F1804173
:1011B00001F5A041D1F8401111F0010F11D142F019
:1011C0001001C1F3031104EB811101F1804101F51C
:1011D000A041D1F8401111F0010F04BFBDE8F003A8
:1011E000704702EB42018E0106F1804101F5A041FA
:1011F000D1F82431C3F30809144BDB69D1F800118D
:1012000003F008071FFA81F8002142EA0113C3F333
:10121000031304EB831303F1804303F5A043D3F8D6
:10122000403113F0010F20D006EB811303F180430E
:1012300003F5A043D3F844C1CCF3080517F1000C23
:1012400006E00000E0FE0300208400100050004093
:101250001CBFD3F844C1CCF3023CD3F8403105FAAB
:101260000CFCC3F3054360441844491C0229CCD349
:1012700009EBC90100FB08F001EB0911BDE8F0031F
:1012800000EB4100704710B50120FFF782FF0446D4
:101290000220FFF77EFF044400F03DFC20444FF4A1
:1012A0007A7148434CF25031B0FBF1F010BD2DE99A
:1012B000F041FB4E0546306810F01F0408BF0124C2
:1012C0000120FFF766FF07460220FFF762FF074491
:1012D00000F021FC3918F34F002D18BF00294ED023
:1012E000D6F85003002210F0010F36D07820B0EB72
:1012F000151F08D9D6F85C0320F00F0040F001005C
:10130000C6F85C032EE0D6F85403E74BC0F309009F
:1013100060436FF0180C00FB0CF003EB4003E34854
:10132000A0FB05C04FEA502CB3FBF1F0102828BFFA
:101330000F20844598BF6046002808BF012005D0D3
:10134000012884BF00FB1132B2FBF0F2D6F85C3307
:1013500060F30303C6F85C3304E0B7FBF5F08842A2
:1013600088BF421A32206043B2FBF0F0B0F5005F54
:1013700028BF41F6FF70726860F30C0272607068FB
:10138000C0F30C00604300EBC00202EB001001EB65
:101390004000B7FBF0F0BDE8F081C148D0F8501331
:1013A00011F0010F07D0D0F85C0300F00F00C0EB84
:1013B00000108001704770B50168406801F01F059A
:1013C000C0F30C060120FFF7E4FE04460220FFF7FD
:1013D000E0FE044400F09FFB06FB05F1322201FB16
:1013E00002410844AF49B1FBF0F070BDAC48D0F801
:1013F0005C0300F00F007047A9494A684B68C2F3CC
:101400000C0260F30C034B6010467047A448406820
:10141000C0F30C00704700EB4000800100F18040F9
:1014200000F5A040D0F80001A14980B2B1FBF0F076
:10143000401C4008704730B49D4B31B1B3FBF1F113
:10144000491C4A08B2F5804F01D343F6FF72B3FB43
:10145000F2F1491C4D0800EB40018901530801F1EC
:10146000804101F5A041002807BF981FA3F10C0C93
:10147000D1F8040180B218BFA2F1060C2CF0010CC7
:10148000D1F8004162F30F04C1F80041D1F8002106
:1014900063F31F42C1F80021D1F8042160F30F0269
:1014A000C1F80421D1F818016CF30F00C1F818013C
:1014B000284630BC704700EB4000800100F18040BE
:1014C00000F5A040D0F80001000C704700EB40028E
:1014D000920102F1804202F5A042D2F8003161F39C
:1014E0001F43C2F80031002818BF70478A1F901FA1
:1014F00020F001016A48D0F8043162F30F03C0F80C
:101500000431D0F8182161F30F02C0F81821704798
:1015100000F00F0101EB41018901C0F3031001EB61
:10152000801000F1804000F5A040D0F84401C0F3E5
:101530000800704700F00F0202EB42029201C0F374
:1015400003105C4B02EB801000F1804000F5A040DE
:101550009B58D0F84421CB1A61F30802C0F844210B
:10156000D0F844119B1E63F31841C0F84411704732
:101570004B49C969504A11F0100F00F00F0101EBFF
:1015800041014FEA8111C0F3031001EB801000F11B
:10159000804000F5A0405258D0F84401D2B2C0F3C8
:1015A000080008BF0022801A0004000C08BF0120B8
:1015B000704703091B0203EB810101F1405101F562
:1015C00040410007C00E0B6802FA00F018430860A3
:1015D00070470209120202EB810101F1405101F54D
:1015E000404100070968C00E21FA00F000F0030036
:1015F000704700F00F0303EB43039B01C0F303109C
:1016000003EB801000EB810000F1804000F5A0406A
:10161000C0F85021704700F00F0202EB4202920125
:10162000C0F3031002EB801000EB810000F180405A
:1016300000F5A040D0F850017047194A0021D26946
:1016400012F0080F10D000F00F0101EB41018901E9
:10165000C0F3031001EB801000F1804000F5A040C2
:10166000D0F84401C0F30231084670470C4AD369F0
:1016700043F00803D36100F00F0202EB4202920133
:10168000C0F3031002EB801000F1804000F5A04091
:10169000D0F8442161F30E32C0F8442170470000B5
:1016A000005000400008AF2FD8810C00898888883E
:1016B000A08601001C51004028510040F84A00213A
:1016C000D26912F0080F10D000F00F0101EB4101B8
:1016D0008901C0F3031001EB801000F1804000F598
:1016E000A040D0F84801C0F302410846704700F01E
:1016F0000F0202EB42029201C0F3031002EB8010D2
:1017000000F1804000F5A040D0F8482161F312427A
:10171000C0F848217047042988BF704710B40023DF
:10172000DF4CE26912F0080F00F00F0202EB4202F8
:101730004FEA8212C0F3031002EB801000EB0402A8
:101740001CBFD2F84401C0F302330020D4F81CC0FF
:101750001CF0080F1CBFD2F84801C0F30240C91AA0
:101760000844042803DD081A011D042003E00028B2
:10177000BCBF014400201944E36943F00803E3615E
:10178000D2F8443161F30E33C2F84431D2F8481133
:1017900060F31241C2F8481110BC7047C0490028DC
:1017A000886914BF40F0080020F008008861704785
:1017B000BB488069C0F3C000704700F00F0202EB25
:1017C00042029201C0F3031002EB801000F180404E
:1017D00000F5A040C0F84C11704700F00F0101EB7C
:1017E00041018901C0F3031001EB801000F180403A
:1017F00000F5A040D0F84C017047A94AD2F85C131C
:10180000022903D110F0010F18BF7047D2F8400130
:1018100010F0010F0BD0D2F84C01D2F8441100287F
:10182000C1F302311EBF0029C043C2F84C0101219F
:1018300001EB410100204FEA811C0CEB801101F10A
:10184000804101F5A041D1F8402112F0010F0BD0E9
:10185000D1F84C21D1F84431002AC3F302331EBF22
:10186000002BD243C1F84C21401C0228E5D370471D
:101870008B4A0021D26912F0080F10D000F00F013E
:1018800001EB41018901C0F3031001EB801000F16D
:10189000804000F5A040D0F84801C0F30051084650
:1018A00070470120704710B4022ADDF804C026BF3B
:1018B000921E52080022022B26BF9B1E5B080023AB
:1018C000784CA4FB0C4C4FEA1C1400F00F0C0CEBF2
:1018D0004C0C4FEA8C1CC0F303100CEB801000F191
:1018E000804000F5A040D0F864C161F31B6C62F346
:1018F000144C63F30C2C64F3070CC0F864C110BCE7
:10190000704770B400F00F0404EB4404A401C0F36A
:10191000031004EB801000F1804000F5A040DDF8DA
:101920000CC0D0F864010029C0F30366C0F304447E
:10193000C0F30425C0B218BF0E6012B16100891C4B
:10194000116013B16900891C1960BCF1000F04BF5C
:1019500070BC704700EB80008000CCF8000070BCC9
:10196000704770B491B000224FF480456C10EC4683
:1019700001E0082A05D2531C03EB8303B5FBF3F304
:1019800004E0D31F03EB8303B4FBF3F35B1A48BFFC
:101990005B424CF82230521C102AEAD30026009BEE
:1019A00001215CF821209A42BCBF13460E46491C17
:1019B0001029F6D300F00F0101EB41018901C0F3BA
:1019C000031001EB801000F1804101F5A041D1F836
:1019D0006801D1F8682100F00F0066F30302C1F836
:1019E0006821082807D2401C00EB8000B5FBF0F00E
:1019F00011B070BC7047C01F00EB8000B4FBF0F06A
:101A000011B070BC704700F00F0101EB410189017A
:101A1000C0F3031001EB801000F1804000F5A040FE
:101A2000D0F8680100F00F00082834BF401CC01F28
:101A300000EB800034BF4FF480414FF40051B1FB04
:101A4000F0F0704710F00F0F08BF704700F00F0064
:101A500000EB4000800100F1804000F5A04000292B
:101A6000D0F82C110CBF21F4803141F48031C0F842
:101A70002C117047002110F00F0F0ED000F00F0056
:101A800000EB4000800100F1804000F5A040D0F85C
:101A90002C0110F4803F18BF012108467047000058
:101AA00000500040CDCCCCCC00F00F0000EB40004B
:101AB000800100F1804202F5A042D2F83401C2F860
:101AC000341170472F4B58679967DA6770472D4973
:101AD0000028D1F8AC0014BF40F0020020F0020052
:101AE000C1F8AC00704727490028D1F8AC0014BFFA
:101AF00040F0010020F00100C1F8AC00704721481F
:101B0000D0F8E00070471F49C1F8E40070471D4855
:101B1000D0F89800704770B41A4E0020D6F84011E3
:101B200011F0010F04BF70BC704711F0040FD6F81C
:101B3000242101F00805D6F800C1C2F308021FFAFB
:101B40008CF4D6F844C1CCF3080C18BFC1F307409D
:101B5000F369C1F3052113F008031CBFD6F8443123
:101B6000C3F30233002D18BF491C0CFA03F301FB29
:101B70000300604302EBC20170BC01EB021100EBF9
:101B80004100704700500040FEF7ADBE10B5FEF7B3
:101B9000AAFE012818BF10BD0020FEF78CFE2121EF
:101BA0000020FEF7A6FE2121BDE810400120FEF72F
:101BB000A0BE10B5FEF778FEFEF795FE01280AD10B
:101BC0000020FEF778FE21210020FEF792FE212161
:101BD0000120FEF78EFE0121052001F0F4FB01211A
:101BE000052001F0F0FBFF490020C87110BD10B5C1
:101BF0004FF4066001F03DFCBDE810404FF4066074
:101C000001F028BCF74A01465079002818BF01208E
:101C1000002918BF01215171002191717047F14ACB
:101C2000516A506208467047EE490020087188707A
:101C300048707047EB490020087188704870704701
:101C400070B50007C00E0D46801E00EB400101EB91
:101C50000014E5484FF4987200EBC40029461AF0CE
:101C6000DBFFE24805F5987100EBC400BDE8704069
:101C70004FF498721AF0D0BF2DE9F0410546FEF7F7
:101C800058FEDB4FDFF86C830446EDB14C2004FBBB
:101C900000F21646294638461AF0BEFF324605F5D0
:101CA000006140461AF0B8FF04EB440000EB041456
:101CB00007EB84004C211AF0B4FF08EB8400BDE868
:101CC000F0414C211AF0ADBF4C21401C41430C4661
:101CD00038461AF0A6FF21464046BDE8F0411AF00A
:101CE000A0BF10B5BF4CE061FFF718F9FFF7F6F899
:101CF000A1696FF30F01A161A269C1B242EA01219A
:101D0000A161022818BF10BDA06940F00100A061C8
:101D100010BDB9488168B94A114381600168521CFD
:101D20001143016000F065BE2DE9F041B24A0C4656
:101D300005469168B148084390601368B04818435D
:101D4000106000F056FE0026002C76D00020FEF732
:101D5000B2FD206820B1FEF71CFE0020FEF7ABFDAF
:101D60002846FFF7BEFF0020FEF701FE70B3606853
:101D7000FFF782FFA348E16819B102151AF04CFF82
:101D80001DE0A14D4FF440711AF04BFF00200123DC
:101D90002956002910DB0A09120202EB800202F127
:101DA000405202F540420907C90ED2F800C003FABA
:101DB00001F14CEA01011160401C2628E8D3934848
:101DC000616959B14FF400721AF026FF0120FEF745
:101DD000CEFDDFF81482854F48B904E04FF400715E
:101DE0001AF01FFFF2E71120FEF7C1FD70B1A568E0
:101DF00065B140464FF4987229461AF00DFF3846F7
:101E00004FF4987205F598711AF006FF0220FEF75C
:101E1000AEFD18B91220FEF7AAFD70B1246964B1B5
:101E20007B484FF4987221461AF0F6FE79484FF439
:101E3000987204F598711AF0EFFE6A480671867080
:101E40004670466241790021417186714FF4066007
:101E500001F00FFBBDE8F0414FF4066001F0FABA63
:101E600010B50020FEF727FD00F0B0FD5D48C078FA
:101E7000002808BF10BD6048016821F0030141F04F
:101E80000D7141F080510160816821F0020141F043
:101E90000D7141F08051816010BD4FF4066001F07A
:101EA000DEBA10B54FF4066001F0D9FAFEF71BFD5B
:101EB00001280AD10020FEF7FEFC21210020FEF7B8
:101EC00018FD21210120FEF714FD5348D0F84013DE
:101ED00021F48031C0F840130020FEF7ECFC00F044
:101EE00075FD4048C078002808BF10BD4248016811
:101EF00021F0030141F00D7141F0805101608168D2
:101F000021F0020141F00D7141F08051816010BD5E
:101F100010B501F0A9FA10F0600018BF012010BD43
:101F20003048C06970472F488069704772B62D49A4
:101F30008A6922EA0000886162B670472948007801
:101F4000002818BF0120704770B5FEF7CCFC0028B0
:101F500018BF70BD0024234D2C71AC706C70212112
:101F60002046FEF7C6FC21210120FEF7C2FC2C70A2
:101F7000BDE870400120FEF79EBC70B50446FEF738
:101F8000B2FC002818BF70BD0021164D2971A97040
:101F9000697021210020FEF7ACFC21210120FEF711
:101FA000A8FC022C3CBF0120FEF7B3FC01202870E6
:101FB0002C62BDE87040FEF77EBC10B5FEF793FCC6
:101FC000002818BF10BD0020064C2071A070607062
:101FD0002121FEF78EFC21210120FEF78AFC012041
:101FE0001CE0000028840010189D003018BD00304F
:101FF0000080003000A00030008000400200341259
:102000000300341200C000301489001000D00030EA
:10201000489E003048BE003000500040FEF779FC7A
:10202000012020702062BDE81040FEF744BC002073
:10203000FEF741BCFE490020887048700120FEF781
:102040003ABCFB4988627047F948806A70470028AB
:1020500018BF0120F649C8627047F548C06A0028D9
:1020600018BF01207047002000F0CFBB012000F016
:10207000CCBB10B5FFF743FD0446FFF744FDED4828
:10208000044208BF10BDEA48816941F00401816142
:102090000E2101EAD43104F001020A43816962F39E
:1020A0001F418161E448016841F02001016010BDD9
:1020B000002818BF0120DE49C8707047DF4870470C
:1020C000DF487047DA48006B7047D948406B70476B
:1020D000D748806B70472DE9F04FD84F4FF0000C78
:1020E0008DB007F14C04E6464FF0FF3807F80C803E
:1020F00004F80CE00CF1010CBCF1260FF6DB4FF0FC
:10210000000C002807DD12F80C5007F80C500CF1F9
:10211000010C6045F7DC00220126CDF804E06D4695
:10212000CDF800E0002816DD17F902C0BCF1000F61
:102130000EDBBCF1260F0BD24FEA5C190CF01F0C22
:1021400055F829A006FA0CFC4AEA0C0C45F829C0FF
:10215000521C8242E8DB002294460DF108094FEA46
:10216000521A02F01F0B55F82AA006FA0BFB1AEAC6
:102170000B0F1ABF09F802C00CF1010C09F802801C
:10218000521C262AEBDB0022002810DD17F902C0C2
:10219000BCF1000F08DBBCF1260F3ABF19F80CC0E8
:1021A00004F802C004F80280521C8242EEDBDFF821
:1021B00080A200220028CAF830E009DD14F902C02C
:1021C000944502D0CAF8304002E0521C8242F5DB4E
:1021D000DFF870B20020ABF1720404F14C0704F890
:1021E000008007F800E00BF800E0401C2628F6DB32
:1021F0000020002904DD1A5C2254401C8142FADCD4
:102200000020CDF804E0CDF800E0002912DD2256D0
:10221000002A0CDB262A0AD2530902F01F0255F8C5
:1022200023C006FA02F24CEA020245F82320401CC1
:102230008842ECDB00200246430900F01F0C55F8F1
:10224000233006FA0CFC13EA0C0F1ABF09F8002021
:10225000521C09F80080401C2628EDDB00200029D4
:102260000BDD2256002A05DB262A3CBF19F8022086
:102270000BF80020401C8842F3DB0020CAF838E04D
:10228000002909DD1BF90020824202D0CAF838B0CB
:1022900002E0401C8842F5DB11F0010F18BF252039
:1022A00015D0420900F01F0355F8222006FA03F367
:1022B0001A420AD1420900F01F0055F8223006FAEE
:1022C00000F0184345F8220001E0401EE9D5002047
:1022D0000246430900F01F0C55F8233006FA0CFCA7
:1022E00013EA0C0F1ABF09F80020521C09F80080ED
:1022F000401C2628EDDB002000290ADD2256002A9A
:1023000004DB262A3CBF19F802203A54401C8842BC
:10231000F4DB0020CAF834E00029DCBF0DB0BDE8D2
:10232000F08F3A56824204D0CAF834700DB0BDE83E
:10233000F08F401C8842F4DB0DB0BDE8F08F40F216
:10234000DB114843404901EB800070473F49C0EB37
:10235000001001EBC0007047DFF8D4C0012B8CF8EF
:1023600008008CF8091003D9401C20F00100114628
:102370008CF80A008CF80B1000FB01F24FF6FF718D
:1023800001EA4202ACF8122001EA4000ACF8140065
:1023900070472748C07A70472548807A7047244A9A
:1023A0001073517370472248407B70472048007B70
:1023B0007047274A1070517070472549085C704774
:1023C0002DE9F047DFF86890044699F805000028E9
:1023D00004BF99F801001AF029FC99F804000028BC
:1023E00008BFBDE8F0874FF00008D9F81C00474649
:1023F0004646454610F0020F1CBFDFF84C8010F037
:10240000040F05D0B9F812100F4A21F001018F18FE
:1024100010F0010F18BF0D4E10F0200F18BF0D4D1A
:10242000D9F828002060FEF75CFD10F0010F13E0E2
:10243000288400100100070068840010148900102F
:102440003A890010AC890010D48900104091001026
:10245000368400103092001006D0FEF7C7FF022825
:1024600028BF99F8020000D20020E760C4E9010803
:10247000C4E904650120BDE8F087FF48002101712F
:102480008171704770B50546FEF753FA4C2100FB89
:1024900001F21446F94928461AF0BEFB224605F51A
:1024A0000060BDE87040F6491AF0B6BBF0B583B0E5
:1024B000FEF73FFA044600210846FFF7ACF800900B
:1024C00001210020FFF7A7F800220190002C2AD953
:1024D0006E464FF0010C4FF6F07502EB4200002102
:1024E00000EB02104B0901F01F0756F823300CFADD
:1024F00007F73B4211D0CB079B0C03EB80034F083F
:1025000003EB870303F1405303F500431B889BB2A1
:10251000AB4202D903B00020F0BD491C2629E1D30B
:10252000521CA242D9D303B00120F0BD70B50D46B4
:102530000107C80E811E01EB410000EB0114D148D8
:102540004FF4987200EBC40128461AF065FBCE48A0
:102550004FF4987200EBC40105F59870BDE8704027
:102560001AF05ABB2DE9F04F00F00F07780083B046
:10257000A0F1020B0025E9464FF001084FF6F07676
:1025800047EA051A5046FEF7F2F9002843D05046B4
:10259000FFF753F808FA00F4022C88BF0224002148
:1025A0005046FFF738F8009001215046FFF733F806
:1025B00000210190002C2ED90BEB0500982200FB86
:1025C00002FA01EB4102002002EB011C420900F07B
:1025D0001F0359F8222008FA03F31A4215D000F01D
:1025E00001020AEB423202EB8C02430802EB830247
:1025F00002F1405202F51042B2F8182D92B2B242E6
:1026000003D903B00020BDE8F08F401C2628DDD39D
:10261000491CA142D5D36D1C022DB1D303B00120BA
:10262000BDE8F08F2DE9F0410026934D00280C46BF
:1026300040D000F00F01C0F3031001290EBF0021AC
:102640000229BDE8F081022828BFBDE8F0810F18FB
:10265000FEF749F95FEA00081CBF0020FEF72BF9DE
:102660000023982007FB00FC03EB4300002200EB53
:10267000031702F001000CEB4030510800EB87001B
:1026800000EB810000F1405000F51040521CC0F8F2
:10269000184D262AEDD35B1C022BE5D3B8F1000FB1
:1026A00008BFBDE8F081AE706E70BDE8F04101205A
:1026B000FEF701B9FEF717F95FEA00081CBF00201A
:1026C000FEF7F9F8002303EB4300002200EB031CA4
:1026D000D007800C510800EB8C0000EB810707F15C
:1026E000405707F50047521C3C60262AF0D35B1C7C
:1026F000312BE8D3B8F1000FD5D1BDE8F08110B58A
:10270000FEF736FF5C49088210BD5B4AC1B200F497
:102710007F43128A914288BF11464FF0640C01FB3F
:102720000CF1B1FBF2F11A0A02FB0C1110F4803F1C
:1027300012BF08B2484200B2704710B54FF4407162
:10274000524C53481AF06DFA0020012321560029FB
:1027500010DB0A09120202EB800202F1405202F57C
:1027600040420907C90ED2F800C003FA01F14CEA51
:1027700001011160401C2628E8D310BD10B5434C60
:102780004FF4407142481AF04CFA002001232156C0
:10279000002910DB0A09120202EB800202F140520A
:1027A00002F540420907C90ED2F800C003FA01F150
:1027B0004CEA01011160401C2628E8D341F67871EB
:1027C0002E481AF02EFABDE8104041F678712C48D8
:1027D0001AF027BA284810B5808B00F48170FFF7F3
:1027E00080FA4FF440712A481AF01BFA41F618514A
:1027F00022481AF016FA41F6185121481AF011FA37
:10280000BDE810400020FEF7F7BD70B51A4C054634
:10281000A06A401CA062E16A002918BFFEF7EDFF24
:10282000207850B1206A10B1206A401E2062206AD0
:10283000002804BF0020FEF73EF820212846FEF7BE
:1028400058F8616A00291CBF28468847FEF746FBF6
:10285000022827D10F48D0F8481311F0010F21D0DA
:10286000D0F8481341F00101C0F84813D0F84813DC
:1028700021F0010110E000002884001000800030E9
:1028800000A00030189D003018BD003014890010E1
:1028900000C0003000500040C0F84813A06940F06C
:1028A0000200A0610248016841F02001016070BD92
:1028B00068840010F0B40024634E012382B0002825
:1028C00008BF33701CD00128347018BF747017D043
:1028D0005E4D28685E490843286031785D4A0029CA
:1028E00014BF49F608305C48D06014BF5B484FF015
:1028F000BB7090605A48006830F0FF0C08D101E0CE
:102900007370E5E7D2F80CC060F3030CC2F80CC09A
:1029100040F2E24CA9B1906840F0180090600120AC
:10292000009004E00198471E0197FBD20098471ED3
:10293000009728BFCDF804C0F4D2906840F48050CE
:1029400090600120009004E00198471E0197FBD29F
:102950000098471E009728BFCDF804C0F4D27078C5
:1029600018B1D06840F03000D060D2F8B00040F02C
:102970000100C2F8B0000120009004E00198461E5A
:102980000196FBD20098461E009628BFCDF804C0E1
:10299000F4D2D3674FF4E0601061C2F88840002998
:1029A00018BFC2F89430D06820F03000D060906832
:1029B00020F480509060286820F0040040F00D70F2
:1029C00040F08050286002B0F0BC70472148C168D8
:1029D00021F03001C160816821F4805181601B4881
:1029E000016821F0040141F00D7141F08051016056
:1029F000704716480268164911430160124915488C
:102A00000A783AB1826842F018028260826842F421
:102A100080528260497819B1C16841F03001C160CB
:102A2000D0F8B01041F00101C0F8B01070470D4966
:102A3000C0B241EA002007490864704705494FF0D9
:102A4000204008647047000064840010008000404B
:102A5000040034120060004005F4010020009B00D7
:102A6000D0FE0300130000A0424841498161891C47
:102A7000C1614A1E4263036823F0030343F00D73F0
:102A800043F080530360436923F0010343F00D7367
:102A900043F08053436103691A430261364A8260FE
:102AA000364AC260C2681143C160354900200860DF
:102AB000704710B501F035F931480468002C08BFA3
:102AC00030BFFAD00021016001F02FF9204610BD7F
:102AD00010B501F026F92648294B2649421C1C68EE
:102AE0002CB10020186001F020F9204610BD72B60C
:102AF00048638A6120BF88614A6362B6BFF36F8F03
:102B0000BFF34F8FEBE71B48016821F0030141F051
:102B10000D7141F0805101601A49816001691A4AC2
:102B20001143016130BF704772B6114911484163CA
:102B3000C91CC161891E816162B670470D48016878
:102B4000124A1143016070470A48016821F00301ED
:102B500041F00D7141F080510160704772B6044937
:102B600004488161891CC161491E416362B6704796
:102B700000003412008000403C003412280034125F
:102B8000688400100800341201003412030034126B
:102B9000704770470022B2EBD10F26D20368B3F121
:102BA000FF3F04BF4368B3F1FF3F17D18368B3F120
:102BB000FF3F04BFC368B3F1FF3F0FD10369B3F117
:102BC000FF3F04BF4369B3F1FF3F07D18369B3F10E
:102BD000FF3F04BFC369B3F1FF3F01D0002070473E
:102BE0002030521CB2EBD10FD8D30120704710B463
:102BF0000023B3EBD20F30D2D0F800C00C68A4454C
:102C000022D1D0F804C04C68A4451DD1D0F808C02A
:102C10008C68A44518D1D0F80CC0CC68A44513D159
:102C2000D0F810C00C69A4450ED1D0F814C04C697E
:102C3000A44509D1D0F818C08C69A44504D1D0F8B6
:102C40001CC0CC69A44502D010BC002070472030C5
:102C500020315B1CB3EBD20FCED310BC01207047E8
:102C60002DE9F041054601F064F8002021264FF4DB
:102C7000825784464FF4E0221660C5F800C0116800
:102C800041F004011160116811F0040FFBD11760CD
:102C900080232C460021D4F80080B8F1FF3F04BF08
:102CA000D4F80480B8F1FF3F1DD1D4F80880B8F102
:102CB000FF3F04BFD4F80C80B8F1FF3F13D1D4F824
:102CC0001080B8F1FF3F04BFD4F81480B8F1FF3F83
:102CD00009D1D4F81880B8F1FF3F04BFD4F81C80A4
:102CE000B8F1FF3F08D0C2F800C0401CC0B20828AD
:102CF000C2D30220BDE8F081491C2034B1EBD30FD0
:102D0000C9D3C2F800C00120BDE8F0812DE9F0412F
:102D1000054601F00EF80020092684464FF4E02312
:102D20001E60C5F800C0196841F0040119601968F7
:102D300011F0040FFBD12C464FF48062002127686C
:102D4000B7F1FF3F04BF6768B7F1FF3F17D1A7682E
:102D5000B7F1FF3F04BFE768B7F1FF3F0FD1276925
:102D6000B7F1FF3F04BF6769B7F1FF3F07D1A7691C
:102D7000B7F1FF3F04BFE769B7F1FF3F08D0C3F8E1
:102D800000C0401CC0B20328CAD30220BDE8F081B5
:102D9000491C2034B1EBD20FD1D3C3F800C00120BD
:102DA000BDE8F0812DE9F05F8846814604274FF0A9
:102DB0007F0A4FF0020B4FF4E02600F0BAFF4946BD
:102DC000424653464FF0060CC6F800B052F8040BCA
:102DD00041F8040BC6F800C0306810F0040FFBD1B6
:102DE0005B1EF1D2002030604C4645461F20D4E9DE
:102DF00000C3D4E90221D5F800E0E64504BFD5F8C8
:102E000004C09C4505D1AB68934204BFEA688A427E
:102E100008D07F1E03D34846FFF722FFCDE70220EC
:102E2000BDE8F09F10341035401EE0D20120BDE80F
:102E3000F09F70B50D46044600F07BFF4FF4007222
:102E40002146284619F0E8FE012070BD2DE9F04129
:102E50000546C005ADF5007D14460E46C00D25D0D3
:102E6000A8466FF308086F4600F063FF4FF4007246
:102E70004146384619F0D0FEC5F30800C0F500778A
:102E8000A74288BF274668443A46314619F0D3FE28
:102E90004046FFF7E5FE022844D069464046FFF76A
:102EA00081FF022843D03D443E44E41BB4F5007F3B
:102EB00019D34FF400723146684619F0BCFE28461B
:102EC000FFF7CEFE02282DD069462846FFF76AFF9D
:102ED00002282CD0A4F5007405F5007506F50076DF
:102EE000B4F5007FE5D2C4B16F4600F022FF4FF485
:102EF00000722946384619F08FFE22463146684650
:102F000019F099FE2846FFF7ABFE02280AD0694661
:102F10002846FFF747FF022809D00DF5007D012064
:102F2000BDE8F0810DF5007D0A20BDE8F0810DF5CA
:102F3000007D0B20BDE8F0812E490860086100F09B
:102F400010B82C490860486100F00BB8294948675F
:102F50007047284988677047264801210166016546
:102F600070474FF04022116B10F0010F18BF21F491
:102F7000404110F0020F1CBF21F4405141F4805138
:102F800010F0040F18BF21F4406110F0080F18BFB3
:102F900041F4407110F0100F18BF41F0C00110F063
:102FA000200F18BF41F0300110F0400F18BF41F062
:102FB0000C0110F0800F18BF41F0030141F4BE0175
:102FC00041F020411163D2F8901010F4807F1CBFB3
:102FD00021F0030141F0020110F4007F1CBF21F039
:102FE0000C0040F0080141F4BE0040F02040C2F85F
:102FF00090007047001000407047D0488268D04968
:103000000A438260C2681143C1604169CD4A1143DD
:1030100041617047C948416921F0010141F00D71DA
:1030200041F080514161C16821F0400141F00D71D2
:1030300041F08051C160816821F0400141F00D7183
:1030400041F080518160704710B5BC4CA168BC480C
:103050000143A160E1680843E0606069B949084341
:103060006061B94843F63F71C160002181638164AA
:10307000C0F8B01003210A2000F0A5F90A2000F0E2
:10308000C5F9606920F0010040F00D7040F08050FB
:103090006061E06820F0400040F00D7040F080502A
:1030A000E060A06820F0400040F00D7040F08050DB
:1030B000A06010BDA44A1060516048439060704702
:1030C000A14A10605160484310F0010F18BF401C26
:1030D000906070479C49C1F8B00070479A49002839
:1030E00018BF01208864704797498863C86840F01A
:1030F0000200C8607047DFF850C2CCF82000CCF85E
:103100002410CCF82820CCF82C300120CCF830004A
:10311000DCF8340010F0010F05D020BFDCF83400DB
:1031200010F0010FF9D110F0020018BF4FF0FF307E
:1031300070478548C16821F00201C160704782482C
:10314000C16841F00101C16070477F4B186259624C
:103150009A6201201864586C10F0010F04D020BF4F
:10316000586C10F0010FFAD110F0060018BF4FF0A4
:10317000FF3070477448C16821F00101C160704799
:103180007148C16841F00401C1607047027C017B55
:1031900002F03F0241EA02416B4A916501685162C7
:1031A000416891628168D16201211165516D11F010
:1031B000010F04D020BF516D11F0010FFAD1D36D72
:1031C0008382D36D1B0CC382136E0383136E1B0C9F
:1031D0004383536E8383526EC2F30E42C28311F057
:1031E000020018BF4FF0FF3070475748C16821F008
:1031F0000401C16070475448C16841F00801C160D2
:103200007047DFF844C1CCF87820CCF82000CCF827
:103210002430CCF828100120CCF87000DCF87400C1
:1032200010F0010F05D020BFDCF8740010F0010F82
:10323000F9D110F0060018BF4FF0FF307047424838
:10324000C16821F00801C160704701684FEA31424E
:103250003D49C1F89C204068C1F8A000C86840F012
:103260002000C860704701684FEA31423649C1F812
:103270009C208088C1F8A000C86840F02000C86089
:103280007047314B18625A6299620120C3F894006A
:10329000D3F8980010F0010F05D020BFD3F89800A4
:1032A00010F0010FF9D110F0060018BF4FF0FF30F9
:1032B0007047254A106251620120C2F89000D2F88E
:1032C000980010F0010F05D020BFD2F8980010F040
:1032D000010FF9D110F0060018BF4FF0FF30704712
:1032E0001948C16821F02001C16070471648C168C3
:1032F00041F01001C1607047A3F1050C124BC3F8F7
:1033000088C018625A6299620120C3F88000D3F81D
:10331000840010F0010F05D020BFD3F8840010F016
:10332000010FF9D110F0060018BF4FF0FF307047C1
:103330000548C16821F01001C1607047008000405D
:103340004000341201003412009000401B4810B5B8
:10335000022140F8501F012101611021416241F218
:103360000601416100218161042181639021416353
:10337000416B41F0010141634FF4817101610161D1
:10338000032000F043F80021032000F01CF8002087
:1033900010BD10B5032000F045F808484FF48071C7
:1033A000016600210166102181670221416500202C
:1033B00010BD034900200870704700000030004035
:1033C0006C840010704700F00303DA004FF0FF0C2C
:1033D0000CFA02F24FF0050C0CEBC30301FA03F3F5
:1033E00000F00C0101F1E021002807DAD1F8140DFA
:1033F00090431A401043C1F8140D7047D1F80004EF
:1034000090431A401043C1F80004704700F01F01B8
:10341000012202FA01F14009800000F1E020C0F829
:103420000011704700F01F01012202FA01F140096A
:10343000800000F1E020C0F88011704700F01F010B
:10344000012202FA01F14009800000F1E020C0F8F9
:10345000801270474FF0E021C1F8000170474FF033
:10346000E021C1F8800170474FF0E020D0F8000162
:1034700070474FF0E021C1F88002704708480068AB
:103480007047074A1168106008467047044A12687E
:1034900000F1100352F8230042F823107047000097
:1034A00008ED00E002210C20FFF78DBFB8488268CC
:1034B000B8490A438260C2681143C1607047B4488A
:1034C000816821F4805141F00D7141F0805181609B
:1034D000C16821F4805141F00D7141F08051C1600B
:1034E0007047AD4881B0016F11F4007FFBD1816E50
:1034F00011F0010F1CBFD0F88410009104D0D0F857
:103500008410009A9142FAD0016F11F4007F04BF39
:103510004CF27101016642F24131816601B070479F
:103520009D4981B04FF40D528A660A6FCA66012820
:1035300098BF012005D9401EB0F5803F28BF4FF647
:10354000FF7082B24FF05C5040EA022048664FF0B4
:103550001140C1F88000086F10F4007FFBD1886E25
:1035600010F0010F1CBFD1F88400009004D0D1F8F6
:103570008400009A9042FAD0086F10F4007F04BFD4
:103580004CF27100086642F24130886601B0704723
:10359000814881B0016F11F4007FFBD1816E11F081
:1035A000010F1CBFD0F88410009104D0D0F8841013
:1035B000009A9142FAD04FF40D51816601B07047E4
:1035C0007348806810F4805008BF70477248806E5E
:1035D00000F0010070477048406EC0F30F20704744
:1035E0006D48D0F88400704710B50C20FFF726FF17
:1035F0000C20FFF70BFF68490220486710BD6649A1
:1036000010B5032088670C20FFF70CFFBDE81040C1
:103610000C20FFF713BF614A11681060084670471D
:103620005D4810B5016FC1665C480068002818BF8E
:1036300080475B48016841F48051016010BD5748E4
:1036400040687047524810B5826852490A43826008
:10365000C2681143C1605049032088670C20FFF7FE
:10366000E1FE0C20FFF7EAFE00F05CF94D4B042070
:10367000C3F888004FF6FF70C3F88C0072B6603351
:10368000FFF74EFF4FF40070186062B610BDF8B53A
:1036900072B64148016F11F4007FFBD1816E11F0C9
:1036A000010F1CBFD0F88410009104D0D0F8841012
:1036B000009A9142FAD04FF40D51816639494FF486
:1036C00000320A6662B6D1F80412314D002946D0A4
:1036D000324C4FF6FF73591AA160AA69D5F81CC085
:1036E00002F00F020CF00F0C6244121D01FA02F2FC
:1036F000A2F54341DFF8B0C0513961452FD2D0F86F
:103700008400191AE160B1F5803F28D2274B4FF0B1
:10371000000CA1FB03070CFB037301FB0C31634698
:1037200019F08EFA401C40082061B0F57A7F38BF4E
:103730004FF47A701E4B9968002908BF98605A6848
:103740001A609968C3E901108A421BD9824205D9DF
:10375000814201D9616002E0606000E0626000F0D7
:10376000EDF8A86820F4805040F00D7040F08050D3
:10377000A860E86820F4805040F00D7040F0805060
:10378000E860F8BD8242E9D88142E5D8E2E700006E
:10379000008000400010341200C00040708400100F
:1037A0006884001000A000404F62250000E1F5058C
:1037B000A89200100F4881680F4A114381600F489A
:1037C000016841F404710160001F016841F00401C7
:1037D0000160016841F0100101607047084908600C
:1037E0007047BFF34F8F084906480860BFF34F8FFB
:1037F000FEE70000008000400400341214ED00E0F9
:1038000008ED00E00400FA050CED00E015488168C1
:10381000154A114381601003416941F00101416182
:10382000016A21F00F0211490A430262104B8A1EFD
:10383000C3F8C420016570474FF04020006900F0D4
:10384000700070474FF040200A4940F8301F0A4985
:1038500041600A4901660A49416670474FF04020BD
:1038600040687047008000400400341203005FA0ED
:1038700000600040C0845FA055995FA00A005FA06F
:1038800000005FA0022824BF00207047DE4B53F8E1
:10389000202043F820101046704770B5DB4C206F95
:1038A000D94D10F0010F05D00120E06628680028EE
:1038B00018BF8047206F10F0020F08BF70BD0220B4
:1038C000E0666868002808BF70BDBDE8704000472A
:1038D000CF4810B58268CF490A438260C26811435D
:1038E000C160CA4902220A6501230B660323CB6625
:1038F0004A65816821F0800141F00D7141F08051ED
:103900008160C16821F0800141F00D7141F080516A
:10391000C1600920FFF77AFD0221BDE810400920AF
:10392000FFF751BDBA488268BA490A438260C2684B
:103930001143C160B549022008657047B3490220B0
:103940004865B348816821F0800141F00D7141F074
:1039500080518160C16821F0800141F00D7141F01A
:103960008051C1607047AA488068C0F3C01070479A
:10397000A648016F11F4007F14BF4FF440714FF45B
:1039800080710166704710B5A04CE06F10F0020F17
:103990004FF0010018BF0320606700F066F99C49F2
:1039A0008A69C96902F00F02D04001F00F01C840D6
:1039B0000521B0FBF1F04FF405710009C4F8801047
:1039C0009549A1FB00104009C4F88400206F10F451
:1039D000007F14BF4FF440704FF48070206610BD1C
:1039E0008A48016F11F4807F14BF4FF440714FF487
:1039F000007101667047854B30B4DA6F12F0010F29
:103A000014BF032202225A6700EB4005C5EBC01029
:103A1000C1EBC0004FF4FA744C43C0EB001000EB54
:103A200040007E4904EBC000A1FB00107849002251
:103A30004FF0020C8C69C008C96904F00F0401F052
:103A40000F012144C8400521B0FBF1F0B0F5803FE3
:103A500005D3511C4008CAB2B0F5803FF9D242EA02
:103A60000C2141F01001C3F88810C3F88C00186FC6
:103A700010F4807F14BF4FF440704FF4007018664C
:103A800030BC70476148016F11F4003F14BF4FF420
:103A900040314FF48031016670475C48016F11F48A
:103AA000803F14BF4FF440314FF40031016670473E
:103AB0005648006FC0F3002070475448006FC0F3B1
:103AC0004020704752498968C1F3C011002904BFE2
:103AD000002070474D4900280CBFD1F80002D1F8F2
:103AE000040270474A4B9A68C2F3C012002A04BF0E
:103AF00000207047454A00280CBFD2F88000D2F859
:103B00008800C0F30A200CBFD2F88020D2F88820A9
:103B100002F00F02D3F818C0DB690CF00F0C03F0B1
:103B20000F0363441A449140012202EB40004843D2
:103B30003949A1FB0010000970473949012008707C
:103B4000704770B4324B322251439A69D3F81CC08B
:103B500002F00F020CF00F0C6244121DD14008BF9E
:103B6000012104D0B1F5803F28BF4FF6FF719A685C
:103B7000C2F3C012002A1CBF70BC7047D3F808C043
:103B8000244A4CEA020CC3F808C0D3F80CC04CEA33
:103B90000202DA601D4A4FF0020CC2F850C04FF426
:103BA000003414660425C2F88850C2F88C101D4DEC
:103BB000D566C2F874C01C4902283CBF124E46F8B4
:103BC00020100021164801704FF400711166017831
:103BD00019B920BF01780029FBD014669567D56616
:103BE000C2F854C0986820F0800040F00D7040F09A
:103BF00080509860D86820F0800040F00D7040F050
:103C00008050D86070BC70478884001000A00040CD
:103C100000800040800034121F85EB51CDCCCCCC0D
:103C20008484001002000202EB5A00004FF0E021F1
:103C30000020886108611F494860704710B54FF047
:103C4000E02460610020A0610221401EFFF7BBFB61
:103C50000720206110BD4FF0E0210020086170476F
:103C600014480188491C01807047124880687047D9
:103C70002DE9F0410F4C002705462780A0684FF43E
:103C80007A71B0FBF1F04FF0E026401E7061B76131
:103C90000221C81EFFF797FB072030612188A94247
:103CA000FCD33761BDE8F08103494843014988608E
:103CB000704700009084001040420F00704770B5BC
:103CC00005464FF40D500406A0660320E066264822
:103CD00060664CF2710020662448C4F8800042F20D
:103CE0004630A06602210020FFF76DFB0020FFF7A1
:103CF0008DFB002D08BF70BDA06E42F2413108431C
:103D0000A06670BD012110B5880781674FF40D5181
:103D100081660020FFF786FBBDE810400020FFF71A
:103D20008DBB0120810748677047012081078867A4
:103D300070474CF271008107086670470C4A1168A1
:103D40001060084670470A4808B5006818B18047F7
:103D5000002818BF08BD4CF2710188070166016F89
:103D6000C166006F009008BD075E5F3700AF2F91FE
:103D70009C84001070B5F94D00244FF4E4612C7060
:103D80006C70EC70F64818F04CFF4FF4E461F548A5
:103D900018F047FFAC602C714C21F34818F041FF3C
:103DA0004C21F24818F03DFF6C717421F04818F076
:103DB00038FF7421EF4818F034FFEC60AC71EC610F
:103DC0002C626C62AC62EC622C632C6170BDE349C6
:103DD000002048707047E14840787047DF4800791C
:103DE000002818BF01207047DC488079002818BFE0
:103DF00001207047D9484079002818BF012070473A
:103E0000D648C078002818BF012070470021D34849
:103E1000C16201637047D848704770B5D74A0546FC
:103E2000107851784218520014462946D24818F0AA
:103E300002FF22462946D24818F0FDFEC74901205C
:103E4000887170BDC54800697047C448407800EB70
:103E50004001C1EB4010C64901EB800070472DE9DD
:103E6000F041BE4D0446C2496A78C64F02EB42009B
:103E7000C0EB4210C44E01EB80033A783078214603
:103E800010444200184618F0D6FE6A78B94902EB91
:103E90004200C0EB421001EB80033A7830782146B3
:103EA00010444200184618F0C6FE01206871BDE8B3
:103EB000F081AA48C0687047A8484078C0EBC001AC
:103EC000C1EB8010A64901EB401070472DE9F0418D
:103ED000A24E07463078002814BFAC48AC4804789E
:103EE00014BFAC48AC48057804FB05F8FFF785F82B
:103EF00029462046FFF7DEF870789A4CC0EBC001E7
:103F0000C1EB801004EB4012A4F5E46101EB40101A
:103F10003B460146FFF7EFF8FFF77CF870784FEA71
:103F20004802C0EBC001C1EB801004EB40103946E1
:103F300018F081FE0120F070BDE8F0812DE9F04716
:103F4000864D044686496A78DFF84082C2EBC2009B
:103F5000C0EB821001EB40132878DFF834928D4ECD
:103F60008D4F002815BF98F8000099F800003278AE
:103F70003A7800FB02F04FEA40022146184618F05A
:103F80005AFE6A787749C2EBC200C0EB821001EB9F
:103F9000401C28782146002815BF98F8002099F881
:103FA000002033783B7802FB03F04FEA4002604682
:103FB00018F041FE0120E870BDE8F087674880688E
:103FC000704770B5754C0546014622786648520028
:103FD00018F031FE227829465200644818F02BFE72
:103FE0005E490120087170BD2DE9F04FADF26C7D86
:103FF000DFF868910120CDF84C0799F80300CDF85F
:10400000480799F80400CDF8440799F80500CDF861
:10401000400799F80600CDF83C0701F0BDFB80464B
:10402000FDF7B2FDCDF86407FDF788FFCDF8600716
:10403000FDF7ECF9CDF85C07FCF753FF0446FCF7FD
:104040004DFF0746FDF7A2FD99F802001E26002548
:10405000002804BF0420C9F8180008D0B8F1020FE6
:1040600018BF0A200ED0C9F8180089F80250FDF7D1
:1040700094F9083000094FF0010BCDF85007022FDA
:104080000AD023E011F03EFC10F4817F14BF0F2012
:10409000C9F81860E7D1E8E7B8F1020F03D0B8F12A
:1040A000050F08D012E04FF47A71484390FBF1F00D
:1040B000C9F8180008E01220C9F8180011F0C7FC70
:1040C000002818BFC9F8186089F802B0D9F818009C
:1040D0000428BCBF0420C9F8180099F80200B9F8F8
:1040E0001810000240EA014040F001020023912133
:1040F00007200AF059F814F0010F51D1B8F1020F5E
:104100004ED00020FDF778F9FDF757FF18F09DFD20
:1041100000252F46CDF8385705F0F4FD012845D08D
:104120000DF5E460FEF74CF9002800F0DD820DF596
:10413000E46006F0ECFC002089F80100D9F81800D2
:10414000C01E8542CABF874201240024DDF82C0727
:1041500018B1DDF8440770B359E058E0A0840010AE
:10416000B4920010D499001034AF001080AF00104A
:10417000CCAF001040B00010BC84001006850010C9
:10418000C484001003850010048500100185001010
:10419000FE84001002850010FF84001005850010C9
:1041A000FDF7D2FE0020CDF84C07AFE70120CDF897
:1041B000380700F083BAFFE7DDF82CA77CB1FA4E90
:1041C000514630784200F94818F035FD30785146B4
:1041D0004200F74818F02FFD89F804B017E0FEF709
:1041E0000CFFF14E01213078FEF764FFF04A534690
:1041F000A2F14C010846FEF77EFFFEF70BFF307878
:1042000051464200EA4818F016FD89F804B0DDF87E
:104210002807002800F0D780DDF84807002840F084
:10422000D28099F80000DDF82867E0BBD9F808A033
:10423000BAF1000F24D0DF480078CDF85807DE48E7
:104240000078CDF85407FEF7D8FEDDF85417DDF8F6
:104250005807FEF735FF314652460846FEF775FF10
:10426000FEF7D8FED5480078022804BF504606F075
:104270001EF9D2480078092804BF304606F017F925
:10428000CF480078012816D9DFF830A39AF800004B
:10429000042804BF304606F00AF93146684618F093
:1042A000D9FC064600E006E09AF80000052804BFA5
:1042B000304606F0FCF8CCB399F8010099F80020DC
:1042C000C0EBC001C1EB8011BE48002A00EB4110D9
:1042D00031460CBFBC4AB74A137814BFB64ABB4A32
:1042E000127803FB02F24FEA420218F0A4FC99F89C
:1042F0000100C0EBC001C1EB8011B54800EB4113D8
:1043000099F800003146002814BFAA48AE4800784A
:1043100014BFA94AAD4A127800FB02F04FEA4002EE
:10432000184618F088FC89F803B03DE0FFE7CDF8A7
:10433000546799F80000002814BF9E48A24890F8DE
:1043400000A014BF9C48A14806780AFB06F0CDF8EF
:104350005807FEF752FE31465046FEF7ABFE99F87D
:1043600001009B4EC0EBC001C1EB801006EB401278
:10437000A6F5E46101EB40100146DDF85437FEF785
:10438000BAFEFEF747FEDDF85807420099F8010033
:10439000C0EBC001C1EB801006EB4010DDF85417F4
:1043A00018F049FC89F803B08448007803280AD142
:1043B00099F80100C0EBC001C1EB8011814800EB0E
:1043C000411006F074F8DDF8300700287DD0DDF8E4
:1043D0004007002879D199F80000DDF8306748BB24
:1043E000D9F80CA0BAF1000F24D07A4801787A48A5
:1043F00000780844401C4008019002200090FEF71D
:10440000FCFDDDE90010FEF75BFE31465246084632
:10441000FEF79BFEFEF7FEFD70480078022804BF01
:10442000504606F052F96D480078092804BF30461E
:1044300006F04BF94CB399F80100DFF898A100EBB6
:104440004001C1EB401166489AF8002000EB81035F
:1044500061483146007810444200184618F0EBFBE2
:1044600099F801005C4A00EB4001C1EB40115D4846
:104470009AF80030127800EB81001A44314652005D
:1044800018F0D9FB89F805B030E052480096017861
:10449000514800780E18FEF7B0FD701C400802214C
:1044A000FEF708FE99F80100DFF838A100EB4001A3
:1044B000C1EB4010AAF174010AEB800201EB80010C
:1044C0000846009BFEF717FE00E01EE0FEF7A2FD87
:1044D00099F80100720000EB4001C1EB40100AEBBB
:1044E0008000009918F0A7FB89F805B03B480078D8
:1044F00003280AD199F8010000EB4001C1EB4011FB
:10450000374800EB810006F0E0F8DDF834070028BA
:1045100073D0DDF83C0730B1B8F1020F18BFB8F125
:10452000050F6BD0BDE099F80000DDF8346740BBA3
:10453000D9F810A0BAF1000F23D02B4801784078A9
:104540000844401C4008019002200090FEF755FDF1
:10455000DDE90010FEF7B4FD314652460846FEF78D
:10456000F4FDFEF757FD21480078022804BF5046AD
:1045700006F0CAF91D480078092804BF304606F045
:10458000C3F9194801784078B4B30844440022467E
:104590003146174818F04FFB22463146154818F0AF
:1045A0004AFB89F806B042E00585001034AF0010E0
:1045B00080AF001001850010028500107D8500107D
:1045C00000850010B4920010FE840010FF840010DB
:1045D000D499001003850010048500108285001016
:1045E000CCAF001040B00010068500108785001089
:1045F000BC840010C484001001E052E028E00C18D4
:10460000FEF7FBFC601C40080221FEF753FDFB4A4D
:104610003346A2F108010846FEF76DFDFEF7FAFCED
:1046200062003146F54818F006FB89F806B0F448F8
:104630000078032804BFF34806F066F918F00FFB72
:104640000020C9F82C00C9F8300000F086FE28E0F0
:104650000021DDF8340718F007FBDDF85007782853
:1046600028BF15F0010F1CD0E74C207A58B1082064
:10467000FCF7AEF8E54A1378527899184A000146DB
:104680000820FBF752FEE07958B10720FCF7A0F8AC
:10469000DE4A01460720137852781A445200FBF78D
:1046A00044FEFDF7EAFED9F818006D1C7F1C854218
:1046B000A8BF874211DBD9F8140070B1FDF766FA84
:1046C000DDF85C07FCF798FEDDF8640788B1DDF8DB
:1046D000600760B1FDF771FC0BE0DDF84C070028C6
:1046E00018BFFDF76AFC17E501F0A3F814E5FDF724
:1046F0002BFCDDF83807002804BF0420C9F8180097
:104700000FD0DDF8480789F80300DDF8440789F881
:104710000400DDF8400789F80500DDF83C0789F85A
:104720000600DDF83807B9F81810000240EA014227
:1047300000239121072009F037FDDDF838070DF23D
:104740006C7DBDE8F08F10B50024FDF7E9FBB049A2
:1047500010F0020F0AD0CA78002A08BF012410F016
:10476000040F03D00A79002A08BF012410F0010FBA
:1047700003D04A79002A08BF012410F0200F03D08B
:104780008879002808BF01240020002C08BF10BD34
:1047900000200870BDE8104026E438B505460F2417
:1047A00011F0B0F840B100F0F7FF022803D000F09C
:1047B000F3FF052800D10E242146284601F047F9D1
:1047C000012804D1FFF7BFFF009001F0B9FA90482B
:1047D000C17800291CBF4179002906D081790029C0
:1047E0001FBF00790028012038BD002038BDD4E764
:1047F000704770B5864C00250646E57025716571D9
:10480000FCF737F8002818BFA571002E1CBF012047
:10481000A070BDE870400AF098B9002818BF0120C8
:104820007B49C87170477A48C079704710B54FF41A
:10483000E461784818F0F5F9BDE810404FF4E46100
:10484000754818F0EEB92DE9F041714D069A2978B6
:10485000002914BF714972490978D21A4A4303FBEF
:1048600001F469785200C1EBC103C3EB8111694BBC
:10487000164603EB411101EB440300EB44010F46E4
:10488000184618F0D8F968783246C0EBC001C1EB81
:104890008010614901EB401000EB4400394618F0EC
:1048A000CAF90120E870BDE8F0812DE9F047584FC2
:1048B000804608983978002914BF584958490D781E
:1048C000A0EB030905FB09F603FB05F4FEF795FBD6
:1048D00049462846FEF7EEFB78784F4DC0EBC00105
:1048E000C1EB801005EB401101EB4402A5F5E4613A
:1048F00001EB401000EB440008EB4408434601463E
:10490000FEF7F9FBFEF786FB78787200C0EBC0017A
:10491000C1EB801005EB401000EB4400414618F05D
:104920008AF90120F870BDE8F0873E4870473C489E
:1049300001783D480078484341003A4818F071B981
:1049400070B506463648047837480578FEF755FBBB
:1049500029462046FEF7B4FB2D484078C0EBC00145
:10496000C1EB80102B4901EB401231462D48FEF778
:10497000ECFBFEF74FFB2D480078152818BF70BDE3
:104980002848BDE8704005F092BD002818BF0120FE
:104990001F49C870704710B51D4C002804BFA060A7
:1049A00010BDDFF88CC01D490B7822490A780146FA
:1049B0005A435200604618F03EF91D48A06010BDF1
:1049C00010B54C211C4818F02CF9BDE810404C21C2
:1049D0001A4818F026B918487047002818BF012057
:1049E0000B490871704710B57421154818F019F972
:1049F000BDE810407421134818F013B9C4840010A6
:104A000087850010BC840010F8880010068500100F
:104A1000A0840010B4920010D499001001850010F9
:104A2000FE840010F4A00010FF8400107D850010AB
:104A300014A800100285001034AF001080AF0010E1
:104A4000CCAF001040B00010002818BF0120FB4977
:104A50004871704710B5F94C002804BFE06010BDE4
:104A600074220146F64818F0E6F8F548E06010BDFB
:104A7000F2480021C161016241628162C162016349
:104A80007047002818BF0120EC498871704710B5A5
:104A9000EA4C002804BF206110BDEA490A78497831
:104AA00011444A000146E84818F0C5F8E64820617C
:104AB00010BDE6487047E34A0146E448137852784F
:104AC0001A44520018F0B7B830B44FF0000C029CF2
:104AD000634304BF30BC704732F91C4051F82C507E
:104AE0002C4440F82C400CF1010C6345F4D830BC48
:104AF0007047002B08BF704710B4DDF804C0BCF14C
:104B0000000F4FF0000C11D0002A9CBF10BC704762
:104B100051F82C4004EB5304B4FBF3F420F81C4090
:104B20000CF1010C6245F3D810BC7047002A9CBF01
:104B300010BC704751F82C4094FBF3F420F81C4053
:104B40000CF1010C6245F5D810BC704770B5BB4D37
:104B500000260446EE702E716E71FBF78AFE002867
:104B600018BFAE7109F0F1FF002C14BF0120002026
:104B70002870BDE87040FFF737BA2DE9F04F8FB0CD
:104B80004FF4E461B24818F04CF87421AC4818F0C6
:104B900048F8AA4E00207063B06300900190029024
:104BA0000390FDF7BDF90446FCF7EEFF0C90FDF70E
:104BB000C5F90B90FCF72AFC0A90FCF7E7FF0020F0
:104BC000FCF71AFCFDF7F9F900273D4605F09AF8C5
:104BD000012878D004A8FDF7F3FB002872D004A8C0
:104BE00005F095FF14F0020F1DD099480D908346F3
:104BF0009848DDF818A090F80080974890F8009049
:104C0000FEF7FBF90120FEF769FA49464046FEF738
:104C100057FA5A4651460D98FEF797FA0020FEF7CC
:104C20005DFAFEF7F7F914F0010F21D084480D90DA
:104C300083468A484FF00209DDF820A001788848B1
:104C400000780844401C4FEA5008FEF7D6F90120CE
:104C5000FEF744FA49464046FEF732FA5A465146B4
:104C60000D98FEF772FA0020FEF738FAFEF7D2F937
:104C700014F0200F1DD073496B46099891F800C0BD
:104C800049781A466144491C4FEA510C00214FF003
:104C900002085FEA4C0918BF0CFB08FC09D030F988
:104CA000118052F82190C84443F82180491C8C455A
:104CB000F5D8FDF7E2FB7F1C102F05D2FDF77DF93B
:104CC00084E700E00CE00125FCF760FF0A98FCF7A0
:104CD00093FB0C9848B10B9828B1FDF76EF904E0EE
:104CE00000F0A7FD72E7FDF72FF9002D52D114F067
:104CF000020F18D05748564B017857489C46007809
:104D000001FB00F210200021002A0AD93CF9118091
:104D100008EB5008B8FBF0F723F81170491C8A42E1
:104D2000F4D84B48B06014F0010F18D04B48444BF6
:104D300001784B481F4600780A184FF010004FF0DA
:104D400000010AD037F9118008EB5008B8FBF0FCDD
:104D500023F811C0491C8A42F4D83948F06014F095
:104D6000200F17D03748384C6B46017840780A1826
:104D70004FF010014FF000000AD053F820C00CEBA8
:104D8000510CBCFBF1FC24F810C0401C8242F4D84A
:104D90002D4830610FB02846BDE8F08F01207047E4
:104DA0004FF43F3070474FF43F30006870474FF486
:104DB0003F310A68B2F1FF3F15D0052804BFC87A19
:104DC000704728DC012804BF08797047022804BF17
:104DD000087A7047032804BF487A7047042804BF44
:104DE000887A704727E0052813D007DC012822D0F5
:104DF00002281CBF032804280BD01CE0142812BF73
:104E000015282D207047162804BF28207047172822
:104E100011D100207047142804BF087B7047152863
:104E200004BF487B7047162804BF887B704717284B
:104E300004BFC87B7047FF2070470000A0840010AB
:104E4000B4B0001006850010D4840010CC8400108B
:104E500014A80010018500100285001003850010C1
:104E60000485001070B5ADF5007D00244FF400718D
:104E7000684617F0D6FE4FF43F36FF224FF400711C
:104E8000684617F0F6FEFF21254661F307052D223F
:104E9000214662F3070162F30F2128224BF6BB3053
:104EA00062F3174164F31F61CDE90005CDE90241CA
:104EB00004943046FDF7D4FE69463046FDF772FF94
:104EC0000DF5007D70BD2DE9F04F4FF43F34ADF589
:104ED000017D834620688A9F984691468A46B0F1B4
:104EE000FF3F08BFFFF7BEFFD4E901106AF30700D8
:104EF00069F30F20256868F31740D4E903646BF366
:104F0000070167F31F608B460746FF224FF40071CD
:104F1000684617F0AEFE0297CDE90364CDE9005B69
:104F20004FF43F342046FDF79BFE69462046FDF7CF
:104F300039FF012818BF00200DF5017DBDE8F08F75
:104F40002DE9F04F4FF43F3389461D680021ADF540
:104F5000017D90468246B5F1FF3F02BF08460DF540
:104F6000017DBDE8F08FFF22D3E902744FF4007198
:104F70006846D3F810B05E6817F07BFE6AF307044A
:104F800069F30F2468F31744012060F31F64CDE92F
:104F90000274CDE900564FF43F34CDF810B02046EE
:104FA000FDF75EFE69462046FDF7FCFE0DF5017D2E
:104FB000BDE8F08F2DE9F04F4FF43F30894E0025CA
:104FC0000368ADF5017D74422F461720FFF7EFFE11
:104FD00084461420FFF7EBFE40B2B3F1FF3F04D04C
:104FE000BCF1000F03D12D2801D0FFF73BFF1420A7
:104FF000FFF7DDFE40B202901520FFF7D8FE4FFA12
:1050000080F91620FFF7D3FE40B201901620FFF77B
:10501000CEFE404240B20090FCF782FFDFF8C8A10C
:10502000834600208AF803008AF804008AF8050005
:10503000FBF71FFC00281CBF00208AF8060009F0BF
:1050400084FD00208AF80000FEF7CEFF1BF0010F60
:1050500004D017F013FE012808BF01251BF0020F32
:105060007ED062489AF801104FF0000890F800C016
:105070005F48C1EBC102C2EB811100785D4A002894
:1050800002EB4112C8BFACF1010A1EDD0021BAF1EA
:10509000000F16DD01F1010B01FB00830BFB008B00
:1050A00032F8133032F81BB0A3EB0B031BB2002B0A
:1050B000B8BF5B421BB2BB42C8BF1F46491C51452B
:1050C000E8DB08F101088045E0DBB945B8BF45F0F1
:1050D00002054FF00008C146BCF1000FC8BFA0F1A7
:1050E000010A1BDD0021BAF1000F13DD09FB0013DB
:1050F00032F813B002EB43035B88ABEB03031BB244
:10510000002BB8BF5B421BB24345C8BF9846491C41
:105110005145EBDB09F10109E145E3DB029941452A
:10512000B8BF45F004054FF00009BCF1000F13DDD6
:10513000002300280CDD09FB003132F91110B142C7
:10514000C8BF0E46A142B8BF0C465B1C8342F2DBCF
:1051500009F10109E145EBDB0198B04204DB00E015
:1051600004E00098A04201DD45F00805604208F027
:10517000FF0B4FF43F3400F0FF08206807F0FF0AF0
:1051800006F0FF09B0F1FF3F08BFFFF76BFED4E95F
:1051900001106BF307006AF30F20266869F31740CC
:1051A000D4E9037465F3070168F31F600D46804678
:1051B000FF224FF40071684617F05BFDCDF80880C0
:1051C000CDE90374CDE900654FF43F342046FDF787
:1051D00047FD69462046FDF7E5FD0DF5017DBDE87B
:1051E000F08F0000F1D8FFFFA0840010FF840010B2
:1051F000FE840010B4920010FE4800897047FD48FC
:105200004089704770B515460E46044609F025FDE5
:10521000002C18BF70BD042806D0F748006890F82D
:105220002400A84288BF70BD3046BDE8704017F02A
:105230002ABD2DE9FF5F8346F0480027DDF838A03E
:1052400005780398109EB9463C4650452CD006FB85
:10525000050E0F983BF91EC006FB05093BF9190026
:10526000BCEB000348BFA0EB0C0306FB05A83BF911
:105270001840B4EB000C48BFA0EB040C03EB0C008F
:1052800004B231F91EC031F91900BCEB000348BF6C
:10529000A0EB0C0331F918C0BCEB000148BFA0EB38
:1052A0000C0158180FFA80F9012A2DD04FF001088F
:1052B00017F0EEFCD249002C0A782EDD0F9906FB80
:1052C00005113BF911101431282926D9039902EB55
:1052D0000A0C11448C4520D9119B129D13442A4479
:1052E0008B421CBF8D1A15F1020F30F9115000EBE3
:1052F0004106B6F90260A5EB060508D01E353C2D27
:1053000008D94FF0000808E0A1450CDD0AE00A3595
:10531000142DF6D8491C8C45E2D8A14503DDB8F11F
:10532000000F00D0012704B03846BDE8F09FB14817
:105330000021817181817047B24A02804280002140
:105340008280C1800181534243818181C181018278
:105350004182C182018382827047A6490020C881B0
:1053600008617047A3480021416181617047A648E8
:105370007047A64A0146A448137852781A4452004E
:1053800017F059BC2DE9F04383B00C460546FFF7F2
:1053900090FB02469C480021031F002C88BF4FF061
:1053A000010C0AD95E5C2EB935F911603C2EA8BFFC
:1053B00003F801C0491CA142F4D38E4EB6F80E800A
:1053C000B8F1000F09D10021002C06D935F811C021
:1053D00020F811C0491C8C42F8D80021EC46002C62
:1053E0000AD935F8117030F81190A7EB09072CF89D
:1053F0001170491C8C42F4D8B8F11E0F24BF002153
:10540000002C11D9585C00281CBF3CF9110010F188
:10541000140F06DD142804DC32F81170384422F829
:105420001100491CA142EDD31046FFF744FBF0895F
:1054300042F2107188423ABF401CF081F1817348FA
:10544000294602784078104442006F4817F0F3FB79
:1054500003B0BDE8F083009800140028CCBF012001
:10546000002070472DE9F047814617F016FC0546ED
:1054700062482824012706784FF0060A4FF00908F1
:1054800000F08AF9052808BF32240AFB067035F9B6
:105490001010A142D8BFBDE8F08705EB4000B0F97D
:1054A00002008442D8BFBDE8F08708FB067035F9DA
:1054B0001010A142D8BFBDE8F08705EB4000B0F95D
:1054C00002008442D8BFBDE8F0874FF0FF30C9F832
:1054D00000004848C770BDE8F0872DE9FF4F85B050
:1054E0001F46DDE9129A90460446DDF854B009F0F3
:1054F000B4FB09F03BFB00253E4E00285ED010F0C7
:10550000A6FA002834D017F0C8FB82463B48062193
:105510004FF0280990F800B0012004900290092073
:105520000091039000F038F9052808BF4FF03209C8
:105530000099049801FB0B003AF91010494517DD5A
:105540000AEB4000B0F90200814511DDDDE90210EF
:1055500000FB0B103AF91010494509DD0AEB400039
:10556000B0F90200814503DD01204FF0FF34F070F7
:10557000B4F1FF3F00F0D680002C07BF70780128FF
:1055800009B0BDE8F08F757009F067FB042800F0E2
:10559000DF8005F0CEFC04287ED0B8F1000F1CBFE0
:1055A0004046FEF7CBFC002F04BF09B0BDE8F08FEA
:1055B000384609B0BDE8F04FFEF751BC09F074FC65
:1055C000009009F0BFFA002804BFB571B58130D052
:1055D000B6F90C008345C8BFA6F80CB0B6F90C00AC
:1055E0000B4900EB801081FB00104111A1EBE07032
:1055F00058450FE0DC84001064860010FE84001023
:1056000004850010F1D8FFFFF0840010068500101B
:105610001F85EB5125DD0098012822D0B079401C70
:10562000C0B2B071032804D9B5710120B581F07002
:10563000841E069803900A2002904E48DDF850B070
:10564000BAF1010F007800904B480078019008BF34
:10565000BBF1000F07D0308948B309F0C1FA40B15F
:1056600025E0B571E5E77079052824BF0520707144
:105670003CE0B9F1010F02D17089C82817D87089B0
:10568000002804BF3089002811D009F05BFA0128F6
:1056900018BF1E210DD000E05AE0DDE900230020F4
:1056A000D31817D0039A32F910208A420EDD757193
:1056B0001CE0BBF1010F08BF4121ECD005203C21CB
:1056C0000290B9F1000FC8BF3221E4E7401C80B25C
:1056D0008342E7D87079401CC0B270710299814250
:1056E00004D20120F0704FF0FF34757109F02AFAEE
:1056F00001287FF43DAFB9F1000FC8BF35713FF706
:1057000037AFBAF1010F3FF433AF3079401CC0B26C
:1057100030710A287FF62CAF0120F0704FF0FF3473
:10572000357125E7F07801281CBF09B0BDE8F08F7E
:105730004046FFF705F9F570B8F1000F1CBF404671
:10574000FEF7FCFB002F7FF433AF09B0BDE8F08F0C
:10575000B8F1000F1CBF4046FEF7B8FB002F04BF96
:1057600009B0BDE8F08F384609B0BDE8F04F17F03A
:1057700099BA0000038500100485001010B506F0EA
:10578000DDF906F086FA002010BD0000FE498870A1
:105790007047FD4880787047FB4800787047FA48AA
:1057A00040787047F8480078022805D005281CBFCB
:1057B0000020704705F0BDBB09F04FBAF2490870F0
:1057C000704770B5F04E04460D463078A04212D0B6
:1057D00002281AD0052814BF002005F0AAFB44EACD
:1057E00005213278002341EA024141EA0062612149
:1057F000072008F0D9FC7570072C28BF70BDDFE8C2
:1058000004F016070B13160F160009F026FAE6E748
:10581000284600F0A3FA0AE0284609F019FA06E043
:10582000284605F07BFB02E0284608F075FD347041
:1058300070BDD64900200968B1F8641011F4807F6A
:1058400008BF7047FDF735B9D04900200968B1F8A5
:10585000641011F4807F08BF7047FDF739B9CB4958
:1058600000200968B1F8641011F4007F08BF704788
:1058700017F01DBAC54900200968B1F8641011F489
:10588000806F08BF704717F017BABF49C878002863
:105890001CBF401EC870704770B5BD49D1F8CC0020
:1058A000B94C10F0030F0AD040F4BE0040F0204085
:1058B000C1F8C800E078002804BF0120E070B548B6
:1058C0008068B24D10F0020F296807D14FF04020D8
:1058D000406910F0010F01D0E07840B1B1F86410D8
:1058E000002011F4807F18BFFDF7F2F807E0B1F84F
:1058F0006410002011F4806F18BF17F0DDF9A6497D
:10590000084208BF70BD2968496E090CE17070BD7E
:1059100010B572B6FEF7F6F9BDE81040FDF761BFAD
:1059200010B5012802D0022805D008E04FF443301A
:10593000FDF796F903E04FF040219848086772B6EA
:10594000FEF7E0F9BDE81040FDF74BBF8E49002897
:105950000A7918BF01200871C0B2824208BF70479F
:105960000022002818BF012200230121022008F094
:105970001BBC85480079002818BF01207047824869
:10598000407970472DE9F0417F4E00281CBF002070
:10599000707104D17079002818BFBDE8F0814FF014
:1059A00040273D6B0120FDF7CCFA0420FDF7C9FA32
:1059B0007B4C0520E066FEF7BCF940F2CF70216F0A
:1059C00011F0010F04D0707940F00E00707103E007
:1059D000011EA0F10100F2DC707978B1FEF7A9F99F
:1059E0007048216F11F0040F04D0707940F001006D
:1059F000707103E0011EA0F10100F2DC45F4BE006D
:105A000040F020403863BDE8F0815F48406970474E
:105A10005D48006970475C480069002818BFC07A7B
:105A2000704759498861704757488069704756499F
:105A3000C86170475448C06970475448026802F50D
:105A4000C073118A508A02F5A072FCF744BB2DE99D
:105A5000F04FDFF8349197B08A46C9F8140005F08A
:105A60008FFFC9F81000002800F0B78090F800C040
:105A700089F806C0417889F80710837804460CF14C
:105A8000010089F8083000F0FE0089F80900E2788A
:105A900089F80A20207989F80B00607989F80C00D0
:105AA00009F10E05A0792870E0796870207889F8EE
:105AB0000D006046FCF750FC99F80C1099F80B00AB
:105AC000FCF76DFC69782878FCF773FC6946204682
:105AD00005F07FFF608AD9F8185000281CBF684382
:105AE000050BB4F81A80D9F81C60B8F1000F08BF94
:105AF0004FF48058678C002F08BF4FF48057002068
:105B00001AF0040F18BF4FF485701AF0080F18BF71
:105B100040F004001AF0020F1CBF40F201210843BC
:105B20001AF0010F18BF40F48460616A6FF30F0A26
:105B300008406FF30F0108434AEA000A00981090EA
:105B400004981190089812900C9814900198139052
:105B50000798159010A95046FCF7E6F81AF0020FC6
:105B600077D005F00CFC5FEA000B43D005F01EFC7B
:105B70006843050B59460020FBF75DFC218A00298C
:105B800018BF002010E00000F884001064860010A8
:105B9000006000400080004008000300AD2007B016
:105BA000001000403F0D030018BFFBF7C3FC05F0D9
:105BB0001DFC7043000B8030020A0820012101FA0D
:105BC00000F3134201D1401EF9D5061FA07B002827
:105BD00018BFA0F1010B17D112E05E480068B0F8C1
:105BE000640010F4807F18BFFCF772FF002017B02C
:105BF000BDE8F08FB4F80CB0BBF1000FBAD1BDE72F
:105C00000020FBF71AFD8346E07B002814BF401EEE
:105C1000FBF754FD0BEB0601042903DD711A0E1D81
:105C2000042103E00029BCBF761A00210644042E9B
:105C300003DD301FC540042604E0002E02DA704266
:105C4000854000260020FBF711FD31460020FBF7C0
:105C50004EFD1AF0010F23D0A18A00291CBF01209C
:105C6000FBF7E9FB268B3EB131460120FBF762FCD6
:105C700031461120FBF75EFCA67D3EB1711E01206E
:105C8000FBF7F4FC711E1120FBF7F0FCE67D3EB142
:105C9000711E0120FBF72BFD711E1120FBF727FD64
:105CA0001AF0200F23D0A18B00291CBF0220FBF784
:105CB000C2FB268C3EB131460220FBF73BFC31464D
:105CC0001220FBF737FCA67F3EB1711E0220FBF7C6
:105CD000CDFC711E1220FBF7C9FCE67F3EB1711EA0
:105CE0000220FBF704FD711E1220FBF700FDE07A95
:105CF00000281CBF0001FBF7DAFA029805F01BFB35
:105D0000039830B12B4699F8072099F8061016F041
:105D1000D8FF3A464146284616F0D8FF0598FEF7C8
:105D20003AFE0998FEF796FE05F050FE10F4005F6B
:105D30001CBF0D98FEF7ABFE012017B0BDE8F08F39
:105D400010B5FCF7AEF805F0FEFA03490020086133
:105D5000012010BD64860010F8840010FE49087010
:105D60007047FD4800787047FC4810B4FC4A016851
:105D7000914218D14168B1F5907F14D80022D0F833
:105D800008C003461146B2EB9C0F24BF10BC7047FD
:105D900053F82140491C2244B1EB9C0FF8D3002A50
:105DA00004BF10BC7047002010BC7047EB48FCF7E4
:105DB00057BF2DE9F041ADF5007D044605F0C0FD6B
:105DC00040B181692162C16961624169A162C068B3
:105DD000E06205E04FF0FF30E062A06260622062A6
:105DE00038250020C4E90250DD4F4FF49076C4E915
:105DF0000076224601462B4652F820C0401C6144E2
:105E0000B0EB930FF8D3C1F10008FF224FF40071FB
:105E10006846C4F80C8016F02CFFCDF80C80009773
:105E2000CDE9016510340DF110080FCC88E80F00A2
:105E30000FCC0DF1200888E80F00D4E90001C74C11
:105E4000CDE90C012046FCF70BFF69462046FCF724
:105E5000A9FF012818BF00200DF5007DBDE8F081E5
:105E6000BD4901200870704770B50E4605461024E4
:105E7000FFF7CEFD15F0020F18BF052408D115F06D
:105E8000010F18BF092403D115F0200F18BF0D24EE
:105E90003246102C28BF70BD002A08BF70BD2044B8
:105EA00090F928102046BDE8704005F0C5BDF0B55A
:105EB00081B0ADF5805D0446FFF7AAFD054614F0FC
:105EC000020F0AD0684604270646FCF7DBFA95F96C
:105ED0002C103246384605F0AFFD14F0010F0BD000
:105EE000694608270E460120FCF720FB95F9301083
:105EF0003246384605F0A0FD14F0200F02BF01B075
:105F00000DF5805DF0BD0C2669460C460220FCF7BD
:105F10000DFB95F934102246304605F08DFD01B099
:105F20000DF5805DF0BD2DE9F34FE9B000208A4604
:105F30005690559072B6FBF7F3FF0546FDF713FD3B
:105F400048B1FDF7B5FD5690FDF79CFDFDF7B5FD99
:105F50005590FDF7A2FDFBF7DCFEFBF715FE5D900B
:105F6000FBF7ECFF5C90FBF711FEFCF776F8649012
:105F70000020FCF76CF80120FBF72FFC6290112049
:105F8000FBF72BFC63900220FBF727FC60901220AC
:105F9000FBF723FC6190FDF713FB5B90FDF7F8FA2C
:105FA0004FF49350FDF765FA62B6FBF701FC5A9087
:105FB0000120FBF7F3FB0120FBF773FC6590002049
:105FC000FBF72DFE5F900020FBF71CFE5E9000208B
:105FD000FBF712FA66900020074636AE46F82070AE
:105FE000401C0628FAD3DFF87C8115F0020F4FF031
:105FF00001040AD041F618514046369416F011FEBD
:1060000041F61851584816F00CFEDFF8609115F073
:10601000010F15D04FF41871554816F002FE4FF4D9
:106020001871484616F0FDFD0120FAF7A0FC002883
:1060300018BF38941120FAF79AFC002818BF399439
:1060400015F0200F15D04FF41871494816F0E9FDEE
:106050004FF41871484616F0E4FD0220FAF787FC69
:10606000002818BF3A941220FAF781FC002818BFC4
:106070003B94DFF80091384D36984FF0405B68B3A1
:1060800000210846FBF7C7FA009001210020FBF72A
:10609000C2FA019099F800008DF80800364800789F
:1060A000012894BF3548364800788DF80900002053
:1060B000FBF7DEFB002818BF4FF0FF3004908DF88F
:1060C0000AA06888ADF80C000020FBF751FAADF883
:1060D0000E002C48CDF81880CDE907B037984FF066
:1060E000FF0A68B300210846FBF795FA09900121E1
:1060F0000020FBF790FA0A9099F800008DF82C0028
:106100008DF82D400D978DF82EA06888ADF83000E1
:106110000020FBF72DFAADF832009DF8090000EBE6
:10612000400101EB001108EB81010F919DF808106F
:1061300048430BEB40011091124901EB40001190D4
:10614000114FDFF848803898F0B300210120FBF7A9
:1061500062FA012112901BE01885001000FE020077
:10616000544352460080003000A0003018BD00307B
:10617000189D00300185001000850010FF8400107C
:1061800002850010004000300385001004850010D7
:106190000846FBF740FA1390FAF7BDFE00280CBF43
:1061A00098F8000038788DF850000120FBF745FA88
:1061B00004FA00F08DF851000120FBF70EFBC043FC
:1061C00016908DF852A000E00DE0A888ADF85400BC
:1061D0000120FBF7CDF9ADF85600FE481890FE48B7
:1061E0001990FE481A90399870B300211120FBF7DE
:1061F00012FA1B9001211120FBF70DFA1C90FAF7FF
:106200008AFE00280CBF387898F800008DF87400DA
:106210001120FBF712FA04FA00F08DF87500112036
:10622000FBF7DBFAC0431F908DF876A0A888ADF885
:1062300078001120FBF79CF9ADF87A00E84821902E
:10624000E8482290E8482390E84F3A9840B300216C
:106250000220FBF7E0F9249001210220FBF7DBF993
:10626000259038788DF898000220FBF7E6F904FABB
:1062700000F08DF899000220FBF7AFFAC043289098
:106280008DF89AA0E888ADF89C000220FBF770F921
:10629000ADF89E00D6482A90D6482B90D6482C9030
:1062A0003B9840B300211220FBF7B5F92D90012156
:1062B0001220FBF7B0F92E9078788DF8BC001220F0
:1062C000FBF7BBF904FA00F08DF8BD001220FBF7D4
:1062D00084FAC04331908DF8BEA0E888ADF8C000C4
:1062E0001220FBF745F9ADF8C200C4483390C4480A
:1062F0003490C44835909DF851000227022809D9EE
:10630000042805D99DF85010199800EB81001990C8
:106310008DF851709DF87500022809D9042805D917
:106320009DF87410229800EB810022908DF8757012
:106330000120FBF752FA4FF0553830B14FF0AA3137
:106340000120FBF73AFACDF858801120FBF745FA07
:1063500030B14FF0AA311120FBF72FFACDF87C8035
:106360009DF89900022809D9042805D99DF89810AC
:106370002B9800EB81002B908DF899709DF8BD0053
:10638000022809D9042805D99DF8BC10349800EBDF
:10639000810034908DF8BD700220FBF71EFA30B1F9
:1063A0004FF0AA310220FBF708FACDF8A0801220A6
:1063B000FBF713FA30B14FF0AA311220FBF7FDF9C9
:1063C000CDF8C480BDF8540000F58060ADF85400ED
:1063D000BDF8780000F58060ADF87800BDF89C004D
:1063E00000F58060ADF89C00BDF8C00000F580604D
:1063F000ADF8C000FBF7E1FD00204E9054904F90A7
:106400003D90449003F07EFC012800F0B88354983E
:10641000802800F2B48346A8FBF7D2FF002800F0E2
:10642000A88346A804F073FB4F98401C4F9000F0DF
:10643000958300204F905498401C549000203EAA11
:10644000012142F82010401C0628F8D33D9800286E
:1064500008BF3C9013D0012804BF00203C9000F0FE
:106460000481022804BF00203C9000F02882032809
:1064700004BF01204E9000F04F8300F080BB3C9998
:1064800036A850F8210000287ED001EBC1016846F3
:1064900000EB810000214C9101685291449A4168BF
:1064A0005391077A417A4591D0E90681B0F90C60A1
:1064B00000694D9054484069131AC3F10805904291
:1064C00048D848D145984FF00004002888BF4FF0C5
:1064D000010E3FD94D980EFA04F2024214BF4FF05C
:1064E000010B4FF0000B002004EB440202EB0412FE
:1064F0008446509228E0430952AA52F8232000F023
:106500001F030EFA03F31A421BD000F0010208EB3E
:106510004233509A4FEA500903EB820A31F9023BA9
:106520005AF829209B1B0CF1010CBBF1000F18BF7E
:106530005B42002BC8BF42F4803242F400424AF86A
:106540002920401C262801D2BC45D4D34598641C80
:106550008442BFD378E0002D7ADB45984FF0000AE3
:10656000002871D905F10800012202FA00FBE81D9C
:1065700002FA00F0519001234D9803FA0AF21040FC
:1065800018BF0120002200E067E057900AEB4A00A4
:1065900000EB0A10944650904FE0530952A802F0C5
:1065A0001F0450F823300120A040034242D002F0E3
:1065B000010008EB403350984FEA520903EB800486
:1065C00031F9023B54F829009B1B0CF1010CDDF85A
:1065D0005CE11BE0189D0030CC090030CC49003054
:1065E000B09D0030CC0E0030CC4E0030068500103F
:1065F000489E00304C1800304C580030E09E00306F
:106600004C1D00304C5D003018850010BEF1000FAD
:1066100018BF5B4210F4803F02D0002B04DA01E087
:10662000002B01DD20EA0B00002DC4BF519B184355
:1066300044F82900521C262A01D2BC45ADD3459806
:106640000AF1010A824596D3002D04BF01204C9027
:106650003EA93C9A4C9841F822003C98401C3C9042
:106660000628FFF40CAF00F057BA3C9936A850F852
:106670002100002800F01B813C98449900EBC002E7
:10668000684600EB82000022519202684C924268F8
:106690004D92037A457A847A5094D0E906C2B0F9D3
:1066A0000C8004695294C089509CC1F1080600EA2C
:1066B0000407E9B1002E75DB4FF0000A002D70D9F8
:1066C000012000FA06FB701E012101FA00F059902A
:1066D0000124529804FA0AF1084018BF0120002151
:1066E00045900AEB4A0000EB0A108946589093E067
:1066F0004FF0000A002D54D90124529804FA0AF1EF
:10670000084018BF0120002145900AEB4A0000EB29
:106710000A10894657903EE04C094CA801F01F0B27
:1067200050F82440012000FA0BF0044230D001F070
:1067300001000CEB403457984FEA510B04EB8000FA
:10674000539032F9024BDDF814E150F82B00A4EB22
:10675000080409F10109BEF1000F18BF644210F4EA
:10676000803F09D0002C0EDA10F47F4018BFA0F54E
:10677000807040F4803006E0002C04DD10F47F408F
:1067800018BFA0F5807040F08000539C44F82B00A7
:10679000491C262901D29945BED30AF1010AAA450E
:1067A000AAD340E043E04C094CA801F01F0E50F87A
:1067B0002440012000FA0EF004422AD001F001002A
:1067C0000CEB40345898DDF814E104EB80004C08E1
:1067D0005394579050F8240032F9024B09F1010903
:1067E000A4EB0804BEF1000F18BF644210F4803F10
:1067F00002D0002C04DA01E0002C01DD20EA0B00BD
:10680000002EC4BF599C2043DDF84CE1579C44F84E
:106810002E00491C262901D29945C4D30AF1010A48
:10682000AA45FFF455AF002EC8BF51983BDC0026A7
:10683000002D36D95098C0F5807A40F4807E002033
:1068400006EB4601024601EB061B25E044094CA974
:1068500000F01F0851F82440012101FA08F10C4210
:1068600017D000F001010CEB413101EB8B094FEA2D
:106870005008521C59F82840E1B201EB5A0101EAD4
:106880000E01B94288BF394624F0FF04214349F87C
:106890002810401C262801D29A42D7D3761CAE423B
:1068A000CDD3012051903C9A3EA941F822003C985A
:1068B000401C3C900628FFF4D8AE00F02DB93C995E
:1068C00036A850F8210000287ED04498529001EB61
:1068D000C101684600EB810000214D910168509193
:1068E0004168519190F808A0417A4591817AB0F9B8
:1068F0000C9082695792D0E90784C289006953904D
:106900005298C1F5807602EA010710F0010F14D009
:1069100045984FF0000B002872D90122539802FAD3
:106920000BF1084018BF012000214C900BEB4B00ED
:1069300000EB0B108C466790D6E00020FAF7B1FF11
:106940000546459800FB0AF1032000EB410020F0CA
:1069500003024146204616F06EF92846FAF7A1FFD9
:1069600045984FF0000B00284AD90122539802FAAB
:106970000BF1084018BF012000214C900BEB4B009D
:1069800000EB0B100D4659904DE04A0950A801F05C
:106990001F0350F8222001209840024240D038F9CD
:1069A000020B6D1CA0EB09034C98002818BF5B423A
:1069B00001F0010257984FEA510E00EB423259980C
:1069C00002EB8000589000E0A0E050F82E20C2F3C7
:1069D000072002F0FF0C12F4803F02D0002B02DBF4
:1069E00004E0002B02DDACEB060401E00CEB060436
:1069F000BC4206DDFF283ABF0024401C3C4607E0AD
:106A00007AE0002C04DA0028C6BF3C46401E002471
:106A100002F4803242EA0020589A204342F82E00C5
:106A2000491C262901D25545AFD345980BF1010BDE
:106A300083459AD360E04A0950A801F01F0350F83B
:106A400022200120984002424BD034F9020B4C9A8C
:106A5000A0EB09000CF1010C002A18BF404238F9E4
:106A6000022BA2EB090218BF52420028B4BF4342D6
:106A70000346002AB8BF52429A4232D9579A01F0CF
:106A8000010302EB4333679A03EB82024B08CDE923
:106A9000583252F82330C3F30722DDB213F4803F9B
:106AA00002D0002802DB03E0002801DD354400E0CD
:106AB000AD1BBD4205DDFF2A3ABF0025521C3D46F5
:106AC00006E0002D04DA002AC6BF3D46521E00250E
:106AD00003F4803040EA0220DDE95823284343F8DC
:106AE0002200491C262901D2D445A4D345980BF194
:106AF000010B8345FFF411AF5298032826BF0120F4
:106B00004D904D983EA93C9A41F822003C98401C7B
:106B10003C900628FFF4D3AE012300203EA951F893
:106B2000202002B3401C0628F9D3E3B13D981F286A
:106B300012D2401C01463D90012000FA01F26999F1
:106B40000A4209D13D99491C3D91032904D800FA14
:106B500001F269990A42F5D000204490FBF78DFCC0
:106B60004E9818B10BE04498401CF6E7FBF725FA65
:106B700048E4FEF769FE4E9800283FF443ACFBF76B
:106B80007CFCFBF703F801206299FAF716FE11204E
:106B90006399FAF712FE02206099FAF70EFE1220AE
:106BA0006199FAF70AFE6498FBF751FA5A98FAF7D6
:106BB000F5FD6598FAF775FE5F98FBF730F85E987B
:106BC000FBF720F86698FAF717FC5D9830B15C98EF
:106BD00010B1FBF7F2F901E0FBF7B6F9FCF7C3FEE1
:106BE00048B15698002818BFFCF7C2FE55980028F7
:106BF00018BFFCF7F5FE5B98002818BFFCF771FC86
:106C00004E9800280CBF012000206BB0BDE8F08F2B
:106C10002DE9F843074600200E46054600907DE02A
:106C2000284604F0ADFE002877D0008900EA07046A
:106C300024F0CC0030F47C406FD00F212846FEF7C2
:106C400006FF002869D0FBF76BF90099002962D193
:106C5000FBF747F8FF210F20FFF765F90090FAF7DF
:106C600095FF0098002856D19EB114F0010F1CBF6B
:106C70000220FFF71CF914F0100F1CBF0120FFF7D2
:106C800016F914F4807F1CBF2020FFF710F900983C
:106C9000E8BB24F0990030F4794006D0FDF76DFF91
:106CA0000090FAF773FF009888BB86B314F0020FC8
:106CB0000DD0FDF783F98046FEF7AAFE05235FEAB3
:106CC000080204D090F92D10184604F0B5FE14F017
:106CD000200F0DD0FDF7EDF88046FEF799FE092351
:106CE0005FEA080204D090F93110184604F0A4FEBF
:106CF00014F4007F0FD0FDF7A5F80446FEF788FED8
:106D00000D23220007D090F93510184601E002E06B
:106D100003E004F091FEFFF713F86D1C04F02CFE65
:106D2000A842009803D900283FF47AAF04E0002875
:106D300004BF0120BDE8F8830020BDE8F883F0B56A
:106D4000AD4E91B001243578FEF726FD012865D1BE
:106D5000AA480068B0F93610B0F9340015F0BBFF4E
:106D600015F0020F4FF000072ED002A800F00FF927
:106D700007982146401C079040F27770FFF748FFC4
:106D8000012803D1FEF70AF8012813D0099800233F
:106D9000401C0990502006901A462121072007F038
:106DA00003FA00231A461946FE200097FEF78BF8D7
:106DB00002A828E015F0080F14BFA220A120069019
:106DC0000898401C0890F3E715F0100F1DD0B0682C
:106DD000032824BF0024B76005D2684600F0D7F826
:106DE0000C98401C0C9021464FF4E060FFF710FF18
:106DF00008B1C4B106E0002301222121072007F0D9
:106E0000D3F914B16846FEF7D4FF0020FDF7F1FC7A
:106E100000232A464021072007F0C6F911B0BDE83B
:106E2000F04002F0F9BE04F0D1FD20F4E04004F09F
:106E3000CAFDEAE7704A002804BF51807047012864
:106E400004BF91807047022808BFD18070470100BD
:106E50004FF00000684A04BFB2F9020070470129F0
:106E600004BFB2F904007047022908BFB2F9060056
:106E7000704770B50126FEF777FF20B10069A128A1
:106E800018BFA22801D0002070BD002404F074FDBA
:106E9000002842D9204604F073FD00281EBF058952
:106EA00025F0CC0030F47C4032D00F212046FEF794
:106EB000CEFD68B315F0010F0AD0FBF7F7FA38B929
:106EC00044F4807200232021072007F06DF900268A
:106ED00015F0100F0BD00120FBF744FB38B944F438
:106EE000805200232021072007F05EF9002615F4C8
:106EF000807F0BD00220FBF735FB38B944F4803299
:106F000000232021072007F04FF90026FEF718FF85
:106F1000641C04F031FDA042BCD8304670BD002096
:106F20007047002070473448C068704770B5064607
:106F30000024FEF72EFC40BB2F4D286928B3B6F97C
:106F4000020046F678118142A4BF47F23051C84290
:106F500002DB0020A86070BDA968491CA960032954
:106F600013D3C0F3072144EA014141EA0062002340
:106F70006821072007F018F910210120FEF721FCF5
:106F8000E868401CE860012070BD002070BD10B5AD
:106F90000446FEF7E9FE80B1B0E80E10A4E80E103A
:106FA000B0E80E10A4E80E10B0E80E10A4E80E1021
:106FB000D0E90010C4E9001019E0FF223821204672
:106FC00015F057FE0E4820604FF490706060382036
:106FD0000021C4E902015020C4E90401481EE06216
:106FE000A062A1616062C4E9071021636163054882
:106FF000FBF736FE012010BD1885001064860010D6
:107000005443524600FE020070470020704710B5FE
:1070100003F00700042808BFFEF77AFC002010BD2B
:1070200070B503F007020025F84CF94B012A02D095
:10703000022A14D011E0052018709D60FCF70EFCA8
:107040002268532111702268452151702268010A7B
:1070500091702168C87020680571002070BD1A7891
:10706000052A13D19A68052A28BF104607D2D4F8FA
:1070700000C01CF802C080F800C0501C98600528B1
:1070800004D101209D60087003201870012070BD9C
:107090002DE9F04103F0070201260025DB4CDC4B13
:1070A000012A02D0022A3BD037E0052018709D60EB
:1070B000FCF7D4FB2168AC270F702268010A5170DD
:1070C0002168887004F0F2FBDFF8488380B1D8F8BB
:1070D000000004F0F5FC58B1D8F8000090F820004A
:1070E00010F0020F04D02068477021684320887098
:1070F0002068C6702068057104F0D8FB50B1D8F83C
:10710000000004F0DDFC28B1D8F800002168007E02
:10711000487102E02168FF2048710020BDE8F0813D
:107120001A78052A12D19A68062A28BF104607D273
:10713000D4F800C01CF802C080F800C0501C986051
:10714000062803D19D600E70032018700120BDE851
:10715000F08103F00702022A1CBF002070472022A2
:1071600002700120087070472DE9F041A84F0D46CC
:10717000064613F0070F04D003F00700022808D0DA
:1071800004E012F0040F1CBF0020B8700020BDE81E
:10719000F08102F03BFD002814BF0124002402F01E
:1071A00038FD002814BF0222002242EA0403B87806
:1071B000002814BF0422002242EA0300307001209C
:1071C0002870BDE8F08170B503F0070C0026904CE4
:1071D0008E4DBCF1010F0AD0204613F0070F007846
:1071E0000DD0BCF1040F08BF062818D029E0A66016
:1071F00028680670286846700520207021E0052860
:107200001FD1A068022803D22B681A54401CA0602A
:10721000022816D10120A6600870062010E0286818
:10722000007855280BD128684078AC2818BFBC28B6
:1072300005D128680122411C062002F0CDFC032064
:107240002070002070BD70B503F0070200256F4C60
:107250006F4B012A02D0022A24D021E005201870A9
:107260009D6002F084FC41F6E8710144B0F53C3FBA
:1072700010D8CA78086862F31F60674A904208BF56
:10728000002007D10A18236812791A54401C1428C8
:10729000F8D305E0002021680D54401C1428FAD3CF
:1072A000002070BD1A78052A13D19A68142A28BFC5
:1072B000104607D2D4F800C01CF802C080F800C005
:1072C000501C9860142804D101209D600870032090
:1072D0001870012070BD70B503F0070200254B4CFB
:1072E0004B4B012A02D0022A3FD03CE00520187007
:1072F0009D6002F03CFC41F6E8710144B0F53C3F72
:107300002BD8CA78086862F31F60434A904224D1A0
:107310002268087C10702268487C50702268887C43
:1073200090702068CA7CC27020680A7A0271226854
:10733000487A50712268887A90712268C87AD07130
:107340002268087D10722268487D50722268887D0C
:107350009072C87D2168C87205E0002021680D5434
:10736000401C0C28FAD3002070BD1A78052A13D1CE
:107370009A680C2A28BF104607D2D4F800C01CF81F
:1073800002C080F800C0501C98600C2804D1012075
:107390009D60087003201870012070BD70B503F067
:1073A00007020025194C1A4E012A02D0022A3FD0AA
:1073B0003CE004F0C5FA40B3D0E906212368C06878
:1073C0001A70D4F800C0130A8CF80130D4F800C049
:1073D000130C120E8CF802302368DA7022681171D7
:1073E00023680A0A5A7123680A0C090E9A712268E6
:1073F000D171216808722268010A51722268010C59
:107400009172010E2068C1720DE007E0EC050200E8
:10741000388500106486001034CD12AB21680D54FD
:10742000401C0C28FAD305203070B560002070BDD8
:107430003278052A10D1B2680C2A28BF104604D22F
:1074400023689B5C0370501CB0600C2804D10120A1
:10745000B560087003203070012070BD70B503F076
:1074600007020024F84DF94B012A02D0022A3ED02F
:107470003BE00520187000269C6002F078FB00F5C8
:107480000051B0F53C3F98BF11F0030F27D1F04AEF
:107490000868904204BF0022104620D151F82030E5
:1074A000401C1A440728F9D302B1C6B128680A7CE7
:1074B00002702A68487C50702A68887C90702A681C
:1074C000C87CD0702A68087D10712A68487D507188
:1074D0002A68887D9071C87D2968C87105E0002000
:1074E00029680C54401C0828FAD3002070BD1A7873
:1074F000052A13D19A68082A28BF104607D2D5F862
:1075000000C01CF802C080F800C0501C9860082819
:1075100004D101209C60087003201870012070BD08
:107520002DE9F04103F0070C0027C84E4FF0050885
:10753000BCF1010F0DD013F0070F0FD03246BCF194
:10754000020F127810D0BCF1040F08BF062A26D013
:1075500058E086F800807770B76053E07270BD48DD
:10756000B062062030704DE0052A15D1B268042AB9
:1075700028BF104609D2C2F10303D6F828C0DB00A9
:107580002CFA03F30370501CB060042804D10120CE
:10759000B7600870032030700120BDE8F08170787A
:1075A0000125002410F0010F11D002F0E0FAB0F52F
:1075B0003C3F23D86A030021B1EB900F07D252F869
:1075C000043B491C1C44B1EB900FF8D3B5B1707863
:1075D00010F0020F0ED004F0B3F978B182680021E8
:1075E000B1EB920F06D250F8043B491C1C44B1EB9E
:1075F000920FF8D3002D18BFB46200D1B762777034
:1076000086F800800020BDE8F081F0B503F0070C9B
:1076100000268D4D8D4C83B0BCF1010F0ED013F0C0
:10762000070F1DD0224603271278BCF1020F26D087
:10763000BCF1040F08BF062A36D03CE002AA01A91B
:10764000684602F05FFE05202070296801980870E6
:10765000296800984870296802988870A6602AE016
:10766000A068032803D229680A54401CA06002289D
:1076700021D306212170032808BFA6601BE0052A3C
:107680000FD1A268032A28BF104604D22B689B5C46
:107690000370501CA060032803D10120A66008706D
:1076A000277003B00120F0BD286882780178407807
:1076B00002F01BFE277003B00020F0BD08B503F0F8
:1076C000070001280AD104F0F1F838B101208DF843
:1076D0000000024669460D2002F07EFA002008BD37
:1076E00008B503F0070001280AD104F0DFF838B12B
:1076F00000208DF80000012269460D2002F06CFA8E
:10770000002008BD08B503F00700012809D104F0E6
:10771000CDF830B103208DF800000122694602F057
:107720005BFA002008BD0020704708B503F0070091
:1077300001280AD104F0BAF838B10B208DF8000006
:1077400001226946032002F047FA002008BD1FB558
:1077500013F0070F0ED104F0A9F858B19DF80800F6
:10776000F0280AD004F0A2F820B1012202A90920D1
:1077700002F032FA04B0002010BDFEF717FBF9E763
:1077800008B503F0070001280AD104F08FF838B1DA
:1077900010208DF8000001226946032002F01CFA37
:1077A000002008BD70B503F00700274C274D0128C5
:1077B00008D013F0070F12D0042804BF2878062839
:1077C00016D01FE00020A86021680870216848706A
:1077D000216888702168C8700520287012E0A868A8
:1077E00004280FD221680A54401CA860062008E033
:1077F00004F05CF830B104221046216802F0ECF984
:1078000003202870002070BD10B503F00700012888
:1078100004D103F04FFA0D4900200871002010BD7B
:1078200010B503F0070C094CBCF1010F06D013F0A2
:10783000070F11D0BCF1020F20D01DE00020A06086
:1078400006F0A9FCA06117E0EC05020038850010E5
:1078500054464953EFBEADDEA068002804BF1002B5
:10786000A06106D0012804D1A0691043A06106F0F0
:1078700091FCA068401CA060002010BDA26812B15D
:10788000012A04D007E0218B090A017003E0237E5E
:10789000037001200870501CA060012010BD10B5BD
:1078A00003F0070CF74CBCF1010F06D013F0070FE3
:1078B00009D0BCF1020F18D015E00020A06006F03E
:1078C0006DFCA0610FE0A068002804BF1002A06159
:1078D00006D0012804D1A0691043A06106F061FC24
:1078E000A068401CA060002010BDA26812B1012A4F
:1078F00004D007E0218B090A017003E0237E0370A6
:1079000001200870501CA060012010BD70B503F06C
:10791000070CDC4D0E460446BCF1010F06D013F0F7
:10792000070F07D0BCF1020F18D015E00020A860A7
:10793000E86011E0A868002804BF1002A86108D020
:10794000012806D1A869104381B2A861E8880DF02A
:10795000EEFFA868401CA860002070BDE8680228FF
:107960000ED2E8880DF0E7FFEB6882B2002B04BF6F
:10797000100A207004D0012B02D122700120307037
:10798000E868401CE860012070BD10B403F0070CEB
:10799000BC4CBCF1010F08BF00200BD013F0070F47
:1079A00003D0BCF1020F09D005E0A068002808BF91
:1079B000E280401CA06010BC00207047A2681AB989
:1079C000A379037001200870501CA06010BC012036
:1079D00070472DE9F047064603F00700A94F894696
:1079E000012808BF002039D0DFF89C82A74D13F092
:1079F000070F02D0022835D031E0B868002808BF50
:107A00007A7029D0012804BF1002B86124D002285E
:107A100022D1B8691043B8617E7884B203F046FF82
:107A2000D0B1062E18D2DFE806F00306090C1014B8
:107A3000A8F80E4010E0A8F80C400DE028688486F5
:107A40000AE02868A0F80C4106E02868A0F8504039
:107A500002E02868A0F85240B868401CB8600020D6
:107A6000BDE8F087F86802282CD297F801A000241E
:107A700003F01CFFD8B1BAF1060F18D2DFE80AF004
:107A80000306090C1014B8F80E4010E0B8F80C40CA
:107A90000DE02868848E0AE02868B0F80C4106E002
:107AA0002868B0F8504002E02868B0F85240F86802
:107AB000002804BF200A307004D0012802D134709D
:107AC00089F80000F868401CF8600120BDE8F087E4
:107AD0002DE9F0411C4615460E46074603F0E6FE2A
:107AE00080B1694814F0070F04D004F0070102299F
:107AF0000BD007E0002D1ABF90F86C00C0080020E2
:107B00000AF086FA0020BDE8F08190F86C00C00809
:107B1000387001203070BDE8F0812DE9F0411C463D
:107B200015460F46064613F0070F08D103F0BEFEB8
:107B300028B1022D3CBF284607F09DFF03E004F06A
:107B40000700022802D00020BDE8F08107F08CFF7A
:107B5000307001203870BDE8F08170B503F0070285
:107B600000264B4C474D012A02D0022A15D012E0C4
:107B700007F091F821680870FDF70EFE2168487043
:107B800003F0FAFB21688870FDF70CFE2168C870CD
:107B900005202870AE60002070BD2A78052A10D11B
:107BA000AA68042A28BF104604D223689B5C03708D
:107BB000501CA860042804D10120AE600870032086
:107BC0002870012070BD70B503F00702304C00250D
:107BD0002C4E012A02D0022A5CD051E0FEF7C4F8F4
:107BE000002836D04169FF292CBFFF21C9B2226885
:107BF00011708169FF2934BFC9B2FF212268517019
:107C0000C169FF2934BFC9B2FF212268917022687F
:107C1000017CD170226890F820101171018C2268CB
:107C2000090A5171016A2268090C9171016A22687E
:107C3000090ED171016BFF2934BFC9B2FF2122683F
:107C40001172406BFF2834BFC0B2FF202168487218
:107C500015E02068057020684570206885702168EF
:107C60005020C8702168FF20087121684871216880
:107C700088712168C8712068057220684572B560F6
:107C8000002070BD388500101011011064860010AE
:107C9000EC050200B2680A2A28BF104604D2236805
:107CA0009B5C0370501CB0600A2802D10120B560B3
:107CB00008700120E5E703F00702FC4B4FF0000CD1
:107CC000012A08BFC3F808C001D0022A01D0002051
:107CD00070479A68022A3DBF80F800C0501C986027
:107CE0001046022803D10120C3F808C00870012003
:107CF00070472DE9F047064603F00700EB4F894631
:107D00004FF00008012808BFC7F8088001D00228FA
:107D100002D00020BDE8F087B86880BB002425466B
:107D200001F025FF00F50051A1F1180340214FF4A7
:107D30000052B0F53C3F1ED893F803A0D3F800C022
:107D40006AF31F6CDFF868A3D44514D1001FB4EBAD
:107D5000900F07D252F804CB641C8CEA0505B4EBF3
:107D6000900FF7D3DA7D586962F31F60A84204BF11
:107D70008020307000D03170B868401CB860012895
:107D800003D1C7F8088089F800000120BDE8F0871A
:107D90002DE9F04103F007020026C64CC34D012A2D
:107DA00002D0022A56D052E0FBF758FD0520287079
:107DB00003F07CFD002849D0BF4F386803F080FEF7
:107DC000002843D00DF096FD80460DF097FD3968F0
:107DD0000A7E12F0040F11D0C98A2268090A1170B4
:107DE00039682268897D517039682268898A090A50
:107DF000917039682268097DD17010E0898A226803
:107E0000090A117039682268097D51703968226841
:107E1000C98A090A917039682268897DD1702268FF
:107E20004FEA18211171216881F805802268010A42
:107E300091712168C87138682268817C117222684A
:107E4000017C5172008B2168000A8872AE600020AC
:107E5000BDE8F0812A78052A10D1AA680B2A28BF2C
:107E6000104604D223689B5C0370501CA8600B284A
:107E700004D10120AE600870032028700120BDE805
:107E8000F0812DE9F04703F007020026894D874B6A
:107E9000012A02D0022A5DD059E005201870002482
:107EA0009E6001F064FE00F50053B0F53C3F98BFC2
:107EB00013F0030F45D1814A1968914204BF002293
:107EC000114608D153F821C0491C62440729F9D34F
:107ED000002A08BF01249F7C93F8138084B341F6E5
:107EE000E8710144B0F53C3F07D8CA78086862F3EE
:107EF0001F606F4A904208BF012491F8129091F8D8
:107F000013A0002C08BF002014D003F019FD29682D
:107F1000806981F80090296881F801A02A68010C25
:107F2000000E91702968C87028680771286880F869
:107F300005800CE029680E54401C0628FAD306E0A0
:107F4000FFE7002029680E54401C0628FAD30020C1
:107F5000BDE8F0871A78052A13D19A68072A28BF46
:107F6000104607D2D5F800C01CF802C080F800C047
:107F7000501C9860072804D101209E6008700320DF
:107F800018700120BDE8F08710B503F0070C474CCE
:107F9000BCF1010F06D013F0070F0AD0BCF1020F9D
:107FA0001AD017E00020A060E0600DF021FDA06174
:107FB00010E0A068002804BF1002A06107D00128CB
:107FC00005D1A0691043A06180B20DF00EFDA0683C
:107FD000401CA060002010BDE268022A0BD212B142
:107FE000012A04D007E0218B090A017003E0237EF7
:107FF000037001200870501CE060012010BD70B5B6
:1080000003F007010026294D0446012908BFEE624E
:1080100001D0022901D0002070BDE86A002804BF09
:10802000274814F05DFEE96A082928BF267002D2AD
:108030002348405C2070481CE862012070BD2DE997
:10804000F04103F007010026184D0746012908BF3B
:10805000EE6201D0022902D00020BDE8F08195F83F
:108060002C0000F007042879204304D1144814F0B0
:1080700037FE01202871052C28BF2E711048005DA5
:108080003870E86A401CE8620120BDE8F08170B5F4
:10809000044603F007000D4602281CBF002070BDF7
:1080A00014F023FE20700120287070BD3885001068
:1080B00034CD12ABEC0502006486001054464953DF
:1080C0006885001070B503F007020025F74C012AFF
:1080D00002D0022A12D00FE00520207000221146A3
:1080E0001046A56002F00EF94FF6FF7101EA40005C
:1080F000206102F01AF96062002070BD2278052A22
:1081000017D1D4F810C0A268624528BF104607D224
:1081100012F0010F1CBF637803700CD0501CA060DC
:10812000604506D10120A56008700320207002F090
:1081300009F9012070BD666A22F00103F35A1E0A94
:1081400006706370EAE770B503F007020025D74CAC
:10815000012A02D0022A11D00EE0D548052200687B
:10816000B0F91210B0F91000227008444000A56068
:10817000206102F05AFA6062002070BD2278052A60
:1081800017D1D4F810C0A268624528BF104607D2A4
:1081900012F0010F1CBF637803700CD0501CA0605C
:1081A000604506D10120A56008700320207002F010
:1081B00065FA012070BD666A22F00103F35A1E0AB7
:1081C00006706370EAE7F8B503F007020025B74CC4
:1081D000012A02D0022A13D010E000216A46084684
:1081E00002F090F805202070A56000984FF6FF710E
:1081F00001EA4000206102F05AFB60620020F8BDF5
:108200002278052A17D1D4F810C0A268624528BF89
:10821000104607D212F0010F1CBF637803700CD018
:10822000501CA060604506D10120A56008700320A5
:10823000207002F046FB0120F8BD666A22F00103BF
:10824000F35A1E0A06706370EAE77FB51C460E46B5
:10825000054613F0070F08D103F028FB28B10122CF
:1082600002A9212001F0B8FC03E004F00700022875
:1082700002D004B0002070BD06F00DFE2870012071
:10828000307004B070BD7FB51C460E46054613F035
:10829000070F08D103F00AFB28B1012202A922200E
:1082A00001F09AFC03E004F00700022802D004B0B9
:1082B000002070BD06F0F5FD28700120307004B07C
:1082C00070BD7FB51C460E46054613F0070F08D15A
:1082D00003F0ECFA28B1012202A90C2001F07CFC89
:1082E00003E004F00700022802D004B0002070BDB3
:1082F00006F0D1FC28700120307004B070BD7FB54D
:108300001C460E46054613F0070F08D103F0CEFABF
:1083100028B1012202A90F2001F05EFC03E004F065
:108320000700022802D004B0002070BD10F04AFF00
:1083300000F00F0040F0100028700120307004B0F1
:1083400070BD10B503F00702584C012A02D0022A72
:108350000DD00AE003F054FD0021E06100281ABFAF
:108360004FF4056020622162A160002010BD236AE5
:10837000A2689A4228BF104607D2D4F81CC01CF845
:1083800002C080F800C0501CA060984204BF0120C9
:108390000870012010BD10B413F0070F4FF0402CEF
:1083A00004D003F00702022A13D00FE0012A04BF11
:1083B000DCF8140040F0010006D0002A04BFDCF80D
:1083C000140020F0010001D1CCF8140010BC0020F2
:1083D0007047DCF81430002213F0010F18BF01229F
:1083E000344BD3F83CC0324B1B68B3F8A430C3F312
:1083F0000334012303FA04F41CEA040F18BF42F00B
:10840000020202700B7010BC0120704770B5144658
:108410000E46054613F0070F04D003F007000228AC
:1084200013D010E0002C14BF0120002002F034FC17
:108430004CB14FF04020016B21F4405141F4BE019A
:1084400041F020410163002070BD02F02CFC0028A7
:1084500014BF012200222A700120307070BD2DE966
:10846000F04103F0070C114C0F468046BCF1010FA0
:1084700012D0104E13F0070F4FF0030510D0204616
:10848000BCF1020F027829D0BCF1040F02BFA06832
:108490000128062A36D039E00520207000201BE094
:1084A000A06848B101280BD014E000003885001006
:1084B000648600100010004062700620207009E001
:1084C000607800EA0201316320EA02017163FAF781
:1084D00033FD2570A068401CA06017E0A06801284B
:1084E00008BF062A03D16078FAF72BFD2570F06BE0
:1084F00088F8000001203870A068401CA0600120AE
:10850000BDE8F0816078FAF71CFD25700020BDE819
:10851000F08170B5044603F007000D4602281CBF29
:10852000002070BDFDF725FA002814BF01220022AB
:1085300022700120287070BD70B50D46044613F0FE
:10854000070F04D003F00700022805D002E0104610
:1085500006F0F2FA002070BD06F0F1FA207001205A
:10856000287070BD70B50D46044613F0070F04D097
:1085700003F00700022805D002E01046F8F7B4FC2B
:10858000002070BDF8F7B3FC20700120287070BD8A
:1085900070B503F00702DFF87CC40C460546012ADB
:1085A00008BF05200DD013F0070F08BF062008D024
:1085B000022A09D0042A04BF9CF80000062809D02A
:1085C0000EE08CF800000BE0FDF7D9F928700120CF
:1085D000207070BD03208CF800000120FDF7D2F957
:1085E000002070BD70B5044603F007000D46022858
:1085F00007D013F0070F04BF1046FDF7C7F800209F
:1086000070BDFDF7C6F820700120287070BD70B5F0
:10861000044603F00700FF4D0E46012804BF00206A
:10862000A86014D013F0070F02D0022811D00EE07A
:10863000A868F94904283CBF0B681A54401CA8607C
:10864000042804D104220968122001F0C5FA002090
:1086500070BD0AF097FFAA68002A04BF000E2070C0
:108660000FD0012A08BF000C06D0022A08BF000A5A
:1086700002D0032A02D004E0207002E02070012022
:108680003070501CA860012070BD70B503F0070C5D
:10869000E04D0E460446BCF1010F04BF0020A86067
:1086A00015D013F0070F03D0BCF1020F11D00EE06C
:1086B000A868D94902283CBF0B681A54401CA8601E
:1086C000022804D102220968132001F085FA002053
:1086D00070BD0AF02FFFAA68002A04BF000A2070AC
:1086E00004D0012A02D1207001203070501CA860F3
:1086F000012070BD70B5044603F00700C54D0E465D
:10870000012804BF0020A86014D013F0070F02D086
:10871000022811D00EE0A868BF4904283CBF0B68AE
:108720001A54401CA860042804D1042209681420AB
:1087300001F052FA002070BD0AF051FFAA68002A29
:1087400004BF000E20700FD0012A08BF000C06D015
:10875000022A08BF000A02D0032A02D004E02070D7
:1087600002E0207001203070501CA860012070BD14
:1087700070B5044603F00700A64D0E46012804BF5D
:108780000020A86037D013F0070F02D0022834D0A1
:1087900031E0A868A04C002804BF21680A70216855
:1087A0000978012901D039B11BE0002818BF04283D
:1087B0003CBF21680A5414E00AF02CFF216800092C
:1087C00048700AF01BFFC0F303260AF023FF21685C
:1087D00046EA001088700AF011FF2168C870032073
:1087E000A860A868401CA860042804D104221520B1
:1087F000216801F0F1F9002070BD0AF017FFAA68A6
:10880000002A04BF000E20700FD0012A08BF000C00
:1088100006D0022A08BF000A02D0032A02D004E0D0
:10882000207002E0207001203070501CA8600120F0
:1088300070BD10B503F00702764C012A02D0022A5F
:1088400027D024E003F0DCFA0023002804BFE36112
:1088500023621BD000F15001E1614168B1F5887FCE
:1088600090F820100CD390F8212001EB020C01FBB2
:1088700002C190F8222090F823001044084404E03C
:1088800090F822000A1801FB00202062A36000205B
:1088900010BD236AA2689A4228BF104607D2D4F8B6
:1088A0001CC01CF802C080F800C0501CA060984298
:1088B00004BF01200870012010BD03F00702012A47
:1088C00002D0022A05D002E0524900208860002030
:1088D0007047012202700A701046704710B513F0FD
:1088E000070F04D003F00702022A05D002E0104669
:1088F00001F035FD002010BD484A127802700120B9
:10890000087010BD10B513F0070F04D003F0070274
:10891000022A05D002E0104601F0BDFE002010BD85
:108920003F4A127802700120087010BD10B513F094
:10893000070F04D003F00702022A05D002E0104618
:1089400001F0CCFF002010BD364A127802700120E1
:10895000087010BD1FB513F0070F07D102F0A6FF76
:1089600020B1012202A90B2001F036F904B0002049
:1089700010BD70B503F00700264C1546012804BF52
:108980000020A06024D013F0070F21D102F08EFF49
:10899000F0B1A068204E03283CBF31680D54401C44
:1089A000A060032814D1F9F7B4F93068B0F80100D9
:1089B00045BAF9F7E9F8040018BFF9F738FB306851
:1089C00029460078F8F737FD002C18BFF9F732FB7D
:1089D000002070BD70B503F007000E4C164601284C
:1089E00004BF0020A06034D013F0070F31D102F093
:1089F0005DFF70B3A068084D02283CBF29680E5483
:108A0000401CA060022824D1F9F783F9F9F7BCF8DB
:108A1000040009E038850010EC0502007D85001097
:108A2000828500108785001018BFF9F700FB2868C1
:108A3000007880B129684978F8F77CFD286841788A
:108A4000007840F01000F8F775FD002C18BFF9F71A
:108A5000F1FA002070BD286841780020F3E77FB567
:108A60001C460E46054613F0070F08D102F01EFF04
:108A700028B1012202A9192001F0AEF803E004F0A8
:108A80000700022802D004B0002070BD06F0DAF81A
:108A9000002814BF012200222A700120307004B087
:108AA00070BD7FB51C460E46054613F0070F08D172
:108AB00002F0FCFE28B1012202A91A2001F08CF874
:108AC00003E004F00700022802D004B0002070BDCB
:108AD00006F0A4F828700120307004B070BD2DE9B4
:108AE000F04103F0070CFB4C0E460746BCF1010FAA
:108AF00007D0F94D13F0070F07D0BCF1020F19D0C2
:108B000015E00020A060E06011E0A06803283CBFF1
:108B100029680A54401CA060032808D12868B0F8CE
:108B2000010040BA01B228680078FEF783F90020FE
:108B3000BDE8F081E268022A12D242B928680078C2
:108B4000FEF785F92A68010A51702968887028683B
:108B5000E2681044012A4078387004BF0120307068
:108B6000E068401CE0600120BDE8F08170B503F0D2
:108B70000700D84C1546012804BF0020A06017D07C
:108B800013F0070F14D102F091FE88B1A068D24B08
:108B900003283CBF19680D54401CA060032807D16E
:108BA0001868B0F8010041BA18680078F9F73AFD82
:108BB000002070BD10B503F00702C64C012A02D098
:108BC000022A07D004E00020A060FAF738FDA06177
:108BD000002010BDA268042A07D2C2F10303D4F812
:108BE00018C0DB002CFA03F30370501CA0600428AB
:108BF00004BF01200870012010BD10B503F007006C
:108C0000012807D102F052FE20B1002211461E2099
:108C100000F0E2FF002010BD2DE9F04103F0070550
:108C2000AC4E174688460446012D04BF0020B060B4
:108C30001BD013F0070F16D102F038FE98B1B068C0
:108C4000A54B03283CBF19680F54401CB060032893
:108C50000BD1186890F9022090F9011090F90000EA
:108C6000FCF76EF901E0022D02D00020BDE8F08192
:108C7000B06830B1012809D002280CD003280FD0E9
:108C800015E01420FCF793F8207010E01520FCF795
:108C90008EF820700BE01620FCF789F8207006E0B3
:108CA0001720FCF784F82070012088F80000B068D5
:108CB000401CB0600120BDE8F08170B50D4604464F
:108CC00013F0070F04D003F00700022805D002E0DC
:108CD000804900208860002070BD0120FCF767F803
:108CE00020700120287070BD70B503F0070C0026BD
:108CF000794C784DBCF1010F06D013F0070F0CD062
:108D0000BCF1020F1FD01CE006F09AF8AE6021689B
:108D100008702168000A487013E0A868022803D28E
:108D200021680A54401CA86002280AD1AE6020685D
:108D3000007810F0010F04D002221B20216800F0FF
:108D40004BFF002070BDAA68022A28BF104604D23B
:108D500023689B5C0370501CA860022804D101208A
:108D6000AE60087003202870012070BD7FB51C46DE
:108D70000E46054613F0070F08D102F097FD28B103
:108D8000012202A9252000F027FF03E004F00700DC
:108D9000022802D004B0002070BD0CF018FE28702C
:108DA0000120307004B070BD7FB51C460E460546EC
:108DB00013F0070F08D102F079FD28B1012202A9B2
:108DC000202000F009FF03E004F00700022802D091
:108DD00004B0002070BD0CF005FE2870012030703A
:108DE00004B070BD7FB51C460E46054613F0070F54
:108DF00008D102F05BFD28B1012202A9242000F075
:108E0000EBFE03E004F00700022802D004B00020CB
:108E100070BD10F011FC28700120307004B070BDDE
:108E20007FB51C460E46054613F0070F0ED102F023
:108E30003DFD58B19DF80800002818BF0CF0DBFD7F
:108E4000012202A91F2000F0C7FE03E004F0070082
:108E5000022802D004B0002070BD0CF0CFFD2870B5
:108E60000120307004B070BD2DE9FF41194E1C4641
:108E70000F46054613F0070F1CD102F017FDC8B1CD
:108E80009DF80800002818BF012802D0022807D04A
:108E900014E0F070012202A9082000F09DFE0DE010
:108EA000F07004208DF80800012202A9082000F0CB
:108EB00093FE03E004F00700022803D004B0002072
:108EC000BDE8F081F07828700120387004B0BDE86A
:108ED000F081000038850010EC0502007FB51C46CB
:108EE0000D46064613F0070F08D102F0DFFC28B14B
:108EF000012202A9082000F06FFE03E004F0070041
:108F0000022802D004B0002070BDFCF745FC801E92
:108F100005280ED2DFE800F0030709050B0000204A
:108F200008E0012006E0022004E0032002E0042023
:108F300000E0FF2030700120287004B070BD2DE9E2
:108F4000F0411C4617460E46054613F0070F0BD19D
:108F500002F0ACFC40B1384605F0E8FD00221146B5
:108F6000012000F039FE03E004F00700022802D0DF
:108F70000020BDE8F08105F0DCFD28700120307094
:108F8000BDE8F08110B5104613F0070F08BF05F0DB
:108F900070FE002010BD10B5104613F0070F08BF7B
:108FA00005F06EFE002010BD70B5044603F007000A
:108FB0000D4602281CBF002070BD05F069FE207020
:108FC0000120287070BD03F0070230B4F74B4FF05A
:108FD000000C012A05D0022A04BF1A78022A0BD0FD
:108FE0001EE002201870F248C3F808C06FF07F41FD
:108FF0000068081A986113E09A68042A28BF10468E
:1090000006D29D69D40025FA04F40470501C9860BF
:10901000042805D10120C3F808C008700320187087
:1090200030BC0120704713F0070F04BFE148027005
:109030000020704710B503F00700DC49012804BF89
:109040000020886013D013F0070F10D18868DA4B26
:1090500004283CBFD3F800C00CF80020401C8860F6
:10906000042804D104221120196800F0B5FD002065
:1090700010BD2DE9F047164603F007020024CB4F40
:10908000012A04BFBC60FC6064D0DFF8308313F0B9
:10909000070F07D0022A33D0042A04BF38780628E5
:1090A0004FD058E0BD68002D08BFFE6125D0012DCE
:1090B00006D0D7F81090AC1E4C4516D284B908E003
:1090C000701C3861F9690844B0F5007F88BF3C61C5
:1090D00013E04FF400724FF43E31B94813F09CFD99
:1090E000B549F869096820440E54601C484504D10C
:1090F000B348C0F8FC8106203870681CB8602AE0CC
:10910000FF2202703B69CBB1D7F81CC0FA689444C7
:10911000BCF5007F10D2AB4D2D68454518BF0470DB
:1091200005D10CF53C3C9CF800C880F800C0501CF0
:10913000984204BF01200870501CF8600120BDE86F
:10914000F0874FF43E30F9F78BFD9D494FF43E30E8
:10915000F9F728FE3C700020BDE8F0872DE9F047C4
:109160008C4603F007010024904F1646012904BFE6
:10917000BC60FC6062D013F0070F934BDFF84C82A9
:1091800007D0022932D0042904BF387806284DD0F0
:1091900055E0BD68002D08BFFE6124D0012D06D02A
:1091A000D7F81090AC1E4C4515D27CB908E0701C65
:1091B0003861F9690844B0F5007F88BF3C6112E06E
:1091C0004FF4007219467E4813F026FD7A49F8697B
:1091D000096820440E54601C484504D17848C0F802
:1091E000FC8106203870681CB86028E0FF210170FF
:1091F0003B69C3B1FA69F9680A44B2F5007F10D23D
:10920000734D2D68454518BF047004D102F53C32FA
:1092100092F800260270481C984204BF01208CF886
:109220000000481CF8600120BDE8F0871D46184684
:10923000F9F716FD62492846F9F7B4FD3C700020A5
:10924000BDE8F08770B503F00700584C15460128BB
:1092500004BF0020A06014D013F0070F11D102F05A
:1092600025FB70B1A068544902283CBF0A68155418
:10927000401CA060022804D102220968052000F0E9
:10928000ABFC002070BD2DE9F041054603F007005E
:10929000494C464E0F4601280AD013F0070F14D050
:1092A00002281BD0042804BF3078062834D03FE0C1
:1092B0000020B060216808702168487021688870BB
:1092C0002168C8700520307032E0B06804282FD2C1
:1092D00021680A54401CB060062028E0B06860B9DC
:1092E00005F018FC216808702268010A5170226894
:1092F000010C000E91702168C870B06804283ABF54
:109300002168095CFF21297024BF01213970401CAC
:10931000B0600120BDE8F08102F0C8FA40B12068D9
:10932000C178006861F31F6005F0EFFB0320307027
:109330000020BDE8F08170B503F007011B4C064624
:1093400001290BD01C4D13F0070F0CD0022914D0AB
:10935000042904BF207806281DD025E00020A06045
:109360000520207020E0A068B0F5007F1CD229689D
:109370000A54401CA060062015E0A06818B900211E
:10938000286813F0B7FC2868A168405C3070481C5E
:10939000A060012070BD02F089FA28B1A168286898
:1093A00013F0ADFC03202070002070BD3885001044
:1093B000948400102F840010EC050200554E564D89
:1093C00018B70010FCF9020000F60200324E564DAC
:1093D000FCF702007FB51C460E46054613F0070F4A
:1093E00008D102F063FA28B1012202A9102000F08E
:1093F000F3FB03E004F00700022802D004B00020D1
:1094000070BD0FF0DCFE28700120307004B070BD1C
:109410002DE9F041054603F00700F74CF74E0F46E3
:1094200001280AD013F0070F14D002281BD00428FB
:1094300004BF3078062834D03FE00020B0602168B7
:10944000087021684870216888702168C8700520FC
:10945000307032E0B06804282FD221680A54401CD2
:10946000B060062028E0B06860B913F04DFC2168B8
:1094700008702268010A51702268010C000E917078
:109480002168C870B06804283ABF2168095CFF21D0
:10949000297024BF01213970401CB0600120BDE853
:1094A000F08102F003FA40B12068C178006861F3EE
:1094B0001F6013F02EFC032030700020BDE8F08107
:1094C0007FB50D46044613F0070F04D003F00700E4
:1094D000022808D004E0012202A9262000F07CFB2B
:1094E00004B0002070BD13F019FC2070012028701A
:1094F00004B070BD2DE9F041044603F00700BF4EF3
:109500000F46012804BF0020B06001D0022802D01D
:109510000020BDE8F081B84DB06860B9FDF703FDEB
:109520002A68010E11702A68010C51702A68010A1C
:1095300091702968C870B06804283ABF2968095C2E
:10954000FF21217024BF01213970401CB06001202F
:10955000BDE8F0812DE9F04103F00702A74D0E466A
:109560000446012A04BF0020A86001D0022A02D0CC
:109570000020BDE8F081A04FA86830B913F0D3FBFC
:109580003A68010A117039684870AA68022A3ABF1D
:109590003868805CFF20207024BF01203070501C90
:1095A000A8600120BDE8F0811FB513F0070F04D1BA
:1095B000012202A91C2000F00FFB04B0002010BD06
:1095C00003F007008D49012806D013F0070F04BFF0
:1095D0000878012806D014E0012008700020886077
:1095E00048610DE08868042805D24B69401C42EAB6
:1095F00003224A618860042803D103200870486967
:10960000C8610020704703F00700DFF8F0C10128AF
:1096100007D013F0070F04BF9CF80000022809D000
:109620001EE002208CF800000020CCF80800CCF8E6
:10963000180015E0DCF80800022808D2DCF8181041
:10964000401C42EA0121CCF81810CCF8080002288E
:1096500006D1DCF81800CCF8200003208CF80000BC
:109660000020704770B403F007020025634C012A04
:1096700002D0022A06D002E002202070A56070BC51
:10968000002070472278022A1CD1D4F820C0A2689A
:10969000624528BF10460ED212F0030F04D1E369D1
:1096A00053F8046BC4E90663237E0370A069000AC3
:1096B000A061501CA060604504D10120A560087025
:1096C0000320207070BC0120704770B503F00700C4
:1096D00000254A4C0E46012806D013F0070F04BFA0
:1096E0002078022805D02BE002202070A560A5611B
:1096F00026E0216AA068884219D2A169090A41EAD4
:109700000262401CA26110F0030FA0600FD1E0695B
:10971000B0F5443F28BF026006D2B0F5005F03D326
:1097200004223749F9F792FBE069001DE061216AE4
:10973000A068884204D10120A56030700320207009
:10974000002070BD30B403F007040025DFF8ACC082
:10975000012C08BFCCF8085035D013F0070F02D009
:10976000022C33D02FE0042A08BF4FF4403028D019
:1097700013DC002A08BF4FF4005022D0012A08BF92
:109780004FF443301DD0022A08BF4FF41C3018D0CC
:10979000032A08BF1B4814D010E0052A08BF4FF465
:1097A0003E300ED01848102A00680AD0112A08BF8F
:1097B000164806D0202A08BFB43002D0CCF8145086
:1097C00001E0CCF8140030BC00207047DCF8082021
:1097D000042A07D2C2F10303DCF81440DB0024FAA8
:1097E00003F30370501CCCF80800042824BF0120A8
:1097F0000870012030BC7047EC050200388500106D
:109800005085001000FE0200648600101011011047
:1098100070B403F0070CDE4DBCF1010F07D0DD4C36
:1098200013F0070F07D0BCF1020F21D01DE000207C
:10983000A860E86019E0A86805283CBF21680A54C0
:10984000042810D123682268D4F800C0D3F801306E
:10985000696912781BBA9CF804C023F0FF0343EA3D
:109860000C0341F82230401CA86070BC00207047F7
:10987000EB6873B1042B07D22268032B1A44527889
:10988000027004BF01200870581CE86070BC012001
:1098900070472268D5F814C012785CF82220266838
:1098A0004FEA126C86F801C026684FEA124C86F81F
:1098B00002C026684FEA122C86F803C0D4F800C014
:1098C0008CF80420D8E710B503F00700012804D174
:1098D000002211460E2000F07FF9002010BD2DE976
:1098E000F04103F00704AA4E174688460546012CAE
:1098F00004BF0020B06017D013F0070F12D101F0A1
:10990000D5FF78B1B068A34902283CBF0A68175454
:10991000401CB060022807D102220968072000F02D
:109920005BF901E0022C02D00020BDE8F081B268B2
:1099300012B1012A04D009E0FBF72EFF287005E0E0
:10994000FBF730FF2870012088F80000B068401C49
:10995000B0600120BDE8F08170B503F0070000257C
:109960008B4C012808D013F0070F0BD0042804BF3C
:109970002078062825D02DE06561A5616570A56079
:10998000257027E0A068022807D2616942EA012118
:10999000616161781144617010E0042807D2A16907
:1099A00042EA0121A16161781144617006E0052855
:1099B00004D261788A4204BF06212170401CA06055
:1099C00008E0D4E9050101F057FA002804BF01209E
:1099D000A0702570002070BD10B56D4C13F0070FFE
:1099E00007D003F00700042804BF2078062822D0FF
:1099F0002BE0A068022807D2616942EA0121616177
:109A000061781144617013E06349091808D2614913
:109A10000968014401F8022C61781144617007E083
:109A20005E49091804D261788A4204BF0621217078
:109A3000401CA06009E05A49606901F03FFA002823
:109A400004BF0120A07000202070002010BD03F092
:109A5000070CBCF1010F00D0BEE74D490020486162
:109A6000487088600870704730B403F00705002420
:109A7000DFF81CC1012D07D013F0070F0DD0022D08
:109A80003CD0042D54D06FE0CCF81440CCF81840F2
:109A9000CCF808408CF8004066E0DCF808000228AA
:109AA0000BD2DCF8141042EA0121CCF814109CF817
:109AB000011011448CF8011019E0042817D2DCF8C9
:109AC0001810032842EA0121CCF818109CF8013044
:109AD0001A448CF801200AD106228CF80020DCF808
:109AE0001420114304BF4FF4C471CCF818102D4951
:109AF000401CCCF82810CCF8080035E0DCF8082031
:109B0000042A28BF10460AD2C2F10303DCF8285009
:109B1000DB0025FA03F30370501CCCF8080004287E
:109B200003D10120CCF80840087030BC01207047F8
:109B30009CF80000062815D1DCF814000022410230
:109B4000DCF8180043021046B2EB930F06D251F82E
:109B5000045B401C2A44B0EB930FF8D3CCF82820C8
:109B60008CF80040CCF8084030BC002070474FF41F
:109B700043300168880A424211EB822218BF401C20
:109B8000404201EB8000C01C20F003007047000041
:109B900038850010EC050200FEFDFFFFFDFDFFFF14
:109BA00018B70010EFBEADDEFC4800220270427014
:109BB000827002714271C270DFF8E4C3114601EB9A
:109BC000410300200CEB43031A54401C0628FBD32E
:109BD000491C2029F3D3704713F0AAB82DE9F041AE
:109BE00015460E460746F9F73FFC00F0080408202A
:109BF000F9F735FC2A463146384613F099F8054600
:109C00002046F9F727FC2846BDE8F081E348807834
:109C10007047E24840787047E0490020487070473C
:109C2000DE490820887170472DE9F0410026F8F7D9
:109C30007AF9044610F00F0547D02846F8F776F970
:109C4000012D18D0FBF7AEFD44EA00640023224644
:109C50000321072004F0A8FA14F0060F35D00126DE
:109C6000FBF79AFD054604F0F8FF0746022D3CD0AD
:109C7000052D09D029E0FBF78FFDC8498A7990426C
:109C800018BF8871DED1E7E714F0020F20D0F6F795
:109C9000DEFD00281CBF0020F6F7E5FD0120FAF7E5
:109CA000A8FD0120F6F7EBFD0020FAF7B6FD01F064
:109CB00057F9002818BF01F05AF9022F05D0022DDC
:109CC0004FF002001BD001F029F93046BDE8F081C9
:109CD00010F0BDFB007810F0080F0AD0F6F7B7FDC2
:109CE00000281CBF0020F6F7BEFD0120FAF781FD19
:109CF000DDE710F0040F08BF0120D8D1D5E704F04C
:109D0000A7FFE2E72DE9F84F0026FAF712F8FBF774
:109D100043FD022804D101F083FD002818BF01266D
:109D2000FBF73AFD052814D1FAF77DFD88B101F063
:109D300009F95A280DD3F6F78AFD00281CBF002028
:109D4000F6F791FD0120FAF754FD0020FAF765FDC2
:109D50000126FFF769FF002818BF0126DFF83C92B3
:109D600099F80200002800F06E82D9F808006D46CC
:109D70004FF0FF34002740B1D9F80820002301211B
:109D8000084604F011FAC9F80870F9F76DFB00F005
:109D9000080A0820F9F763FB99F80300DFF800B21E
:109DA00000B399F8050000EB4001401CC0B20BEB7A
:109DB000410189F80500202828BF89F8057099F825
:109DC0000300401E89F803004C7891F800800020C1
:109DD000002C05DD0A1892782A54401C8442F9DCD4
:109DE0000F704F705046F9F735FB002CC0F21B8204
:109DF00008F0FF000024272880F0D281DFE800F07F
:109E0000B225F81D28371444F74BB2888EBFF6935D
:109E1000ADF5F4F3F2F1B2B2B2D7F9FEEEB2EDEC79
:109E2000EBEAE9B2E8E7E6009DF80000AC280CBFD9
:109E300001200220FBF774FD07E09DF800100120CF
:109E4000FBF7BFFC012089F80100012400F0A8B94C
:109E50009DF80310009861F31F6001F0CBFF012112
:109E60000320FBF7AEFC012089F80100EDE7BDF807
:109E7000000040BA04F051FE02210320FBF7A1FCD0
:109E8000012089F80100E0E79DF801109DF800002D
:109E9000FBF797FCD9E74FF0010A89F801A099F880
:109EA000000088BBF8F734F870B39DF8005089F8CB
:109EB00000A0FBF771FC012808BF002515F0040F76
:109EC00018BFFDF72CF815F0020F07D0FF210F2067
:109ED000FCF729F8FAF751FE45F0010515F0010FDE
:109EE00010D0FBF759FC022802D104F0B6FE48B1AD
:109EF000FBF752FC052802D101F01BF810B100203D
:109F0000FAF724FE89F8007089F8017000F048B96A
:109F10009DF80000401E01F0B9FA96E79DF8000098
:109F200004F0BCFE91E79DF8000010F00F0F0BD07D
:109F300001200FF06FF99DF80000102100F00F00D4
:109F40000FF044F900F02CB900200FF063F99DF8F0
:109F50000000002100F00F00F2E79DF8000010B1B2
:109F6000012805D01CE100200FF026F9002003E0B5
:109F700001200FF021F901200EF0EAFD10E19DF81B
:109F8000000078B1FBF708FC022818BF012404F098
:109F90006AFE01460220FBF714FC01E17085001007
:109FA00018B9001000210620FBF70BFC4DE79DF8C7
:109FB0000000002818BF012004F03AFE9DF80000C0
:109FC000002818BF012000F09FFFE9E0E4E0DCE09A
:109FD000D6E0B7E0B1E0BAE0A2E05AE013E00DE06D
:109FE00007E085E076E06FE056E047E01DE02EE018
:109FF0009FE09DF8000004F006FED1E0BDF80000EF
:10A0000004F0A9FE21E79DF8000020B101283FD00F
:10A01000022805D0C4E04FF44330F8F721FEBFE03A
:10A0200001F087FC00210420BEE7F9F71DFA00F0DB
:10A0300008040820F9F713FA99F80300002808BF6C
:10A0400089F802702046F9F705FA0121ABE79DF87F
:10A050000000012804BF02210520A5D0022804BF6A
:10A0600000210320A0D0032804BF002104209BD09E
:10A0700004281CBF0221084694D095E79DF80300F0
:10A08000009A002360F31F626221072004F08CF81D
:10A0900086E0FAF78FFFD8E69DF800009DF80110E2
:10A0A000000140EA111009F054FA9DF801109DF8E2
:10A0B000020001F00F0140EA012009F050FA9DF87A
:10A0C000030009F058FA6BE0BDF8000040BA09F04F
:10A0D00034FA65E09DF8000009F060FA9DF801008F
:10A0E00009F068FABDF8020040BA09F06FFA57E0CB
:10A0F0009DF8000009F07FFA9DF801009DF802101C
:10A10000000140EA111009F088FA9DF802109DF84C
:10A11000030001F00F0140EA012009F072FA3FE06C
:10A120009DF800000BF067FC9DF8000000287FF40C
:10A130008CAE0020FAF75DFB87E69DF8000004F086
:10A14000A5FE82E69DF8000004F0A8FE7DE60BF077
:10A1500049FC9DF8004004F073FE012C0AD0022C4B
:10A1600008BF40F0805005D0042C14BF082C40F0EC
:10A17000005001D104F0CEFD20460BF02EFC64E629
:10A180009DF800000FF05BFA0AE09DF800000BF06C
:10A190001BFC04F0F0FC03E09DF8000012F0CDFD84
:10A1A0000CB101263FE0D9F808006D464FF0FF34AE
:10A1B00040B1D9F8082000230121084603F0F4FF3C
:10A1C000C9F80870F9F750F900F0080A0820F9F703
:10A1D00046F999F8030000B399F8050000EB400137
:10A1E000401CC0B20BEB410189F80500202828BFB4
:10A1F00089F8057099F80300401E89F803004C782F
:10A2000091F800800020002C05DD0A1892782A546D
:10A21000401C8442F9DC0F704F705046F9F71AF970
:10A22000002CBFF6E5ADF9F71FF900F0080408208F
:10A23000F9F715F999F80310002908BF89F8027099
:10A240002046F9F707F9002E14BF01200020BDE8D1
:10A25000F88F000002460020022928BF70473AB15B
:10A26000012A0AD0022A04BFF74800EBC100704758
:10A2700040F2DB104843F54904E001EB4100C0EB3C
:10A280004110F34901EB8000704770B5F9F7ECF825
:10A2900000F008060820F9F7E2F8EE4D002468788F
:10A2A000FF2806D240F6D861E84812F0BAFCAC703C
:10A2B000EC70A879FF2805D2E821E54812F0B1FC3E
:10A2C000EC712C72E87AFF280AD2E349C1F8C04346
:10A2D000C1F8C443C1F8C843C1F8CC432C736C73B4
:10A2E0003046BDE87040F9F7B5B8DFF870C300FB41
:10A2F00001F31CEB030C88BF7047D64B9A61C3E98E
:10A3000004017047DFF84CC30028DCF8103018BF98
:10A310000360D0480029406918BF0860002A1CBFAC
:10A32000DCF81810116058437047CA4801210171C8
:10A33000007840F2DB1180F001004843C34901EB93
:10A3400080007047C3488278002132B1C27822B9B8
:10A35000027882F001020270817001717047BD497C
:10A360001E284A78487008BF002003D01F2808BF65
:10A37000012000D1087010467047B648007840F2BE
:10A38000DB1180F001004843B04901EB80007047C9
:10A39000F0B4B04E96F800C040F2DB140CFB04FCA5
:10A3A000AA4C356904EB8C0C03FB05F40CEB440C54
:10A3B0008D4234BF2C460C467669F31A934238BF5F
:10A3C0001A460026002A9CBFF0BC70470023002CD0
:10A3D00006D930F813702CF813705B1C9C42F8D827
:10A3E000761C0CEB450C00EB41009642EED3F0BC22
:10A3F00070472DE9F041974F14468C4601467A7814
:10A4000006981D468A4218BFBDE8F0810121F97007
:10A41000012802D0022824D029E0387840F2DB114C
:10A4200048438A493E6901EB8001A64234BF324667
:10A4300022467869A84238BF05460023002D16D968
:10A440000020002A06D91CF8007021F81070401C6A
:10A450008242F8D85B1C01EB4601A444AB42EFD327
:10A4600005E000232A4621466046FFF791FFBDE83C
:10A47000F04100F0A4BB002808BF70477549784B35
:10A480004A7878491B78002A097818BF022A05D033
:10A49000042A18BF092A01D0012279E7724A1278EA
:10A4A000012A84BF714A1378012200F0A2BB2DE972
:10A4B000F04FDFF8A0A183B001218AF803106C49A6
:10A4C000694C6A4D0F7866490E789AF80110112987
:10A4D00030D00EDC002918BF02291DD0042918BF76
:10A4E000092919D098B1002332463946FFF750FFA9
:10A4F0000DE0122918BF13291CD0212918BF2229C9
:10A50000F0D120B10023B21C3946FFF741FF03B060
:10A51000BDE8F04F00F053BB2178012902D955491D
:10A520002E780F780028F2D000233246394600F00A
:10A5300060FBECE7F7F7EDFBF7F726FB0090002850
:10A5400018BFF7F774FD2078012888BF2E78F7F739
:10A55000E7FC10F0040F18BF761CDFF81C919AF886
:10A560000100A0F111089AF8000040F2DB11484305
:10A57000364901EB8004DAF81000B84238BF0746CC
:10A58000DAF81400B04238BF0646F7F799FD01909B
:10A590000020F8F7B4F80025002E39DD4FF0000A4E
:10A5A000002FC4BF05EB450000EB051B29DD01981A
:10A5B00010F90A00262824BF002024F81A001CD213
:10A5C00000F0010109EB413100EBD07001EB8B0190
:10A5D0004010B8F1000F51F820104FF0FF301DD09F
:10A5E000B8F1010F08BFC8B205D0B8F1020F04BF1F
:10A5F0000846F8F78AF824F81A000AF1010ABA4561
:10A60000D5DB14486D1CB542006904EB4004C5DB82
:10A610000098002818BFF7F70DFD78E711F4803F88
:10A62000C1F3072018BF4042E5E70A480121417203
:10A63000407980F0010000EB4001C1EB401004497B
:10A6400001EB80007047000098C90010D8B90010D5
:10A65000B0C800107C850010D8C500104AFCFFFF70
:10A66000FF84001005850010008500100285001091
:10A67000FE8400100185001000800030FC48C27983
:10A68000002132B1027A22B9427982F0010242718C
:10A69000C17141727047F6491E288A79887108BFD6
:10A6A000002003D01F2808BF012000D148711046A8
:10A6B0007047EF48407980F0010000EB4001C1EBAA
:10A6C0004010EC4901EB800070472DE9F04FEA495A
:10A6D00085B0012291F80080E84991F80090E449A2
:10A6E0000A728979E34C11291CBF1229132936D02B
:10A6F000F8B1DF49497901EB4102C2EB411104EBAA
:10A700008102002119EB080C18BFDD4C11D0236821
:10A71000B9F1000F5B8A03BF30F811500B4422F8E7
:10A72000135030F8113018BF22F81130491C8C45F5
:10A73000EDD8F8F799FE00F008050820F8F78FFE2D
:10A74000CB4C607A002818BF01217CD0E1712846EB
:10A75000F8F780FE0020207205B0BDE8F08FF7F713
:10A76000D8FAF7F711FA0190002818BFF7F75FFC45
:10A77000BF488179A1F11105C1690091407900EBD1
:10A780004001C1EB401004EB8006F6F7C4FBBD4F5F
:10A79000BD494FF0110A002804BF8B46012004D0A8
:10A7A000BB4650460F464FF0010AF7F7A8FFF7F7F0
:10A7B00085FC00240390B9F1000F28D900984C21A2
:10A7C0004843029003980057262824BF002026F80B
:10A7D000140019D200F001010BEB413200EBD070F4
:10A7E0000299401001EB8000002D11584FF0FF300E
:10A7F00049D0012D08BFC8B204D0022D04BF0846BD
:10A80000F7F783FF26F81400641C4C45DAD306EBF7
:10A8100049065046F7F773FFF7F752FC00248246CB
:10A82000B8F1000F29D900984C2100FB01F94FF035
:10A83000000B1AF90400262828BF26F814B019D2F4
:10A8400000F0010100E02CE000EBD070401007EBBD
:10A85000413109EB800009584FF0FF30D5B1012D8F
:10A8600008BFC8B204D0022D04BF0846F7F74DFF59
:10A8700026F81400641C4445DBD30198002818BF57
:10A88000F7F7D8FB55E711F4803FC1F3072018BF55
:10A890004042B7E711F4803FC1F3072018BF4042A0
:10A8A000E6E7607980F00100607100214EE77048B2
:10A8B00001218173807A754980F0010001EBC000AD
:10A8C00070476B48027B002132B1427B22B9827A09
:10A8D00082F00102827201738173704764491E28FD
:10A8E000CA7AC87208BF002003D01F2808BF012001
:10A8F00000D18872104670475D48807A634980F0C5
:10A90000010001EBC00070472DE9F04F584987B0B6
:10A9100001224A73C97A5D4D5D4C11291CBF122971
:10A9200013292CD0A8B15249897A237805EBC102AA
:10A9300094F801C0002113EB0C0F0AD030F811304D
:10A9400022F81130237894F801C0491C63448B42EB
:10A95000F4D8F8F789FD00F008060820F8F77FFD25
:10A96000434CA07B002500281CBF012121737DD012
:10A970003046F8F76FFD657307B0BDE8F08FF7F765
:10A98000C8F9F7F701F90490002818BFF7F74FFB53
:10A99000404805902078617800EB01083449C87A76
:10A9A0008A7AA0F11109C869896905EBC20B414592
:10A9B00038BF88460221029112210391002500EB45
:10A9C00040012E4601EB001A02AC54F82600F7F7BE
:10A9D00096FE54F826000021F6F71DFE009054F86C
:10A9E00026000121F6F717FE019006EB46000599B7
:10A9F00000EB0610002401EBC0072EE0E01704EB8B
:10AA0000D060421120F01F005DF82210221A0120B0
:10AA10009040014220D004F0010007EB403004EBED
:10AA2000D47100EB8A00491000EB810141F64860C7
:10AA3000B9F1000F09584FF0FF3032D0B9F1010FD2
:10AA400008BFC8B205D0B9F1020F04BF0846F7F736
:10AA50005CFE2BF815006D1C641C4545B8BF262C08
:10AA6000CCDB761C022EAFDB049815E020E0000062
:10AA70007C850010B0C8001003850010048500100C
:10AA800064860010B09D0030189D003098C90010F9
:10AA90000685001000800030002818BFF7F7CAFABA
:10AAA00057E711F4803FC1F3072018BF4042D0E7B9
:10AAB000A07A80F00100A072257359E770B50D46A9
:10AAC0006E490122CA706E4A497816786D4A21296A
:10AAD00014781EBF2229232970BD002818BF002D1D
:10AAE00011D0002322463146FFF752FC631C01229D
:10AAF00021462846FFF74CFC05EB4400A31C01222D
:10AB00003146FFF745FCBDE8704000F058B870B51D
:10AB10005A4D0446687868B9E06858B15A490978CE
:10AB2000012994BF574959490B785949012209789D
:10AB300000F05FF8E87A112804BF0020FFF7E4FE78
:10AB4000E87A122804BF0020FFF7DEFEE87A132817
:10AB500004BF0020FFF7D8FE6878002804BFA06873
:10AB6000FFF7A5FC6878112804BF0020FFF79FFCC1
:10AB70006878122804BF0020FFF799FC6878132832
:10AB800004BF0020FFF793FC206920B1A9790029B8
:10AB900008BFFFF79AFDA879112804BF0020FFF72E
:10ABA00094FDA879122804BF0020FFF78EFDA87934
:10ABB000132818BF70BD0020BDE8704085E570B552
:10ABC000F8F752FC00F008060820F8F748FC2B4C78
:10ABD00020790025002801BF207880F00100207036
:10ABE000A5701CBF0120A0703046F8F733FCE5705B
:10ABF00070BD2DE9F047994616460D460446F7F715
:10AC000064FA5FEA000C1CD01C49087840F2DB12A1
:10AC10005043204AD1F8108002EB800009FB08F273
:10AC200000EB4200454594BF2F4647464969A1EBDA
:10AC30000901B14238BF0E460021002E09D8BDE8F7
:10AC4000F0874B46324629462046BDE8F047FFF7DD
:10AC50009FBB0023002F08D91CF9032034F81220D1
:10AC600020F813205B1C9F42F6D8491C00EB4800DB
:10AC700004EB4504B142ECD3BDE8F0877C850010BD
:10AC8000FE840010FF840010008500100285001073
:10AC900005850010D8B900105849002814BF0020BD
:10ACA0000120087070475548007800280CBF01202B
:10ACB000002070475148017829B14FF040214A697E
:10ACC00042F001024A61002141608160C16001617E
:10ACD00070474A48017829B14FF040214A6942F053
:10ACE00001024A61002141608160C16001617047D9
:10ACF00070B50446F8F7B8FB00F008050820F8F72F
:10AD0000AEFB3E4A3E490023D06801EBC001401C27
:10AD1000D060B0F5807F28BFD3602078087060785D
:10AD20004870A0788870E078C870207908716079E0
:10AD30004871A0798871E079C8711069B0F5807F99
:10AD40003CBF401C106116D31D20087001204870C4
:10AD5000207888706078C870A0780871E0784871B1
:10AD6000207988716079C8719068401C9060B0F556
:10AD7000807F28BF9360506840F0010050601078D9
:10AD800028B14FF04020416921F00101416128467E
:10AD9000F8F760FB012070BD00B50178427883B000
:10ADA000890141EA82018DF80010418809098DF876
:10ADB0000110818809098DF80210817801F00F02D5
:10ADC000017962F31F118DF80310017A8DF80410D8
:10ADD000417A8DF805108179C27901F03F0102F0C6
:10ADE0000C0241EA02118DF80610C07980018DF83D
:10ADF00007006846FFF77CFF03B000BD9C8500108C
:10AE0000A8C90010194A002112684FF0402312F01F
:10AE1000804F26D0164AD2F800C05FEA1C4C04D0FE
:10AE200011686FF30F0141F00101D2F800C01CF46A
:10AE30007F4F0CD011684FF0020C01F47F414CEAB7
:10AE40000121DFF830C0DCF800C0C3F874C0D2F8CC
:10AE500000C01CF0FF0F04D011680322C9B242EAFF
:10AE6000014199678069D867FEE700002CED00E09A
:10AE700028ED00E038ED00E070B50E460446FAF724
:10AE80008BFC042811D1A4F59C7050280DD2A01978
:10AE9000A0F23910502808D265020024002E04D9EF
:10AEA0002846F7F7DDFE012801D0002070BD641CA4
:10AEB00005F50075B442F3D3012070BD70B50D46A1
:10AEC0000446FAF769FC04280AD1A4F59C705028BE
:10AED00006D260022946F7F765FF012808BF70BD5A
:10AEE000002070BD10B5074CFEF70CFF012808BF0D
:10AEF00010BD206800F0E4FD002818BFFAF7A4FC9C
:10AF0000F2E7000064860010FE4A0028516814BF72
:10AF100041F0010021F0010050607047F94B596881
:10AF20000A0E120721F07F4142EA00600843586090
:10AF30007047F4484068C0F303607047F1484068C8
:10AF4000000F7047EF4880687047EE48806970478F
:10AF5000EC49012088617047EA4900208861704708
:10AF6000E84840697047E749012048617047E54972
:10AF70000020486170472DE9F041AEB000270EF087
:10AF800070FB0646A02102A811F04BFE00242546C6
:10AF90004FF00308305D10F0800F18D0601C8DF862
:10AFA000A9008DF8AF508DF8A880ADF8AC508DF8A1
:10AFB000B050ADF8AA508DF8AE508DF8B1508DF864
:10AFC000B450355501272AA902A8F5F795FA601C57
:10AFD000C4B20A2CDED3012F06D1102302AA062107
:10AFE000012000950FF062FA0EF03DF92EB0BDE899
:10AFF000F0812DE9F04FDFF8109387B0D9F8000009
:10B00000B0F90E11B0F90C0111F065FEF5F73CFB3B
:10B010000120F9F7EEFB0020F7F719F80EF0FEFA21
:10B02000042000F04CF9F9F7E2FB0AF010FD0028CB
:10B0300018BF0AF096F8FAF7AFFB05285ED1DFF8E3
:10B04000C4824FF0000A4FF0402BD8F80400C8F833
:10B0500008A0C8F80CA0C0F30365C8F810A0D9F880
:10B060000000A900D0F8F80020FA01F101F00F0467
:10B07000C0F30327C0F30336BC420FD10F2E0DD00F
:10B0800003F039FE20B10AF0ADFC082818BF3446A1
:10B09000D8F81C00A04218BFC8F81C404FF48056D6
:10B0A000BC4205D103F01AFE002808BF4FF4006629
:10B0B0003046FAF7BCFC2946052003F003F9002DC1
:10B0C0007ED0022D30D0042D7BD0D8F804000A2D7C
:10B0D0004FEA106120F07F404FEA017118BF41F044
:10B0E00000710843C8F80400FEF70CFE012805D0E3
:10B0F0000EF0B9F8FAF750FB0528A6D0F9F778FB5F
:10B100000EF091FA4FF48050FAF791FCFAF744FBF5
:10B11000022818BF00207CD0F5F748FB07B00020BC
:10B12000BDE8F04FF5F7ABBB25460D240AF0EAFB6E
:10B13000002818BF0C2421462846FAF788FC00286E
:10B14000D2D011F0FFFD11F002FEF9F7FCFA040075
:10B1500072D1F6F751F96D48F6F761FD0120F6F767
:10B1600051FDF8F7A3F96A48F8F755FAF8F73CFAF1
:10B17000F8F765FA4100D9F80000B0F80621B1FBF4
:10B18000F2F1491CC1F34F01A8F8021090F8080130
:10B1900088F8000058B1F8F752FAD9F800104000CA
:10B1A000B1F80411B0FBF1F0401CC0F34F010846A8
:10B1B000F8F7B6F95748CBF81800F6F7AAFD01E002
:10B1C00060E063E0F6F7F9FE98F8000048B1401E31
:10B1D00010F0FF0088F8000004BFB8F80200F8F78C
:10B1E0009FF9D8F80400C0F3036529460520F5F758
:10B1F0007EF8FEF787FD012807D0D8F80400C0F3D9
:10B200000360A84208BF002C1DD0F7F736F942486A
:10B2100000E03FE0CBF81800F8F7BAF9F8F7EFF9DB
:10B220000020F8F7F8F9F8F74AF9F6F772FDF6F7A3
:10B23000ADFC0020F6F7F3FC11F089FD11F08CFD58
:10B24000FAF77EFD50E76846F7F7BAF870B168463E
:10B25000FFF75DFC0198F8F7BAFD684611F081FD33
:10B260000446F7F70AF9FAF710FBC2E7D9F800002D
:10B27000406E10F0704F02D0FAF7E6FAB9E7FAF72D
:10B280000BFBB6E7204611F071FD2DE7204603F0D9
:10B2900062FF29E7F5F7E1FA10B9F5F7D8FA38B106
:10B2A0000020F5F7E0FA0020F5F7DAFA012033E79D
:10B2B0000120F5F7D8FA0020F5F778FA2EE770B5F7
:10B2C000114980000968D1F8F81021FA00F000F067
:10B2D0000F04C1F30326C1F30335B4420ED10F2D81
:10B2E0000CD003F008FD20B10AF07CFB082818BF41
:10B2F0002C460448C169A14218BFC4614FF480556F
:10B30000B4420BE0B0850010648600103D3E001092
:10B310002737001007005FA000005FA005D103F0F1
:10B32000DDFC002808BF4FF400652846FAF77FFBD4
:10B33000204670BD7047002808BF70478022014634
:10B34000014811F069BC7047A8D100107047082867
:10B350003CBFFE49087070470020FC498860486087
:10B36000FB48006890F88100082838BF08707047D3
:10B370000020F64948607047F4480078704770B57F
:10B38000F34D0024286890F86C0010F0020F0BD0E9
:10B39000FAF702FA022807D1EC482968007801EB95
:10B3A0008000B0F8840084B2204670BD70B5E84DCE
:10B3B0004FF48054286890F86C0010F0020F0DD004
:10B3C000FAF7EAF9022809D1E0482968007801EB88
:10B3D0008000D0F88400000CC0F31304204670BD38
:10B3E000DA488078002818BF012070472DE9F04125
:10B3F000FAF7D2F9022803D103F02FFC022803D078
:10B400004FF48050BDE8F0814FF480552E4603F094
:10B4100042FCDFF83C830446CC4FD8F8000090F89B
:10B420006C1011F0010F0CD0B0F87600B9684042F2
:10B43000814206DC2CB10020641EB860204603F077
:10B440002DFCD8F8001091F86C0010F0040F18BF14
:10B45000002C0AD0B1F87C00621E9040B1F87E202A
:10B46000824238BF1046C0F31306D1F8A40010F092
:10B47000020F1CBFB978002902D0000CC0F31305DD
:10B48000B54298BF35462846BDE8F0812DE9F04F1A
:10B49000DFF8BCA287B0DAF8001091F86C2012F047
:10B4A000020F0DD0A94A91F88090DFF8A8B2177862
:10B4B000002809DB484503D2B84218BF064643D1ED
:10B4C00007B00020BDE8F08F3E464FF0FF38F6F79A
:10B4D0005DFBF7F77FF90025B9F1000F34D9DAF8F1
:10B4E0000000002400EB8500B0F8840081B2204603
:10B4F000F5F7A1FFF6F761FD6846F6F761FF002852
:10B5000066D0029878B1014693489BF800200078F5
:10B510005043421E07D331F9020B0028B8BF404206
:10B520000444521EF7D2F6F7A8FFF6F72FFB0023CC
:10B5300022469221072002F037FEA04584BF2E4606
:10B54000A0466D1C4D45CAD3B74244D0082E3CBF1F
:10B550007E490E70DAF80000B0F8821039B300EBC3
:10B56000870200EB8600B2F88420B0F8840092B223
:10B5700080B2801A484340F30F34F8F79DFC774BB4
:10B580009BF80020002193F800C002FB0CF2002A77
:10B590000DD930F81120224420F811209BF800200A
:10B5A00093F800C0491C02FB0CF28A42F1D84FF418
:10B5B000800003F07CFCDAF80000002300EB86003A
:10B5C0008021B0F8840082B2072002F0EDFD09E08E
:10B5D000FAF73AF990E703F05EFB03283CBF401C02
:10B5E00003F05CFB012007B0BDE8F08F58485749D5
:10B5F0000068B0F87600424288688242BCBF401EB4
:10B60000886070472DE9F04F93B093460E4604468C
:10B610004FF0000A03F03FFBDFF834814B4F050089
:10B62000D14610D111F0A7FBD8F80010B1F878106E
:10B63000884208D30120C7F8089003F02FFB13B00D
:10B640000120BDE8F08F002E1FDDB8680028B8BFCC
:10B65000C7F8089007DBD8F80010B1F874108842DA
:10B66000BCBF401CB860D8F80000B968B0F87400DE
:10B67000884215DC032D13D2681CC7F8089003F02C
:10B680000DFB13B00120BDE8F08F09D1D8F8000000
:10B69000B0F876004142B8688842C4BF401EB86026
:10B6A000B87850B1D8F8000090F8A40010F0040F5A
:10B6B0001EBF002013B0BDE8F08FD8F80000B0F92D
:10B6C00072108C420EDD796821447960B0F86E000A
:10B6D000884210DC4FF0FF30C7F80490FFF7D6FE29
:10B6E000824608E07868002805DD002CD4BF0121DF
:10B6F0002146401A7860DFF8689099F80000072822
:10B700003BD11848594600784200684611F093FA38
:10B71000ADF80040ADF80260ADF804503889ADF8DE
:10B720000600B888ADF80800D8F80000B0F872102C
:10B73000ADF80A10B0F87410ADF80C10B0F86E1037
:10B74000ADF80E10B0F876000EE00000488600104C
:10B7500064860010FE84001002850010FF84001033
:10B760007D85001005850010ADF8100099F80000E7
:10B77000072804BF6846FEF77EFE504613B0BDE8BA
:10B78000F08F3E4810B50068D0F8A40010F4807F18
:10B7900006D0C0F30330012101FA00F0F7F7D1FB26
:10B7A000374900204870887010BD70B5344D0024B2
:10B7B000A878002814BF01260026687828B903F06D
:10B7C00079FA002808BF002100D001218E4225D03F
:10B7D0000A1C18BF0122AA7028480068D0F8A430BB
:10B7E00013F0040F0ED021B1C3F30310082808D2C0
:10B7F00006E00021A960696090F88100082800D265
:10B800002870012413F0020F18BF0124002A18BF6A
:10B81000012200238221072002F0C6FC204670BDD1
:10B82000164900200968D1F8A41011F4807F08BFE0
:10B830007047DFF84CC09CF80120131C18BF01238F
:10B8400030B4104CC1F30332E46B012505FA02F267
:10B85000224011F4007F01D00AB102E00AB10021B8
:10B8600000E001218B4204BF30BC7047081C18BFA8
:10B8700001208CF8010030BC97E7000064860010BE
:10B88000488600100010004007480078704710F507
:10B89000967FA8BF7047012003490870704702498E
:10B8A000002008707047000054860010704800782F
:10B8B00070476F48406800F5407070476C484068BA
:10B8C00000F58070704770B5694C4FF41C326949BF
:10B8D00062601068884204BF5068B0F5087F26D1C6
:10B8E000D2F808C0BCF5064F21D86349D068884219
:10B8F0000DD0002311461846B3EB9C0F07D251F828
:10B90000045B401C6B40B0EB9C0FF8D37BB9012566
:10B9100002F5807000F0D4F848B1606800F540701E
:10B9200000F0DDF800281EBF2570012070BD00204A
:10B9300070BD4F49002008704FF41C30F7F790B9E4
:10B940004B48017841B140684A4A0168914202BFC0
:10B950004168B1F5087F704700207047444B5B6831
:10B9600003F580731844F7F771BA414B5B6803F530
:10B9700040731844F7F76ABA3D4840680069704759
:10B980003B4949680A6982429CBF00207047C0EB6E
:10B99000C00001EBC00000F580607047344A526877
:10B9A00002EB80035B6A1A44344B53F820C04033E7
:10B9B00033F810000CEB0003401E5B1E23EA00006E
:10B9C00000FB012070472A4988607047284880683A
:10B9D00070472DE9F00F264B0022DFF8A080D3E955
:10B9E0000145012708F140069146831893F928C0C4
:10B9F000BCF1000F18DB07FA02F32B4214D0D3B2CC
:10BA000004EB830A58F823B036F81330DAF824A090
:10BA10009B445B1EABF1010BA2442BEA030303FB27
:10BA20000CA341F8223001E041F82290521C102A68
:10BA3000DBD3BDE8F00F70470029B8BF704730B4C2
:10BA400094460B4A0E4C526802EB80035B6A134427
:10BA50000A4A52F8202034F810001418401E641EC0
:10BA600024EA000001FB003030BC6146F7F7EEB974
:10BA70005886001054465053EFBEADDEF00502006C
:10BA80003006020010B5FFF71EFFA8B1FFF711FF47
:10BA90000146D022174811F0BFF8FFF70FFF164CF0
:10BAA00001464FF4E272206811F0B6F82068406D4C
:10BAB000BDE8104003F075B80220F9F731FFE2E766
:10BAC00058B10E4A0168914207D1406820F00F003A
:10BAD000B0F5107F04BF012070470020704730B1DF
:10BAE000006820F00F00602804BF0120704700208C
:10BAF000704700001011011064860010415053522D
:10BB0000B44810B5806810F0020F15D0F6F73CF875
:10BB100090B1F5F7FCFF0402F9F73EFE44EA004459
:10BB2000F9F740FE44EA00604EF2AF0108434FF0DF
:10BB30004021C867012010BD002010BD10B572B6AD
:10BB40000120F6F791FFF7F735FEF7F75FFE4FF0AC
:10BB5000FF30F7F784FCA04880234FF40052002107
:10BB600052F821C040F821C0491CB1EB930FF7D324
:10BB7000F7F787FCF8F7A2F8F8F7C4F89748F8F752
:10BB8000DDF80120F8F79BF8F7F702F81E20F8F728
:10BB90008BF8F7F757FEF7F7DFF9F8F747F8F7F7FD
:10BBA00097FEF7F77FFCF7F74FFAF6F702F8FFF783
:10BBB00069FFF7F7FEFBF7F7C9FBFDF7F5FFFBF7AA
:10BBC00023FAFFF786F862B6F9F737FF844C20684E
:10BBD00090F8640000F00F00F6F76CFE2068018B0F
:10BBE000C1F30722418A008AFEF77FFB2068806E3E
:10BBF000000C02F0D6FA7B480DF012FB2068B0F979
:10BC00000C010DF009FDF4F756FBFFF79FFBF8F769
:10BC1000B1F8FAF725F9FFF78DFB11F0B1F82068BC
:10BC200090F8200010F0010F04BF0021032003D082
:10BC300003F019F801460220F9F7C3FD4FF0402444
:10BC40002069002300F070021946022002F0ACFACD
:10BC5000206910F0200F17D0226F00230521072044
:10BC600002F0A2FA626F00230521072002F09CFA7D
:10BC7000A26F00230521072002F096FAE26F00234D
:10BC80000521072002F090FAFFF77BFD00202067D6
:10BC900010BD0225544CFEF735F8012806D0F9F7FF
:10BCA0007BFD032802D102F03AFB48B3002C05DCEF
:10BCB00002F0D9FF01460220F9F783FDDFF8309149
:10BCC0004FF00108494F4FF04026A9F1030AF9F758
:10BCD00063FD0446F9F766FD0146204602F0F2FADC
:10BCE000F9F760FD01462046F4F701FBFDF798FFE8
:10BCF000072C6BD2DFE804F06A1D08272A192D00F3
:10BD0000641E002CC7DCD3E7387850B9FBF7B1F8D4
:10BD100038B900231A462021072002F045FA87F897
:10BD2000008003F006FD0225D1E7FFF762F9052543
:10BD3000CDE7FBF704F8F9F72FFD012804BF2846EB
:10BD4000F9F73CFDC3E702F08FFEC0E7FFF7CAF842
:10BD5000BDE70024C6F81890FDF7D4FF012806D1EE
:10BD6000F9F71AFD062802D0C6F818A0AFE7F9F7D0
:10BD700016FD40B3002C04DCF9F77CFD43F220549F
:10BD8000EAE7641E00BF00BF00BF00BF00BF00BFE6
:10BD900000BF00BF00BF00BF00BF00BF00BF00BFAB
:10BDA00000BF00BF00BF00BF00BF00BF00BF00BF9B
:10BDB00000BF00BF00BF00BF00BF00BF00BF00BF8B
:10BDC00000BF00BFC8E7F9F73FFDC5E70220F9F75C
:10BDD000A7FD7CE70080004000140110B1DA0000EC
:10BDE0006486001010110110FF70020068860010B8
:10BDF00003005FA0FE4908607047FD494860704736
:10BE0000FB4810B44068002808BF4FF44030F94A9E
:10BE1000016891421CD14168B1F5007F18D3836855
:10BE200000228446B3F5056F88BF4FF405630021F7
:10BE3000B1EB930F24BF10BC70475CF82140491C44
:10BE40002244B1EB930FF8D3002A04BF10BC704713
:10BE5000002010BC704770B50022C260D0F808C046
:10BE6000012113460446BCF5056F88BF4FF4056CED
:10BE70000022B2EB9C0F06D254F82250521C2B44E5
:10BE8000B2EB9C0FF8D35A42C260D94A127812F032
:10BE9000800F07D14FF440304FF405622146F6F78A
:10BEA000D5FF014601290CBF0120002070BDFF22F3
:10BEB00070B50025044605614FF40061503010F064
:10BEC000D8FEA584E584E562A56265632563E56324
:10BED000A56365642564E5640120A56470BD2DE952
:10BEE000F0414FF440310446C24E0868B04218D1C8
:10BEF0004868B0F5007F14D38A6800230D46B2F578
:10BF0000056F94BF94464FF4056C0020B0EB9C0F76
:10BF100026D255F82070401C3B44B0EB9C0FF8D360
:10BF2000F3B1FF224FF40561204610F0A2FE4FF45A
:10BF30000870C4E900604FF40560A0600020E06074
:10BF400084F8200084F8210084F8220084F823007B
:10BF500020616061A061E0612046FFF7A8FF07E073
:10BF6000B2F5056F88BF4FF40562204610F054FE0D
:10BF70000120BDE8F08170B402684FF4087151608F
:10BF8000016801F1500291F821C091F820300CFBBA
:10BF900003F102EB41010022BCF1000F08D900EBD4
:10BFA0004204521CB4F8EA4021F8024B9445F6D8FA
:10BFB0000022002B08D900EB4204521CB4F81241B5
:10BFC00021F8024B9342F6D80468002294F82240EC
:10BFD000002C0BD900EB4204521CB4F8BE4321F8EC
:10BFE000024B046894F822409442F3D8046800227B
:10BFF00094F82340002C0BD900EB4204521CB4F8F7
:10C00000CE4321F8024B046894F823409442F3D8BD
:10C010000022BCF1000F08D900EB4204521CB4F816
:10C02000704021F8024B9445F6D80022002B08D925
:10C0300000EB4204521CB4F8984021F8024B9342A2
:10C04000F6D8B0F8E62021F8022BB0F8E82021F865
:10C05000022BB0F8E42021F8022B00240022BCF1CE
:10C06000000F0ED904EB440505EB041500EB850524
:10C0700005EB4206521CB6F85E6121F8026B624580
:10C08000F6D30022002B0ED904EB440505EB041572
:10C0900000EB850505EB4206521CB6F88E6221F8CE
:10C0A000026B9A42F6D3641C042CD7D30023D0F839
:10C0B00000C000229CF822C0BCF1000F88BF00EB3A
:10C0C000031C0BD90CEB4204521CB4F8DE4321F8DC
:10C0D000024B046894F822409442F3D8D0F800C090
:10C0E00000229CF823C0BCF1000F88BF00EB031CAA
:10C0F0000BD90CEB4204521CB4F8FE4321F8024B5E
:10C10000046894F823409442F3D85B1C022BCED3EE
:10C1100070BC70472DE9F74F88B000250A992C466E
:10C120002E460968049101F150030999002984BF42
:10C130003149D1F800801CD90022002888BFB8F905
:10C14000CE700DD933F9021B0029B4BFC1F1000C28
:10C150008C46BC45BCBF0D44641C521C8242F1D3CA
:10C160000999761C8E42E7D3002CC8BF95FBF4FAE0
:10C1700008DC4908414301EB5002049901EB4201FC
:10C18000B1F950A000210291019104995031009120
:10C19000002103910999002975D91749009E069637
:10C1A00009684FF0000B4FF00109B1F9C0E0D1F878
:10C1B000B4105F46C1F30741D846CDF814B00791DB
:10C1C000002830D9B6F900204FF0000C06999344AE
:10C1D0006346002814D9B1F90040A51A48BF151BC1
:10C1E0007545B8BF0CF1010C01EB49015B1C05E082
:10C1F0006C86001053454C46648600108342EAD397
:10C2000007998C4503D305997F1C1144059108F1CA
:10C21000010806EB49068045D4D3002FC4BF059919
:10C2200091FBF7F101DC9BFBF0F1039B0A9A09B249
:10C2300002EB4302A2F87010FE4A1268B2F9BA305B
:10C24000AAEB030399420ADDB2F9B82052448A42AC
:10C2500005DD019A114401910299491C029100994E
:10C26000099A01EB400100910399491C0391914205
:10C2700093D30299002906DDDDE9011291FBF2F169
:10C28000019103E0FFE75146CDF804A00A9AA2F815
:10C29000E610002102910391049950310091002190
:10C2A0000491002868D9E349009F069709684FF078
:10C2B000000B099EB1F9BCE0D1F8B410D846090EC4
:10C2C000D946CDF814B00791002E2BD9B7F900202C
:10C2D0004FF0000C069993446346002E0DD9B1F936
:10C2E0000040A51A48BF151B7545B8BF0CF1010CDD
:10C2F00001EB40015B1CB342F1D307998C4504D399
:10C30000059908F101081144059109F1010907EBAC
:10C310004007B145DAD3B8F1000FC4BF059991FBCE
:10C32000F8F101DC9BFBF6F1049B0A9A09B202EBDF
:10C330004302A2F89810BF4A1268B2F9BA30AAEBC9
:10C34000030399420ADDB2F9B82052448A4205DD5E
:10C35000039A114403910299491C02910099891C86
:10C3600000910499491C049181429CD302980028B1
:10C37000C4BF039991FBF0FA0A98A0F8E8A00198CD
:10C380000A99504400B200EBD0704010A1F8E400CC
:10C390000BB0BDE8F08F2DE9F04F146889B0154659
:10C3A0000E460746A1F12008202928BF4FF0FF3A8A
:10C3B00005D24FF0010000FA06F0A0F1010A38BFE3
:10C3C0004FF0000B05D34FF0010000FA08F0A0F188
:10C3D000010B202F3DBF0120B840401E4FF0FF3021
:10C3E00038BF002207D3A7F120024FF0010101FA64
:10C3F00002F1A1F10102C6F12009202E34BF20FA7A
:10C4000009F100FA08F1B2401143B040CDE9000152
:10C41000206920F4FE6020618748007810F0010F49
:10C420007ED02A463146384601F07FFC0020A861C4
:10C430006861002F84BFDFF8FCE101221BD905EB06
:10C440004001B1F998100029B8BF494209B2DEF89D
:10C450000030B3F9CC308B420ADD410905EB810194
:10C4600000F01F0C4B6902FA0CFC43EA0C034B6111
:10C47000401CB842E3D30020012F18BFA7F1010EE2
:10C480003BD005EB4001B1F99A30B1F99820991AE7
:10C4900048BFD11A09B2DFF89CC1DCF800C0BCF972
:10C4A000C4C08C4526DAB5F9E810B2EB010C48BFE0
:10C4B000A1EB020C0FFA8CFC5A1A48BFCA1A11B22F
:10C4C0008C450BDB420905EB820100F01F0C0122B9
:10C4D0004B6902FA0CF21A434A610BE0411C4B090A
:10C4E00005EB830201F01F0C0121536901FA0CF1E5
:10C4F00019435161401C7045C3D36969E869B14073
:10C5000008432063A969286AB140014361636869EF
:10C51000202E34BF20FA09F000FA08F0084300E0AA
:10C5200000E0606344480068079010F0040F00F0DA
:10C53000BC8100202863E862002E88BFDFF8F4E0A9
:10C540001BD9DEF8002005EB4001B1F95E11B2F90C
:10C55000D8308B4203DCB2F9DA208A420ADA420987
:10C5600005EB820100F01F0C0122CB6A02FA0CF2EB
:10C570001A43CA62401CB042E3D30020A86268623A
:10C58000002F88BFDFF8ACE01BD9DEF8002005EBF8
:10C590004001B1F98E12B2F9D8308B4203DCB2F906
:10C5A000DA208A420ADA420905EB820100F01F0C08
:10C5B00001224B6A02FA0CF21A434A62401CB8424A
:10C5C000E3D300202864E863002E88BFDFF864E02E
:10C5D0001BD9DEF8002005EB4001B1F9AA11B2F930
:10C5E000DC308B4203DCB2F9DE208A420ADA4209EF
:10C5F00005EB820100F01F0C0122CB6B02FA0CF25A
:10C600001A43CA63401CB042E3D30020A8636863A6
:10C61000002F88BFDFF81CE020D9DEF8002005EBF2
:10C620004001B1F9DA12B2F9DC308B4208DCB2F920
:10C63000DE2003E0648600106C8600108A420ADA6D
:10C64000420905EB820100F01F0C01224B6B02FA3C
:10C650000CF21A434A63401CB842DED3002028651E
:10C66000E864A8646864002E88BFDFF844E71CD93A
:10C67000DEF8003005EB4001B1F9F611B3F9E02026
:10C680008A4203DCB3F9E2208A420BDA410905EB66
:10C69000810C00F01F030121DCF84C20994011436C
:10C6A000CCF84C10401CB042E2D30020002F88BFD1
:10C6B000DFF8FCE61BD9DEF8002005EB4001B1F9FC
:10C6C0002613B2F9E0308B4203DCB2F9E2208A4251
:10C6D0000ADA420905EB820100F01F0C01224B6CC3
:10C6E00002FA0CF21A434A64401CB842E3D3696A66
:10C6F000E86AB14040EA010EC4F838E0A96A286B44
:10C70000B1400843E063696A202E34BF21FA09F181
:10C7100001FA08F141EA0000E0630590696BE86BFB
:10C7200001FA06F140EA01022264A96B286C01FAC1
:10C7300006F140EA01006064696B34BF21FA09F137
:10C7400001FA08F141EA000161646B6CE86C03FADC
:10C7500006F340EA0300A0640490AB6C286D03FA72
:10C7600006F340EA0300E0646B6C34BF23FA09F37C
:10C7700003FA08F343EA0000E0640290059832EA05
:10C780000E0521EA000C4EEA05022564069240EAF5
:10C790000C00C4F844C006EB0701039008BFBCF1CD
:10C7A000000F42D000231A461846002988BF0127EF
:10C7B0003BD94FEA501804EB880800F01F09D8F85D
:10C7C000408007FA09F918EA090F03D0864294BF9E
:10C7D000521C5B1C401C8142EBD8012B0FD105EA97
:10C7E0000A0040EA0E00A06305980CEA0B03184308
:10C7F000E06325EA0A0020642CEA0B006064012A49
:10C8000013D1226C0098A36B10401843A063606C96
:10C81000019BD4F83CC0034043EA0C03E363009B54
:10C820009A432264019A90436064069A049830EA1D
:10C830000202A264069840EA020CDDE9020320EA43
:10C840000300E064039B43EA000508BF002821D0F1
:10C8500000231A461846002988BF012717D94FEA36
:10C86000501804EB880800F01F09D8F8488007FA30
:10C8700009F918EA090F03D0864294BF521C5B1CC9
:10C88000401C8142EBD8002B18BF002A02D10020A7
:10C89000A064E064079810F0010F06D0206B20EA36
:10C8A0000C002063606BA8436063206B0099084212
:10C8B00003D1626B01990A4203D0216941F0100152
:10C8C000216110EA0A0F04BF606B10EA0B0F03D05E
:10C8D000206940F020002061A06B0099084203D13C
:10C8E000E26B01990A4203D0216941F040012161C4
:10C8F00010EA0A0F04BFE06B10EA0B0F03D02069A7
:10C9000040F080002061206C0099084203D1626CE5
:10C9100001990A4203D0216941F48071216110EA32
:10C920000A0F04BF606C10EA0B0F03D0206940F4BB
:10C9300000702061A06C002804BFE06C002803D0C8
:10C94000206940F48060206109B00120BDE8F08FCB
:10C950002DE9F04FBDB016460D460446F5F716F921
:10C96000F4F7D9FA01004FF011001DBF0290012029
:10C970000390012108BFCDE90210CDE93854F5F745
:10C980009DFB0022002D88BF04A904D9835C8B5431
:10C99000521C9542FAD8F5F793FB0021002C88BF72
:10C9A00004AA07D9435C02EB010C491C8CF8203027
:10C9B0008C42F7D8F5F7B4FA3190FE48007810F0C1
:10C9C000200F5DD0F4F7A7FAFB49FC4A00280CBF02
:10C9D000CDE90021CDE9001206F1EA003A902830B5
:10C9E0000025EA460DF1E8090DF1E00B3B9002A8A5
:10C9F0005BF8257050F82500F5F781FE0024002F24
:10CA000084BF04A800EB451818D918F9040026289B
:10CA100028BF00200BD2C10700EBD070890C40105A
:10CA200001EB80005AF825104058F5F76EFE59F8D2
:10CA3000251021F81400641CBC42E6D36D1C022DA5
:10CA4000D5D3DF4804781D2C1AD100210A4614AD35
:10CA50005BF822300020002B88BF59F822C007D98C
:10CA60003CF8107025F81170401C491C8342F7D81F
:10CA7000521C022AECD31D2C04BF2846FDF725FECC
:10CA8000CC4D287810F00C0F00F0DC82F4F743FA5C
:10CA9000CC49CD4A00280CBFCDE91421CDE91412B0
:10CAA000CA48F5F71EF90120F4F7B5FC2F900120D4
:10CAB000F4F701FD2D900120F4F7DCFF1D9002201A
:10CAC000F4F7D8FF1B900298F4F722FD2890039802
:10CAD000F4F71EFD17900120F4F7AFFD2E90112002
:10CAE000F4F7ABFD29900120F4F7E8FD2C9011201C
:10CAF000F4F7E4FD279024A8009022AB20AA1EA9F9
:10CB00000298F4F7FEFE25A8009023AB21AA1FA9E6
:10CB10000398F4F7F6FE0298F4F775FF2690029852
:10CB2000F4F771FFA24C01902068B0F8E4100120E6
:10CB3000F4F781FC00210120F4F784FF002102209A
:10CB4000F4F780FF206890F8E6100298F4F7F2FC02
:10CB5000206890F8E6100398F4F7ECFC002101201F
:10CB6000F4F784FD00211120F4F780FD002101205D
:10CB7000F4F7BDFD00211120F4F7B9FD2068B0F8ED
:10CB8000E8100298F4F7EDFE2068B0F8E81003987A
:10CB9000F4F7E7FE00210120F4F786FF2B9085488B
:10CBA000007810F0040F00F04A812068B0F8EC1013
:10CBB000009190F8EB3090F8EA200B210298F4F7FE
:10CBC00072FE2068B0F8EC10009190F8EB3090F80D
:10CBD000EA200B210398F4F766FE00210120F4F708
:10CBE00063FF32A801F08AF83699002238AD0020A0
:10CBF00055F822C0BCF1000F0ED902EB420303EB43
:10CC0000021306EB031331F8027B03EB4008401CD0
:10CC1000A8F85E718445F6D8521C022AE7D3029820
:10CC2000F3F7A5FE1C900398F3F7A1FE1A900021DC
:10CC30000298F4F7F0FC189001210298F4F7EBFC4D
:10CC4000169000210398F4F7E6FC2A90012103983E
:10CC5000F4F7E1FC564C19902068B0F8EE10009102
:10CC600090F8EB3090F8EA200B210298F4F71BFEC5
:10CC70002068B0F8EE10009190F8EB3090F8EA20C0
:10CC80000B210398F4F70FFE00240DF1080B00218F
:10CC90000120F4F709FF00210298F3F750FE00216C
:10CCA0000398F3F74CFE5BF824000121F3F747FEED
:10CCB00038A8002550F8249014A8B9F1000F50F8B6
:10CCC000240030904BD904A800EB4410009004EBF2
:10CCD000440000EB041006EB001A009800221146F5
:10CCE00010F905801046F4F7EDFEB8F1200F06DBD1
:10CCF0000027A8F12001012000FA01F804E001203A
:10CD000000FA08F74FF000085BF824003A460021CB
:10CD1000F4F76FFC5BF8240042460121F4F769FC4C
:10CD20006FEA0802F9430920F4F7CCFE32AFF5F7B9
:10CD300044F9FCF7E7FF012806D03846F5F740FB39
:10CD400000287DD0F5F799FBF4F720FF3098008894
:10CD50000AEB45016D1CA1F8AA014D45BDD3002287
:10CD600011461046F4F7AEFE641C022C8FD31C99BA
:10CD70000298F3F7E4FD1A990398F3F7E0FD002118
:10CD8000189A0298F4F735FC0121169A0298F4F7E4
:10CD900030FC00212A9A0398F4F72BFC0121199A00
:10CDA0000398F4F726FC024C2068B0F8F0100FE06E
:10CDB000648600106C860010B09D0030189D003015
:10CDC00082850010CC0E0030CC09003001000E002E
:10CDD000009190F8EB3090F8EA200B210298F4F7DC
:10CDE00062FD2068B0F8F010009190F8EB3090F8F8
:10CDF000EA200B210398F4F756FD01210846F4F7C9
:10CE000053FE32A800F07AFF3699002238AC002099
:10CE100054F822C0BCF1000F0ED902EB420303EB21
:10CE2000021306EB031331F8025B03EB4007401CCF
:10CE3000A7F8F6518445F6D8521C022AE7D300E041
:10CE40004BE0FE48007810F0080F7DD0FC4D2868BC
:10CE5000B0F8F210009190F8EB3090F8EA200B2136
:10CE60000298F4F720FD2868B0F8F210009190F8CD
:10CE7000EB3090F8EA200B210398F4F714FD002121
:10CE80000C460DF1E00C00205CF82120002A0CD9A2
:10CE900001EB410303EB011306EB031303EB400724
:10CEA000401CA7F842428242F8D8491C0229EAD322
:10CEB0002868002490F82401B4EB400F7EDA28683B
:10CEC00090F82401A042D4BF012100210120F4F7F1
:10CED000EBFD32AFF5F771F802E0F8F7B5FC28E7A3
:10CEE000FCF710FF012805D03846F5F769FA60B362
:10CEF000F5F7C3FAF4F74AFE36994FF000090DF141
:10CF0000E00E00225EF829701046002F05D931F995
:10CF10001030401C1A448742F9D8B2FBF7F2781E51
:10CF20003ED009EB490303EB091306EB031A31F971
:10CF3000103001EB400C3CF9028CB3EB080348BF06
:10CF40005B4231F9108001E038E01EE0B8EB0208E6
:10CF500031F910804CBFA2EB0808A8EB02083CF99D
:10CF600002BC3CF902CCBBEB020B4CBFA2EB0C0C9D
:10CF7000ACEB020CE0450AEB400C09DDBCF9428247
:10CF80004345C8BFACF8423208E0F8F75DFCA7E7BC
:10CF9000BCF940829845B8BFACF84032401EC6D1BB
:10CFA00009F1010901EB4701B9F1020FA9D3286882
:10CFB000641C90F82401B4EB400F80DB01202F9912
:10CFC000F4F739FA01202D99F4F780FA01201D9920
:10CFD000F4F738FD02201B99F4F734FD28990298E4
:10CFE000F4F7A8FA17990398F4F7A4FA01202E99F8
:10CFF000F4F73CFB11202999F4F738FB01202C9918
:10D00000F4F775FB11202799F4F771FB2498009031
:10D01000229B209A1E990298F4F745FC25980090CF
:10D02000239B219A1F990398F4F73DFC26990298B7
:10D03000F4F797FC01990398F4F793FC01202B99DE
:10D04000F4F732FD3198F4F74CFE3DB0BDE8F08FB7
:10D050002DE9F04FABB091460D460446F4F796FD2E
:10D060000222209212222192CDE90C45F4F758FFBA
:10D07000199072484FF00107007810F0210F6BD023
:10D0800070480E9070480F9000212098F4F7C3FA72
:10D09000089001212098F4F7BEFA09900021219808
:10D0A000F4F7B9FA0A9001212198F4F7B4FA0025AF
:10D0B0000B900CA850F825B020A850F82500F5F7E3
:10D0C0001EFB002408A8264609EB051A00EBC5083C
:10D0D00019E0600904F01F0158F8200007FA01F177
:10D0E00008420FD0E007800C610800EB81010EA818
:10D0F00050F825004058F5F708FB0AEB4601761C6E
:10D10000A1F8BE03641C5E4538BF262CE1D36D1C1C
:10D11000022DCED34D4805781D2D1DD100210A4684
:10D120006C460CAE002056F82230002B88BF09EB6D
:10D13000021C09D90CEB4008401CB8F8BE8324F847
:10D140001180491C8342F5D8521C022AEAD31D2DB6
:10D1500004BF2046FDF7D8FB3848007810F0040FD4
:10D1600000F0D3813A4816903A4817900220F4F71D
:10D1700052F927900220F4F79EF925900120F4F748
:10D1800079FC24900220F4F775FC1B902098F4F7AA
:10D19000BFF91A902198F4F7BBF918900220F4F720
:10D1A0004CFA28901220F4F748FA1F900220F4F766
:10D1B00085FA26901220F4F781FA1D900EA80090AF
:10D1C00006AB04AA02A92098F4F79BFB0FA80090D5
:10D1D00007AB05AA03A92198F4F793FB2098F4F76D
:10D1E00012FC22902198F4F70EFC154D019028684E
:10D1F000B0F8E4100220F4F71EF900210120F4F742
:10D2000021FC00210220F4F71DFC286890F8E610AC
:10D210002098F4F78FF9286890F8E6102198F4F731
:10D2200089F900210220F4F721FA00211220F4F7F5
:10D230001DFA00210220F4F75AFA0DE06C86001066
:10D2400064860010489E0030E09E00308785001004
:10D250004C1800304C1D003000211220F4F747FA22
:10D260002868B0F8E8102098F4F77BFB2868B0F83D
:10D27000E8102198F4F775FB00210220F4F714FC64
:10D2800023902868B0F8EC10009190F8EB3090F8FB
:10D29000EA200B212098F4F706FB2868B0F8EC1080
:10D2A000009190F8EB3090F8EA200B212198F4F7E8
:10D2B000FAFA00210220F4F7F7FB10A800F01EFD97
:10D2C000159900220CAC002054F822C0BCF1000FCC
:10D2D00088BF09EB421308D931F8026B03EB400811
:10D2E000401CA8F8DE638445F6D8521C022AEAD313
:10D2F0002098F3F73CFB1E902198F3F738FB1C9025
:10D3000000212098F4F787F9089001212098F4F77C
:10D3100082F9099000212198F4F77DF90A90012102
:10D320002198F4F778F90B902868B0F8EE10009186
:10D3300090F8EB3090F8EA200B212098F4F7B3FA3C
:10D340002868B0F8EE10009190F8EB3090F8EA20E1
:10D350000B212198F4F7A7FA00250DF1800B00218D
:10D360000220F4F7A1FB00212098F3F7E8FA00214E
:10D370002198F3F7E4FA5BF825000121F3F7DFFACF
:10D380000CA8002450F825002A9016A8264650F82C
:10D390002500299008A800EBC50009EB451A00906C
:10D3A00046E0009861094FF0010850F8210004F0B0
:10D3B0001F0108FA01F1084239D000221146104637
:10D3C000F4F780FB202C23BF0027A4F1200008FAEB
:10D3D00000F808FA04F738BF4FF000085BF82500A2
:10D3E0003A460021F4F705F95BF825004246012191
:10D3F000F4F7FFF86FEA0802F9430920F4F762FB3B
:10D4000010AFF4F7DAFDFCF77DFC012806D03846B2
:10D41000F4F7D6FF00287DD0F5F72FF8F4F7B6FB28
:10D42000299800880AEB4601761CA1F8EE03641CDB
:10D430002A98864238BF262CB3D3002211461046C4
:10D44000F4F740FB6D1C022D89D31E992098F3F749
:10D4500076FA1C992198F3F772FA0021089A20981D
:10D46000F4F7C7F80121099A2098F4F7C2F80021CF
:10D470000A9A2198F4F7BDF801210B9A2198F4F744
:10D48000B8F802202799F3F7D6FF02202599F4F780
:10D490001DF801202499F4F7D5FA02201B99F4F71E
:10D4A000D1FA1A992098F4F745F818992198F4F7C9
:10D4B00041F802202899F4F7D9F812201F99F4F7BF
:10D4C000D5F802202699F4F712F912201D99F4F7E5
:10D4D0000EF90E980090069B049A02992098F4F792
:10D4E000E2F90F980090079B059A03992198F4F7A9
:10D4F000DAF922992098F4F734FA01992198F4F78F
:10D5000030FA02202399F4F7CFFA1998F4F7E9FBDF
:10D510002BB000E001E0BDE8F08FF8F795F972E775
:10D520002DE9F04FFF4DADF2344DFF224FF48461F1
:10D5300068466C680FF09DFB0094288810F4804FBB
:10D540001CBF2046FEF7B3FC6A46009890F82030D6
:10D5500090F821C050300CFB03F100EB410000219A
:10D56000BCF1000F08D902EB410730F8026B491CEF
:10D57000A7F8EA608C45F6D80021002B08D902EB09
:10D58000410730F8026B491CA7F812618B42F6D8AC
:10D590001668002196F82260002E0BD902EB410795
:10D5A00030F8026BA7F8BE631668491C96F8226033
:10D5B0008E42F3D81668002196F82360002E0BD90E
:10D5C00002EB410730F8026BA7F8CE631668491CDE
:10D5D00096F823608E42F3D80021BCF1000F08D9E1
:10D5E00002EB410730F8026B491CA7F870608C45CC
:10D5F000F6D80021002B08D902EB410730F8026B66
:10D60000491CA7F898608B42F6D830F8021BA2F8A4
:10D61000E61030F8021BA2F8E81030F8021BA2F85E
:10D62000E41000260021BCF1000F0ED906EB4607DE
:10D6300007EB061702EB870707EB410930F8028B6F
:10D64000491CA9F85E816145F6D30021002B0ED953
:10D6500006EB460707EB061702EB870707EB4109C6
:10D6600030F8028B491CA9F88E829942F6D3761CB9
:10D67000042ED7D300261768002197F82270002FB8
:10D6800088BF02EB06170CD907EB410930F8028B73
:10D69000A9F8DE83D2F80080491C98F822808845DA
:10D6A000F2D81768002197F82370002F88BF02EB8B
:10D6B00006170CD907EB410930F8028BA9F8FE8355
:10D6C000D2F80080491C98F823808845F2D8761C4F
:10D6D000022ED0D361461846FEF71CFD9148012664
:10D6E000056815F4004F7CD180468F486F460026B0
:10D6F000006890F8B40000F00F0900F016FE012851
:10D7000009D00F214846F8F7A2F9012812D00020CD
:10D7100000F008FEB4E000210846F4F705FBF3F73B
:10D72000E0FB50B18148D0F8401341F48031C0F89B
:10D73000401302E0012000F0F5FD7D4890F80090D4
:10D740007C4890F800A0BAF1000F18BFB9F1000FA3
:10D750007DD0009E002086F8209086F821A086F8D3
:10D76000220086F82300F5F709F8F4F7D9FB834681
:10D77000002015F0030F18BF4FF4817015F0200F33
:10D780001CBF40F20121084315F0100F1EBF98F88E
:10D79000001011F0210F40F4846060B10BEA00002A
:10D7A000F4F79FFAFF210F20F8F7BDFBF4F7EEF92D
:10D7B0005846F4F796FA15F0100F09D05E493A462C
:10D7C000087886F82200497886F82310FFF740FC95
:10D7D00015F02C0F04D03A4651464846FFF7B8F8EA
:10D7E00000E04DE015F0030F47D0CDF82474009809
:10D7F000CDF8200400F15006F4F762FC8346F4F7FC
:10D80000C5F90020F4F77BFF0027BAF1000F25D9F6
:10D8100007EB4700002500EB071816E01BF9050091
:10D82000262811D2C107890C00EBD07001EB8801CA
:10D83000401001EB800000F1405000F5004000680E
:10D84000F4F763FF26F8020B6D1C4D4500E015E070
:10D8500038BF262DE2D37F1C5745D9D337480078EF
:10D860001D2804D1DDF820045030FCF720FE51467D
:10D870004846DDF82424FEF74DFC0126F4F711FBA1
:10D8800094F82000CDF8280494F82100CDF82C0459
:10D89000002E1FBFDDF828040028DDF82C04002826
:10D8A00004BF0DF2344DBDE8F08F1E480068CDF87E
:10D8B000300410F0020F00F02081009DDDF82C7480
:10D8C000DDF8282428696E4620F00F00286147F60D
:10D8D000FF706FEA0009CDF82004002005F1500820
:10D8E00004900390029082460190002F61D90AFBB8
:10D8F00002F04FF0010C38F9101000208B465B4607
:10D90000CDF82404012A2BD90AFB02C038F91000F3
:10D910009842C8BF03468842B8BF0146B0EB0B0E21
:10D920000EE000006C86001064860010005000407D
:10D93000FE840010FF840010068500107D85001015
:10D9400048BFABEB000E0FFA8EFBDDF824E4F34585
:10D95000C8BFCDF824B483460CF1010C9445D3D351
:10D960004B45C8BF9946DDF820048142B8BFCDF8C9
:10D970002014581A48BFC81A01B2FE480068B0F90E
:10D98000C0308B4205DBB0F9C210DDF824048842B8
:10D990000BDD4FEA5A1006EB80000AF01F0C012144
:10D9A000C36801FA0CF11943C1600AF1010ABA45D2
:10D9B0009DD34FF0000A002A4FD938F91A000021F0
:10D9C00083465B464FF0010CCDF82414012F1BD980
:10D9D0000CFB02A138F911109942C8BF0B468142D5
:10D9E000B8BF0846B1EB0B0E48BFABEB010E0FFA08
:10D9F0008EFBDDF824E4F345C8BFCDF824B48B4694
:10DA00000CF1010CBC45E3D34B45C8BF9946DDF88A
:10DA100020148842B8BFCDF82004191A48BFC11A93
:10DA200009B2D4480068B0F9BC308B4205DBB0F9CC
:10DA3000BE10DDF8240488420BDD4FEA5A1006EBD5
:10DA400080000AF01F0C0121436801FA0CF1194310
:10DA500041600AF1010A9245AFD3F068002804BF83
:10DA60003069002803D0286940F0080028617068F8
:10DA7000002804BFB068002803D0286940F00400E3
:10DA800028617168F068B9400843A862B1683069DC
:10DA9000B9400143E9627068202F39BFC7F1200205
:10DAA000D040A7F1200290400843E862DDF820044E
:10DAB000A884A5F82690B6F9E410B9EB010048BF98
:10DAC000A1EB0900AB490968B1F9B820904203DD28
:10DAD000286940F002002861B6F9E420DDF820044E
:10DAE000101A44BFDDF82004801AB1F9BA10884238
:10DAF00003DD286940F001002861DDF830049E4D07
:10DB000010F0050F06D06A46DDF82C14DDF8280465
:10DB1000FEF741FCD5F8009019F0080F7ED0009A6E
:10DB2000DDF82C34DDF828A411694FF0000B21F446
:10DB3000C05111616846CDF860B05946CDF85CB06F
:10DB4000002B84BFDFF82CE201261AD9DEF8007022
:10DB500000EB410CBCF942C2B7F9267167450DDAFA
:10DB60004FEA511C00EB8C0C01F01F08DCF85C70D4
:10DB700006FA08F847EA0807CCF85C70491C994295
:10DB8000E4D3C0F858B00021C0F854B0BAF1000F87
:10DB900084BF784E01271AD9D6F8008000EB410CDB
:10DBA000BCF972C3B8F92681E0450DDA4FEA511885
:10DBB00000EB880C01F01F0BDCF8548007FA0BFB1C
:10DBC00048EA0B08CCF85480491C5145E4D3916BCA
:10DBD000D0F85CC041EA0C01D0F854C00CFA03FC48
:10DBE00041EA0C019163D16BD0F860C041EA0C01AD
:10DBF000D0F858C00CFA03FC41EA0C0CC2F83CC047
:10DC0000416D202B39BFC3F12003D940203B9940FF
:10DC100041EA0C01D163416D002900E011E004BF2D
:10DC2000816D002903D0116941F400611161C16D5A
:10DC3000002904BF006E002803D0106940F4805012
:10DC4000106119F0100F18BF19F0050F06D094F8E5
:10DC5000231094F822006A4600F080F9287810F02A
:10DC6000400F0FD16069401C60612069002814BF1B
:10DC7000E069A06900F1010014BFE061A06168469D
:10DC8000FEF779F90020E060A36821460246A44629
:10DC9000B3F5056F88BF4FF405630020B0EB930F19
:10DCA00006D25CF82070401C3A44B0EB930FF8D3D6
:10DCB0005042C860287810F0800F05D14FF44030F2
:10DCC0004FF40562F5F7C2F841208DF82004207C5E
:10DCD0008DF82104607C8DF82204A07C8DF823044B
:10DCE000E07C8DF82404002305220DF584610720D3
:10DCF00000F08AFA0DF2344DBDE8F08F70B505469C
:10DD00000024F4F75AF9FBF7FDFF012806D0284656
:10DD1000F4F756FB30B1F4F7B0FB0124F3F736FF0C
:10DD2000204670BDF7F790FDEDE72DE9F74F84B081
:10DD30004FF00008C2F82080C2F81C80059B0D4EF1
:10DD400001274146002B23D902EB4103B3F9703080
:10DD5000002BB8BF5B421BB2D6F800C0BCF9CCC0E8
:10DD60009C4511DD4B0901F01F0402EB830307FA08
:10DD700004F403E0648600106C860010D3F81CC025
:10DD80004CEA040CC3F81CC0059B491C9942DBD328
:10DD90000021012B1CBF059BA3F1010940D002EB20
:10DDA0004103B3F97240B3F970C0B4EB0C0348BF40
:10DDB000ACEB04031BB23568B5F9C6509D422CDAB2
:10DDC000B2F9E630BCEB030548BFA3EB0C052DB25E
:10DDD000B4EB030C48BFA3EB040C0FFA8CF39D4289
:10DDE0000DDB4B0902EB830301F01F04D3F81CC0C9
:10DDF00007FA04F44CEA040CC3F81CC00DE04B1CF9
:10DE00004FEA531C02EB8C0C03F01F03DCF81C40A0
:10DE100007FA03F32343CCF81C30491C4945BED311
:10DE2000316891F8CA30002B7DD091F8CB1014687E
:10DE30008B4288BF19460023DDF814C0BCF1000FE7
:10DE400084BF491C00916ED94FF0010EDDF800C06F
:10DE50004FF000090121CA46BCF1010F52D9DFF889
:10DE60002CC303FB0005DCF800C0CDF80CC0BCF9E6
:10DE7000CEC002950EFB0005019503FB001504EBD7
:10DE80004505B5F95080B8F1000FB4BFC8F10005E1
:10DE90004546AC4536DB0EFB001504EB4505B5F9F0
:10DEA0005070002FB4BF7D423D46AC452ADB029D39
:10DEB0006D1A04EB4505B5F94E60002EB4BF7542EE
:10DEC0003546AC451EDB019D6D1A04EB4505B5F9E1
:10DED0004E50002DB4BFC5F1000BAB46E34511DC3D
:10DEE000A7EB0808039FB7F9C8704745B8BF09F109
:10DEF0000109AD1BBD42C8BF0AF1010A491C009DC2
:10DF0000A942BAD3BAEB090148BFA9EB0A01DFF86D
:10DF10007CC2DCF800C09CF8CAC061450FDB59091F
:10DF200002EB810100E015E003F01F064FF0010C49
:10DF3000CD690CFA06FC45EA0C0CC1F81CC0059929
:10DF40005B1C8B4206D2002B18BFA3F1010E7FF49D
:10DF50007DAF79E707B00120BDE8F08F2DE9F04FE4
:10DF600083B04FF0000C1368C2F864C0C2F868C0F8
:10DF7000C2F86CC0DFF818C24FF0010BDCF800E00B
:10DF8000DFF808C21EF0010FDCF800C029D01C69C0
:10DF9000002524F480341C612F46CDE900015DF892
:10DFA00027A00024BAF1000F88BF02EB071915D98A
:10DFB00009EB4406BCF9D480B6F9BE63B04503DC76
:10DFC000BCF9D680B04505DA566E0BFA05F846EA7C
:10DFD00008065666641C6D1CA245E9D87F1C022FFA
:10DFE000DDD31EF0040F71D01C69002524F4C02479
:10DFF0001C612F46EE46CDE900015EF827A0002403
:10E00000BAF1000F88BF02EB471915D909EB440696
:10E01000BCF9D880B6F9DE63B04503DCBCF9DA8020
:10E02000B04505DA966E0BFA05F846EA08069666DC
:10E03000641C6D1CA245E9D87F1C022FDDD300258E
:10E040002F46CDE900015EF827A00024BAF1000FA9
:10E0500088BF02EB471915D909EB4406BCF9DC80EF
:10E06000B6F9EE63B04503DCBCF9DE80B04505DAF5
:10E07000D66E0BFA05F846EA0806D666641C6D1CD7
:10E08000A245E9D87F1C022FDDD34418D2E91A50EB
:10E0900030EA050C4CEA0506C2F86CC013D000212A
:10E0A0000846002C0FD90BFA00F71CEA070F18BF1F
:10E0B000491C401CA042F6D3012904D145EA0C00BA
:10E0C00090660020D066506EB043506693F82000F2
:10E0D00093F821100844516ED9B1196941F4803187
:10E0E0001961D2F864C0196B0CFA00FC41EA0C010A
:10E0F0001963516E202827BFA0F1200C01FA0CF102
:10E10000C0F1200C21FA0CF1D3F834C041EA0C0123
:10E110005963916ED9B1196941F400311961D2F88E
:10E1200068C0996B0CFA00FC41EA0C019963916E8E
:10E13000202827BFA0F1200C01FA0CF1C0F1200C1F
:10E1400021FA0CF1D3F83CC041EA0C01D963D16E3D
:10E15000C1B1196941F480211961D2F86CC0196C00
:10E160000CFA00FC41EA0C011964D16E202827BF8B
:10E17000203801FA00F0C0F1200021FA00F0596CBB
:10E180000843586403B00120BDE8F08F6486001096
:10E190006C86001070474FF0FF3070475D48406854
:10E1A00070475C494860704710B582B007280BD1B2
:10E1B0004FEA111C012404FA0CFC564C64681CEA5A
:10E1C000040F04BF02B010BD9B0100F00F0043EA32
:10E1D000800040F001008DF800008DF801108DF8EE
:10E1E0000220100A8DF80300100C8DF80400100EA8
:10E1F0008DF8050000208DF806008DF807006846B0
:10E200000EF0C3FD02B010BD10B582B007280DD1CD
:10E2100091F800C001244FEA1C1C04FA0CFC3D4C90
:10E2200064681CEA040F04BF02B010BD9B0100F03B
:10E230000F0043EA800040F001008DF80000072A3B
:10E2400088BF072200206B46002A09D911F800C0B8
:10E250001C18401C84F801C09042F7D3072805D24F
:10E2600000211A18401C51700728FAD318460EF0E6
:10E270008CFD02B010BD10B59B0100F00F0082B004
:10E2800043EA800040F002008DF80000072A88BFB2
:10E29000072200206B46002A09D911F800C01C187B
:10E2A000401C84F801C09042F7D3072805D2002112
:10E2B0001A18401C51700728FAD318460EF065FD55
:10E2C00002B010BD70B5134E40EA01250228348813
:10E2D000224618BF052803D1002918BF022900D102
:10E2E0002C46A24209D051B17088002344EA004272
:10E2F00090210720FFF758FF3480758070BDF5F737
:10E300009EF944EA0042002390210720FFF74CFFCA
:10E31000F2E7000074860010FD4908707047FC4861
:10E3200000787047FA4948707047F948407870475C
:10E330002DE9F04FF748F64DADF6641D0068697899
:10E34000836D0229C3F303201AD06A6812F4007F98
:10E350001EBFC3F303310F29084612F0800F1EBF02
:10E36000C3F303110F29084602F00701F7F76FFB0B
:10E37000012814BF00200220687040F06F830DE078
:10E3800000210846F3F7D0FCF2F7ABFD30B1E248CC
:10E39000D0F8401341F48031C0F84013F3F7C0FDCA
:10E3A000CDF81C09287910F0100F18BFF4F7C5F943
:10E3B000287910F0080F03D1FF210F20F7F7B3FDE4
:10E3C000D6480078CDF83C09D5480078CDF840090A
:10E3D000D4480478D4480078CDF83809D34890F868
:10E3E000009090F80180DDF8400900281CBFDDF89E
:10E3F0003C09002816D00EF0A5FC0EF0A8FC002069
:10E40000F6F7C9FA0020F6F725FB0020F6F73FFBE8
:10E41000BF48007910F0100F0CD00120F6F796FBE2
:10E4200001200BE0DDF83809002818BF002CE2D1EC
:10E4300000F014BB0020F6F789FB0020F6F786FBFE
:10E44000F2F74FFD10F0010F04BF0120F2F7D4FFE7
:10E45000F3F77AFD1E20FBF782FF00210846FBF749
:10E46000F9FECDF84C0901210020FBF7F3FEDDF8A1
:10E470004029DDF83C198346002001FB02FABAF17D
:10E48000000F84BF47F6FF73DA4308D9DDF84C1953
:10E4900021F810202BF81030401C8245F6D81E20A1
:10E4A000FCF7F9F800210120FBF7D4FE0646012114
:10E4B0000846FBF7CFFE0546DDF83819002067183F
:10E4C0001CBF47F6FF72D14306D026F8101025F87E
:10E4D0001020401C8742F8D81E20FCF7FFF90021CD
:10E4E0000220FBF7B7FECDF8480901210220FBF717
:10E4F000B1FECDF84409002019EB08091CBF47F60E
:10E50000FF73D9430AD0DDF8482922F81010DDF84E
:10E51000442922F81030401C8145F4D87C484FF043
:10E5200000084088002840F2A181DDF83819781CE5
:10E53000491ECDF85C19DDF8381940082144491E00
:10E54000CDF8501909F101014908CDF85819CDF855
:10E550005409FBF7D7FB012800F088810DF5126004
:10E56000F3F72EFF002800F07A81DDF82409F5F793
:10E570002EFCDDF82809002853D00EF08EFB04464F
:10E580006348007910F0100F0AD02046DDF82819F2
:10E590000EF000FC0190A04208BFDDF8284910E011
:10E5A000002000230090019002901A461946DDF8E1
:10E5B00028090EF0F4FB01905548007910F0200F67
:10E5C0000BD1F5F779FCDDF8402900920146204691
:10E5D000DDF83C39019A0EF0E7FB4D48808810F4D5
:10E5E000804F1EBF01980028F5F7A8FC002C1CBF27
:10E5F0000020BAF1000F14D9DDF84C2934F91010BD
:10E6000032F910208A42BCBFDDF84C2922F81010E4
:10E610003BF910208A42C8BF2BF81010401C8245DD
:10E62000EAD8DDF81C0910F0010F1CBFDDF8300935
:10E6300000286CD00EF02CFB04463548007910F011
:10E64000400F07D000231A461946DDF830090EF0B6
:10E65000B0FB0DE0F5F7F9FB0222009201462046DF
:10E66000DDF85439DDF830290EF09EFBDDF8300975
:10E670002749898811F4005F1CBF0028F5F7EFFBDC
:10E68000002C44D02248426812F4806F33D0DDF869
:10E6900038190020012911D004EB400134F910C0D1
:10E6A000B1F90230B3EB0C0148BFACEB030124F825
:10E6B0001010DDF85C19401C8842EDD34FF0000EBD
:10E6C00024F810E0DDF85019401C884211D204EB08
:10E6D000400134F910C0B1F90230B3EB0C0148BF6E
:10E6E000ACEB030124F81010DDF85019401C8142F6
:10E6F000EDD824F810E00020002F22D934F91010B2
:10E7000036F910308B42B8BF26F8101010E04EE0FA
:10E710007C8600106486001000500040FE840010CB
:10E72000FF8400100385001004850010068500108A
:10E7300035F910308B42C8BF25F81010401C8742B5
:10E74000DCD812F4806F32D0F54A08F10100A2FB48
:10E7500000318908494201EB8101C14227D1A2FB66
:10E7600008108008A2FB00210909494201EB810140
:10E7700000EB810000EB4001C1EB401103A800EB6E
:10E7800081010020002F84BF47F6FF7C6FEA0C0256
:10E790000DD936F8103035F810401B1B21F8103019
:10E7A00026F8102025F810C0401C8742F1D8DDF86B
:10E7B0001C0910F0200F1CBFDDF83409002849D0D7
:10E7C0000EF0FCFA0446D748808810F4807F13D0FE
:10E7D000F5F721FB0146022000902046DDF858396C
:10E7E000DDF834290EF0E0FADDF83409CD498988E6
:10E7F00011F4805F0FD109E00021DDF834090EF03B
:10E8000033FAB8F1040F38BF0024EFE718B1F5F779
:10E8100004FBF5F7FBFA002C1CBF0020B9F1000F38
:10E8200018D9DDF8482934F9101032F910208A423D
:10E83000BCBFDDF8482922F81010DDF8442932F970
:10E8400010208A42C4BFDDF8442922F81010401C71
:10E850008145E6D8F3F711FE08F1010801E0F6F76B
:10E86000F3FFB04840888045FFF473AEF3F78EF9AC
:10E870000EF06DFA0EF070FAAA4C6088804578D3DD
:10E88000DDF81C0910F0020F2AD000224FF6FF73AA
:10E890001046BAF1000F10D9DDF84C193BF910C041
:10E8A00031F91010A1EB0C019142C8BF0A46994200
:10E8B000B8BF0B46401C8245EED842208DF80000C0
:10E8C000100A8DF801008DF80220180A8DF8030057
:10E8D0008DF804300023052269460720FFF794FCD9
:10E8E000DDF81C0910F0010F7DD0A08810F4806FB6
:10E8F00051D08B48A0FB08108308142B88BF142329
:10E900004FF0000844464146002F84BF981E0090F7
:10E9100055D94FF0000CDFF810A247F6FF7B624696
:10E92000002B12D902EB4200C0EB421E03A800EB01
:10E930008E0030F9110084445045C8BF82465845C6
:10E94000B8BF8346521C9A42ECD3002B04BF002070
:10E9500026F811000ED09CFBF3F026F81100022BD4
:10E9600008D9ACEB0A00A0EB0B02009892FBF0F088
:10E9700001E06AE0002025F8110036F91100A042FC
:10E98000C8BF044635F911004045C8BF8046491C40
:10E990008F42BED813E000244FF6FF782046002FA8
:10E9A0000DD936F9101035F91020891AA142C8BFC7
:10E9B0000C464145B8BF8846401C8742F1D84320E9
:10E9C0008DF80000200A8DF801008DF802404FEA12
:10E9D00018208DF803008DF8048000230522694675
:10E9E0000720FFF711FCDDF81C0910F0200F2CD0D8
:10E9F00000224FF6FF731046B9F1000F12D9DDF86F
:10EA0000481931F910C0DDF8441931F91010ACEB98
:10EA100001019142C8BF0A469942B8BF0B46401C4B
:10EA20008145ECD844208DF80000100A8DF80100D3
:10EA30008DF80220180A8DF803008DF804300023A9
:10EA4000052269460720FFF7DFFBFF20FBF787FC65
:10EA5000FF20FBF720FEFF20FBF740FFF3F721FA32
:10EA60000DF6641DBDE8F08F30B5ADF6540D4FF0D6
:10EA7000FF30FCF7A8FF2B4C00206070F3F718FB69
:10EA8000F3F7EBFA05460020F3F7E1FAFF224FF423
:10EA9000056168460EF0EDF86846FDF720FA684615
:10EAA000FDF7ABF9FBF72EF9012803D1F6F774FE59
:10EAB00003281BD1207810F0010F07D0FEF730FD9E
:10EAC000207820F001002070FBF7A6F8207810F0E5
:10EAD000020F07D0FFF72CFC207820F002002070F6
:10EAE000FBF79AF8F6F758FE03280BD00020FDF745
:10EAF00084F92846F3F7ABFA0120F3F7D9FA0DF6BB
:10EB0000540D30BDF6F7A0FECCE706494860002062
:10EB10004870704703484068704702494880704712
:10EB2000CDCCCCCC7C8600100080FFFFFE49087065
:10EB30007047FD4800787047FB49C8717047FA4834
:10EB4000C0797047F848407A7047F748C17911F0AA
:10EB5000010F18BF704710B5002141720846F6F743
:10EB6000F5FEBDE810400020F5F76EBFEE48008CC2
:10EB7000C0F300207047EC4910B5098C0020C1F3A8
:10EB8000002151B106F023FF64280FBF4FF0C040B1
:10EB9000012101FA00F040F08040BDE8104006F08D
:10EBA00019BFE14A10B5C0F3074381B29361116206
:10EBB000C0F30360507090700020C1F30021D06159
:10EBC00051B106F004FF64280FBF4FF0C04001218F
:10EBD00001FA00F040F08040BDE8104006F0FABEB7
:10EBE000D14840797047D04A0028116A14BF41F0DB
:10EBF000020021F0020010627047CB4890F820001C
:10EC0000C0F340007047C84A10F0010F106A14BFEB
:10EC100040F0020020F0020010627047C24900205C
:10EC200091F82010C1F34001002918BF012070475E
:10EC30000028BD4A116A14BF41F0010021F0010013
:10EC400010627047B84890F8200000F0010070474B
:10EC5000B5494A788A7048707047B3484078704721
:10EC6000B14880787047B1480068406DC0F30360D8
:10EC7000704701218140AC48826911408161704731
:10EC800001218140A848826922EA0101816170471F
:10EC9000A54880697047A448C0697047A24910B56B
:10ECA000CC69C8610246002381210720FFF77CFA66
:10ECB000204610BD9C48008CC0F3802070479A48C5
:10ECC00080797047984890F82000C0F38000704722
:10ECD000954890F82000C0F3C00070479248008C1F
:10ECE000C0F340207047904890F82000C0F3C01057
:10ECF0007047FCF775BB8C48008CC0F34030704700
:10ED00008948008CC0F3C02070478748008CC0F34E
:10ED100000307047844A10F0805F116A14BF41F4DC
:10ED2000806121F4806110F0005F14BF41F4005055
:10ED300021F400501062FCF738BD7B48016A0020C6
:10ED400011F4806F18BF4FF0805011F4005F18BFAE
:10ED500040F00050704770B57349044610F0040F3E
:10ED60000E6A304614BF40F4807020F4807014F0B6
:10ED7000080F14BF40F4007020F4007014F0100F5E
:10ED800014BF40F4006020F4006014F0400F14BF82
:10ED900040F4805020F4805014F0200F14BF40F055
:10EDA000800020F0800008620021C0F3002050B1F4
:10EDB00006F00DFE64280FBF4FF0C041012101FA9B
:10EDC00000F040F08041084606F004FEC4F38000E5
:10EDD000C6F30021884227D006F094FD05460120A5
:10EDE000F5F707FD15F4817F0CBF01200020F3F734
:10EDF0002EF915F0020F04D0022009F0A1FE002028
:10EE000009E015F4807018BF012009F099FE484808
:10EE100090F86C00C00803F0FBF815F4C06F03D045
:10EE200006F09FF906F08DF9C4F3C000C6F3402147
:10EE3000884208BF70BD0120BDE87040F5F7D9BC1D
:10EE40003948016A002011F0040F18BF012011F0A9
:10EE5000080F18BF40F0020011F4807F18BF40F087
:10EE6000040011F4007F18BF40F0080011F4006F97
:10EE700018BF40F0100011F4805F18BF40F0400050
:10EE800011F0800F18BF40F02000704703283CBFEE
:10EE90002549486170472448007D70472249C8735E
:10EEA00070472148C07B70471F48C06A70471E49A1
:10EEB0004A6A10434862704770B51B4E706A40F052
:10EEC000007400207062356A15F0040F18BF44F01A
:10EED000010415F0080F18BF44F0020415F4807FF8
:10EEE00018BF44F0040415F4007F18BF44F0080470
:10EEF000FCF776FA002818BF44F0805415F4006F30
:10EF000018BF44F0100415F0800F18BF44F020041F
:10EF100015F4805F18BF44F0400415F4005F18BF7B
:10EF200044F00054F16905E0848600106486001006
:10EF30001011011044EA0140002918BF40F0806020
:10EF400070BDFE4988627047FC4890F8280000F0C8
:10EF500001007047F94890F82800C0F3400070475E
:10EF6000F64890F82800C0F380007047002818BFCA
:10EF70000120F249087370472DE9F05FF0498000E5
:10EF800000260968896D21FA00F000F00F04C1F332
:10EF90000325C1F3031AC1F30339C1F30358C1F3C5
:10EFA000036BAC421CBF2046BDE8F09FE348B8F1BC
:10EFB0000F0FC76C16D006F0A5FC10F4817F0ED0A1
:10EFC000BBF10F0F0AD0DD48008CC0F3403028B1F0
:10EFD00006F008FD082818BF5C4600D14446A74249
:10EFE00018BF0126AC420FD1B9F10F0F0CD0D34896
:10EFF000008CC0F3403020B106F0F4FC082818BFA4
:10F000004C46A74218BF0126AC4207D1BAF10F0FF8
:10F0100004D0F6F7AEFC002818BF5446A7421EBF26
:10F02000002E0020F5F7E5FBC448C4642046BDE887
:10F03000F09F2DE9F047002586B02E46F6F7ACFB91
:10F04000BF49052808680CBF90F8F80090F85800F0
:10F0500000F00F094846FCF793FCB84F4FF0000A48
:10F060004FF00108002808BF54460FD0446A06F04C
:10F0700049FC10F4C06F08BF87F80BA006D014F04D
:10F08000020F18BF24F0010487F80B8014F0010F61
:10F0900014BF0224042444F400314846F6F7D7FC98
:10F0A000002804BF06B0BDE8F08714F0040FA54C9B
:10F0B00007D0F1F73EFC01462078814288BFF1F786
:10F0C00030FC0120F2F798F9F2F777FFFAF71AFE11
:10F0D000012832D06846F3F773F950B36846FBF75E
:10F0E00016FD0198F4F773FE029880B196482178D6
:10F0F0000078400000FB01F2944802990DF09BFD5E
:10F1000093480078492804BF9048FBF7D0F9049849
:10F1100048B19048904900780978084442008F48E7
:10F1200004990DF088FD87F80C80F3F7A6F9012605
:10F1300003E0F6F789FB002DC8D0F2F727FDF6F7BC
:10F14000FFFD06B03046BDE8F0877C48007B002814
:10F1500018BF012070472DE9F04F4FF0000A87B02B
:10F1600005460F24D146F6F717FB0746F6F71AFBBC
:10F17000DFF8C8B10690052F07D1FBF7F1FE002894
:10F1800004BF00208BF80C0002D09BF80C0058B98B
:10F19000F6F750FC06464FF48050F6F748FCFFF7B0
:10F1A00048FF3046F6F743FC052F0CBFDFF8B0816F
:10F1B000DFF8B08106F0A6FB002818BF0E24214618
:10F1C0002846F6F744FC002804BF07B0BDE8F08FDE
:10F1D0000DF0B8FD0DF0BBFDF5F7B5FA04007DD1DB
:10F1E0000125F1F77EFE06460020F2F705F92846D4
:10F1F000F2F7C3FE5148C563F4F724FAA5F1010BF9
:10F20000FAF780FD01280AD0F6F7C6FAB84206D10F
:10F21000F6F7C8FA0699884208BF002C09D0F2F721
:10F22000B5FC464F16F0010F7D7834D0012C27D065
:10F2300031E06846F3F7C4F8F8B116F0010F03D0D7
:10F240000120F4F73FFC82466846FBF760FC01981A
:10F25000F4F7BDFD6846C0470446F3F70EF9002CED
:10F26000CED115B901985845CAD1F2F78DFC0028C6
:10F2700004BF2846F2F781FEC2E7F6F7DAFABFE7E5
:10F280000120F4F71FFC504505D2AAEB0001012034
:10F29000F4F728FC8146F4F7FAF916F0010F29D0AB
:10F2A000012C27D1B9F1000F24D0F1F7ECFF04466F
:10F2B000F1F728FE00EB800004EB400048440021F9
:10F2C00044F20902904284BFA0F580400938002D25
:10F2D00008BF43F6390105D0022D00E00AE008BF5F
:10F2E00041F6F901884205D2091A0120F4F729FCF8
:10F2F0000120B8720DF030FDF6F722FD07B0BDE831
:10F30000F08F2DE9F14F88B00027039705970697F6
:10F310000497F6F741FA01900B48B946CDF80890EA
:10F3200004780848C84623460578089804FB05FA7F
:10F33000009500EB4A060246044915E08486001059
:10F3400064860010FF840010FE84001080140110F9
:10F350007D8500100485001003850010701A0110CF
:10F36000293400109939001030460DF01DFDDFF8EA
:10F3700000B49BF80000492804BFFE48FBF797F84B
:10F38000FB4800784C2804BF3046FBF790F8DFF8C4
:10F39000E8B3019805282DD1B6F90000B6F902109E
:10F3A00006EB4402084436F91410B2F90220DBF8E7
:10F3B000603011440022012B11D1DBF858301B1AA8
:10F3C0009E46CBF85C30DBF85030BEF1230FA1EB4A
:10F3D000030CCBF854C0C4BFBCF1230F0122CBF8FF
:10F3E0005010CBF858000120CBF86000002A18BF5D
:10F3F000FBF7BDFDE048C07A28B30198052822D16B
:10F4000006EB440136F814004988401A3188401A46
:10F410007188084400B202903228C4BF01270497C3
:10F420000021002D0FD901FB04F2002006EB42035E
:10F4300001FB040B5A8A401C26F81B200928F7D32D
:10F44000491CA942EFD306EB4A0293464FF0000C49
:10F45000002D25D90020611E13D006EB410E36F891
:10F4600011303EF802ECA3EB0E031BB2002BB8BF29
:10F470005B421BB222F811308342C8BF1846491EB6
:10F48000EBD1019902297DD0108006EB440602EBF6
:10F4900044024845C8BF81460CF1010CAC45D9D3A4
:10F4A000B548B0F9100000908145A4BF012703972B
:10F4B0000BEB4A034FF0000C002D25D90021601EF4
:10F4C000022812D90BEB40023BF8106032F802EC34
:10F4D00032F8042C7644324412B223F810208A42C7
:10F4E000C8BF1146401E0228ECD800201980588061
:10F4F00098800BEB440B03EB44034145C8BF88469F
:10F500000CF1010CAC45D9D39B4BB3F912209045BB
:10F51000A4BF01270597002F14BF586C986C00F109
:10F52000010014BF5864986491480078FF2849D0BE
:10F53000089820F83A700898039900EBCA004180B7
:10F54000059981800499C18006990181596C4FEA1F
:10F55000E17C01EB1C5C6FF30B0CA1EB0C01418116
:10F56000996C4FEAE17C01EB1C5C6FF30B0CA1EB97
:10F570000C018181A0F80E90A0F8108002994182C0
:10F58000009900E022E08182C282B3F85C1001831E
:10F59000B3F85410418302264FF001000899002F60
:10F5A00000EB8503224600960CBF4E204D20FAF753
:10F5B00020FF012000EB8503224600964720089992
:10F5C000FAF717FF09B03846BDE8F08F02EB4401A7
:10F5D00031F9023C142BB9BF31F9041C142901275D
:10F5E000039751E7654870472DE9F84F8346624815
:10F5F00065490025B0F9108062480978604C0078B0
:10F600002E46AA464718F2F78BFC00905F48A4F1FB
:10F6100074090078492804BF4846FBF756F80020D3
:10F62000002F09D93BF8101039F81020891A24F856
:10F630001010401C8742F5D8DFF8509199F800006F
:10F640004C2804BF2046FBF740F8009810F4007FD8
:10F65000A7F1010012D000281CBF4749B1F91230B0
:10F6600026D034F910100029B4BF4A420A469A4203
:10F67000BCBF0D44761C401EF3D119E000281CBF0E
:10F680003D49B1F9123013D004EB400234F81010A8
:10F6900032F8022C891A09B224F810100029B4BFDC
:10F6A0004A420A469A42BCBF0D44761C401EEBD12A
:10F6B000002EC8BF95FBF6F52EB2268099F8000003
:10F6C0004F2804BF2046FBF700F80025781E0ED017
:10F6D00034F81010891B09B224F810100029B8BFA3
:10F6E000494209B28D42B8BF0D46401EF0D1258077
:10F6F00006F008F910F4817F18BF4FF00508454562
:10F7000006DD99F800004FF0010A4D2807D103E00B
:10F7100099F800004E2802D12046FAF7D6FF99F852
:10F720000000472804BF2046FAF7CFFF5046BDE847
:10F73000F88F2DE9F04F87B0FBF70EFE14480068F4
:10F74000B0F93610B0F934000DF0C5FA0120F5F724
:10F7500050F806F0D7F810F4817F14BF0020012084
:10F76000F2F775FC044F387E10F0100F19D011E03D
:10F770007D8500108014011084860010701A01101D
:10F78000E41A011004850010038500108285001022
:10F79000648600100420FFF7EFFB0F2818BFF5F771
:10F7A00026F8FF2038720021481E09F00FFD08F0EE
:10F7B00063F806F04CF9002818BF05F0D2FCF5F705
:10F7C000EBFF02287ED1DFF89CA1DFF89CB14FF05F
:10F7D00000084FF0E0297C78C7F834802046C7F84D
:10F7E0003880FFF7C9FB054621460220FEF76AFD77
:10F7F000052C7FD2DFE804F0770303037B000F249E
:10F800007E7806F07FF8002818BF0E24214628468F
:10F81000F6F71DF900286DD00DF094FA0DF097FA67
:10F82000F4F791FF050031D1387800281CBF0001A2
:10F83000F1F73DFD0024F2F773FB0690F1F751FB61
:10F8400010F0010F0ED0F1F7D1FD02280AD3B87ADB
:10F8500040B1069840F40030F2F743FA0124F2F781
:10F86000ACFB01E0F2F770FB87F80A8087F80380B1
:10F87000F5F75DF8FAF746FA012807D0F5F78CFF9F
:10F88000022802BF7878B042002D06D00DF05FFA52
:10F890000DF062FAF6F754FA2CE06846F2F790FDA4
:10F8A000F0B12CB1641E0698F2F71BFAF2F74CFB8C
:10F8B0006846FBF72CF90198F4F789FA68460DF0D1
:10F8C00082FA00E023E005469AF8000028B1D9F852
:10F8D0001800CBF80000C9F81080F2F7CEFDC9E798
:10F8E000F5F7B2FFC6E728460DF040FA02E02846D9
:10F8F000FFF731FCFAF706FA012803D1F5F74CFFC0
:10F90000022804D1F5F748FF02283FF464AF09F05C
:10F91000AAFCF4F76DFFFBF71FFDF5F73DFF052887
:10F920001CBF07B0BDE8F08FF0F74CFF58B10020C6
:10F93000F0F799FF0120F0F739FF07B00020BDE88C
:10F94000F04FF0F78DBF0120F0F78DFF07B00020DA
:10F95000BDE8F04FF0F72ABF4A00014603480DF01A
:10F960006AB900002F84001094840010701A0110EE
:10F97000394A30B4146894F86CC01CF0040F1ABFF4
:10F98000012222EA0C050CF00105B0F90030B1F9B2
:10F9900000201DB1E58AAA1A521E12B21CF0020FF5
:10F9A00003D0A48AE31A5B1E1BB21CF0040F19BF1C
:10F9B00002800B8003800A8030BC70474FF6FF71D5
:10F9C000A0F85010A0F85210A0F85410A0F856104B
:10F9D00070472DE9F05F16468A46834605F056FFCC
:10F9E000074605F04BFF002500F1CB09002E8CBF28
:10F9F0004FF6FF78BDE8F09F05EB450000EB0510E2
:10FA000007EBC00494F8880001280DD1A4F85080B9
:10FA1000A4F85280A4F85480A4F8568023464A469D
:10FA20005146584602F04FFF94F89500022818BF3F
:10FA300003280DD0B4F85000A4F85400B4F85200D4
:10FA4000A4F85600681CC5B2B542D5D3BDE8F09FF6
:10FA5000204601F0A3FCF5E7A8870010FE48407897
:10FA6000002818BF01207047FC48006890F870001B
:10FA700000F001007047F94909680A6F60F300025D
:10FA80000A6770472DE9F05F16460D46044605F0FB
:10FA9000F5FE8646F248202300EB050C80270A3845
:10FAA000EE4A4FF010084FF040094FF4807A0544B9
:10FAB000A0F13801A4B3012C73D04FF44076022C8E
:10FAC00070D0032C00F00B81042C18BFBDE8F09F10
:10FAD0001268508AC0EB001C4FEA4C04B2F81AC0FE
:10FAE000B4FBFCF464430C6200EB4004C4EB401430
:10FAF000C000B4FBFCF4B0FBFCF064434043C1E93C
:10FB000009404FF40070C8850E86B2F87400C0F347
:10FB10000330062859D2DFE800F05854585B5F6282
:10FB20001068448A04EBC40202EB041B428BBBFB4B
:10FB3000F2FB0BFB0BFBC1F820B004EB840B4FEA8C
:10FB40008B0BBBFBF2FB04EB4404B4FBF2F20BFBAC
:10FB50000BFB5243C1E909B29EF81420012A12D0CE
:10FB600090F874201407240DC2F30312CC851202FE
:10FB70000A8615F8014C002C04BF1CF801CCBCF11E
:10FB8000000F15D006E0B0F87420C2F30322120271
:10FB9000CA850A86B0F87400C0F30330062814D270
:10FBA00001E020E049E0DFE800F0100C1013171A24
:10FBB00096F895C0BCF1030F08BF02F58072E9D139
:10FBC000E7E7A1F82C80BDE8F09F8B85BDE8F09FAA
:10FBD000A1F82C90BDE8F09F8F85BDE8F09FA1F8BB
:10FBE0002CA0BDE8F09F1268508AC0EB00134FEACA
:10FBF000430C538BBCFBF3FC0CFB0CFCC1F820C08A
:10FC000000EB400CCCEB401C00EB4000BCFBF3FCD9
:10FC1000B0FBF3F00CFB0CFC4043C1E909C0B2F8A7
:10FC200074000207120DC0F303200002CA8500F51C
:10FC3000807008868F85BDE8F09F15F8014C012C77
:10FC400004BF1CF8010C0128D2F800C0BCF8120057
:10FC500033D0C0EBC005BCF81AC005EB850500EB3E
:10FC60000010B5FBFCF54000B0FBFCF06D434043D9
:10FC7000C1E908501068428AB0F81AC0D200B2FB3D
:10FC8000FCF252438A62406FC0F303421202CA85FB
:10FC9000022C08BF0E8603D0C0F3035212020A865C
:10FCA000000F062891D2DFE800F0070607050403DD
:10FCB00095E791E78CE784E787E700EBC00505EB64
:10FCC0000015BCF81AC000EB4000B5FBFCF5C00005
:10FCD000B0FBFCF06D434043C1E90850CAE712682D
:10FCE000508AC0EB001C4FEA4C04B2F81AC0B4FBB7
:10FCF000FCF464430C6200EB4004C4EB4014C0000D
:10FD0000B4FBFCF4B0FBFCF064434043C1E90940A0
:10FD1000B2F87400C0F303221202CA85C0F30330A4
:10FD20000A860628BFF451AFDFE800F00706070592
:10FD3000040354E750E74BE743E746E710B447486E
:10FD4000454C0368598A588B8A00B2FBF0F2524343
:10FD5000226101EBC10202EB0112B2FBF0F202FBE5
:10FD600002FC404AC2F820C001EB810C4FEA8C0C27
:10FD7000BCFBF0FC01EB4101B1FBF0F00CFB0CFC17
:10FD80004043C2E909C0B3F874000107090DD185E9
:10FD9000C0F30311090211864FF4A0515186491096
:10FDA0009186C0F303312020062907D2DFE801F055
:10FDB000060306051517102000E040202A4990850B
:10FDC0004FF6FF7008804880091F4FF0FF30088011
:10FDD00048800020207010BC70478020EEE74FF470
:10FDE0008070EBE72DE9F04F83B09B460D4604464B
:10FDF00005F044FD019005F05DFD0246174894F8BA
:10FE000045A0DFF854E00068164B418A408B01EBB7
:10FE10008101C900B1FBF0F000FB00F194F89500FE
:10FE200002281CBF94F85F00012825D00F4800EB82
:10FE3000CA0050E90267B5F80080B5F8029094F85E
:10FE40007000A0B394F8460000EB400C0CEB0010DF
:10FE500002EBC0000CE00000E8860010A88700104C
:10FE6000EA1B0110A81B011008870010581B011085
:10FE700090F8700098B129E0002003EB0A0C2E885E
:10FE80006F880CF8010C03EB4A08B3F834C0A8F8EB
:10FE900008C0BAF1010F08BF8EF80100CBE703EBF1
:10FEA0004A001A8EB0F808C094450FD90DE0FFE75C
:10FEB0008B450BD394F89500022807D003EB4A003A
:10FEC0001A8EB0F808C0944500D9028194F83A001F
:10FED000012806D094F8700018B98B4538BF988E69
:10FEE00000D3588E588694F870C0BCF1000F05D12D
:10FEF00094F895008B4512D3022810D060469A6A78
:10FF00005A4588BF022000909EF801100122002966
:10FF100004BFBAF1010FBCF1030F0BD101E00220C5
:10FF2000EDE7FF488EF801204189188E814284BF99
:10FF3000FB494881FA4B0C990098D3F820C0DC4566
:10FF400003D8022801D0012908D0F54B4FF0020E4A
:10FF50005A6A5A4508D9022816D105E0F04901EB42
:10FF60000A0000F8012C1BE071B15A4598BFE34527
:10FF70000FD202280FD003EB0A0010F8011C03294E
:10FF800008BF00F801EC0BE003EB0A0000F801ECFD
:10FF900006E0022804D103EB0A00032100F8011C4B
:10FFA00005F06CFCDE4B864603EB0A02988D12F8D6
:10FFB000012C198EB3F82EB0B3F832C0022A04D047
:10FFC000012A1CD0032A7DD032E003EB4A0201EB68
:10FFD000410CB2F808B0E34506D99EF80CB0BBF16D
:10FFE000000F08BFA2F808C0B2F808C08C4588BF4F
:10FFF000ACEB000038BF60441AD0108118E003EB6E
:020000021000EC
:100000004A0CBCF8082091420AD2501AA2EB6000B8
:10001000000A4FF6FF7101EA0020ACF8080007E083
:100020005A4588BF101A38BF104401D0ACF80800F8
:1000300003EB4A000289002A04BF0020014640D099
:100040001046B2F5807F36BF4FF4807101464FF401
:100050008072B448009B022B52D094F845C0002314
:100060000CF80030B0480068B0F814C00CFB08F37E
:10007000B0F810800CFB06F6B3FBF8FAC38AB6FBA7
:10008000F8F603FB09FBB0F812905F43BBFBF9F0F5
:10009000A1F5807B0BFB06F606EB0A26B6FBF1F119
:1000A000B7FBF9F7A2F580767E4306EB0020B0FBA4
:1000B000F2F208FB01F009FB02F1B0FBFCF0B1FB2E
:1000C000F3F100E011E094F84530984A02EBC303E5
:1000D00043F8080C94F8453002EBC30242F8041CC4
:1000E000A880E98003B0BDE8F08F03EB4A021189D4
:1000F000614588BF081A38BF08447FF47EAF97E790
:1001000094F8453013F800C0BCF1FA0F3CBF0CF175
:10011000010C03F800C094F84530185C3C28A1D3CA
:100120000198090A120A90F8420002287E480068E5
:1001300018D3B0F818A0B0F81AC00AFB08F3B0F84A
:1001400010800CFB09F9408AB3FBF8F30AFB06FAAE
:100150000CFB07FCB9FBF0F9BAFBF8F8BCFBF0FCB0
:10016000B34617E0B0F814A0B0F816C00AFB08F3C5
:10017000B0F810800CFB09F9408AB3FBF8F30AFBD6
:1001800006FA0CFB07FCB9FBF0F9BAFBF8F8BCFB6C
:10019000F0FCB346A1F1010000FB0830B0FBF1F325
:1001A000A2F1010000FB0C90B0FBF2F25E48016886
:1001B000B1F8109009FB03F009D3B1F81890B1F829
:1001C00012A0B0FBF9F00AFB02F9498B08E0B1F884
:1001D0001490B1F812A0B0FBF9F0C98A0AFB02F939
:1001E000B9FBF1F1434518BF62457FF46AAF43455F
:1001F00008BF5846624508BF394662E72DE9F04F0F
:1002000090F845C08FB04FF4806300290CBF484C74
:10021000484C04EB4C14484D029205EB4C1705F585
:10022000A5756544203C15F8015C07EB051606EB47
:10023000C10858F8206C921B039290F89520022A6E
:100240001CBF90F85F00012869D058F81C8C04EBA3
:10025000051206EB0809CDF83890D2F80490D6685C
:100260009568106809EB0602DFF8D0902844104426
:10027000D9F800A035445044D9F804A0DFF8C0B044
:100280005244D9F808A0D9F80C9055444E44DDF8F2
:1002900008A0DDF83890AAEB0909CDF82090DDF828
:1002A0000C90A9EB0809CDF82C90DBF80090814464
:1002B000CDF82890DBF8049009EB020ADBF80890EF
:1002C000DBF80CB0A9440BEB060EDDF828B00BFBF5
:1002D0000EFB0AFB19BB9BFBF3FBBBF1000F08BF36
:1002E0004FF0010B4FEA8E2E4FEA8A2A9AFBFBFA57
:1002F0004FEA892999FBFBF99EFBFBFECAF1000A34
:10030000CDF834A0DDF828A0C9F100094FEA8A2A07
:100310009AFBFBFB00FB0EFA02FB09AA12E081E04C
:10032000A81B0110DD220110A8870010581B011026
:10033000E8220110282401106825011034870010DC
:10034000448700109AFBF3FACDF828A0DDF834A01A
:1003500000FB0AFA02FB0BAA9AFBF3FACDF824A0E1
:1003600005FB0EFA06FB09A999FBF3F9DDF834A0A9
:10037000CDF8309005FB0AF906FB0B9999FBF3FBCE
:10038000DDF828A0DDF820900AFB09FEDDF824A0A6
:10039000DDF82C900AFB09EEDDF820A0DDF83090A6
:1003A0009EFBF3FE09FB0AFADDF82C900BFB09A972
:1003B00099FBF3F9DDF838A0C844F244CDE900A870
:1003C000DDF828A0CBF5806ECAF5806808FB00FB3D
:1003D000DDF824A0DDF83090CAF1000AC9F1000967
:1003E0000AFB05BB08FB02F809FB00F00AFB0688C4
:1003F0000EFB05009BFBF3FB98FBF3F890FBF3F07F
:10040000CDF810B0CDE9058009FB02F00EFB060027
:1004100090FBF3F00790F9480022E84604AE00EBA9
:100420000C0315E0F54A00206244039012F8012CF9
:1004300002AB07EB021202EBC10253F8204002EBC1
:100440008005401C00B245F8204C0228F5DB20E076
:1004500013F8015C58F8220007EB051505EBC10500
:1004600005EB820545F8200C002006EBC20513F8C9
:1004700001AC55F8209004EB0A1A0AEBC20A4AF8BC
:100480002090401C00B20228F1DB501C02B2022A6C
:10049000DEDBDA48604410F8010C07EB001000EBDB
:1004A000C10050F8200C0FB0BDE8F08F2DE9F04FDF
:1004B000ADF2BC5D0FFA81F90124DDF8E4C5DDF889
:1004C000E085CA46694600284BD032F81A00CDF8BC
:1004D000AC05BCF1010012D441F8204001EB8006CC
:1004E00032F81A50C6F8D052AAF101050FFA85FA6F
:1004F000BAF1000FB8BFA8F1010A401EECD50024E4
:1005000025464846BCF101020FD433F8107051F86B
:100510002260401E7E43341900B245EBE675002888
:10052000B8BFA8F10100521EEFD500263746BCF136
:10053000010061D401EB800233F819A0D2F8D02277
:10054000A9F1010902FB0AF296190FFA89F947EBA2
:10055000E277B9F1000FB8BFA8F10109401EE9D553
:100560004AE033F81A00CDF8AC05BCF1010012D412
:1005700041F8204001EB800633F81A50C6F8D052FB
:10058000AAF101050FFA85FABAF1000FB8BFA8F178
:10059000010A401EECD5002425464846BCF1010363
:1005A0000FD432F8107051F82360401E7E43341986
:1005B00000B245EBE6750028B8BFA8F101005B1E4C
:1005C000EFD500263746BCF1010015D401EB8003BE
:1005D00032F819A0D3F8D032A9F1010903FB0AF3CC
:1005E0009E190FFA89F947EBE377B9F1000FB8BF0D
:1005F000A8F10109401EE9D54FF000084046CDF8AA
:10060000A085BCF1000F0EDD51F82020DDF8A035EB
:10061000524312EB080843EBE27200F10100CDF8FF
:10062000A0258445F0DC002296461046CDF8A4258E
:10063000BCF1000F13DD01EB800351F82020D3F84B
:10064000D032DDF8A4955A434FEAE27A12EB0E0E4F
:100650004AEB0903401CCDF8A4358445EBDC4FF090
:100660000009CA464846BCF1000F0EDD01EB8002CE
:1006700051F82030D2F8D02200F101005A4312EB99
:1006800009094AEBE27A8445F0DC00200346024681
:10069000BCF1000F0DDD694601EB8001D1F8D012ED
:1006A00049434FEAE17B8A184BEB0303401C844526
:1006B000F1DC1046CDF8B025A8FB002CDDF8A01524
:1006C000CDF8B43501FB00C0AEFB09CBDDF8A415B5
:1006D000CDF8B81508FB030301FB09B10EFB0A10A6
:1006E000B2EB0C0163EB0000CDF8A405CDF8A81522
:1006F00008433DD0DDF8B005DDF8B425A0FB0413B8
:10070000AEFB06CB02FB0432DDF8B83500FB052258
:1007100003FB06B30EFB0733B1EB0C0062EB0301E6
:10072000DDF8A435DDF8A8250CF08AFADDF8E81527
:100730000860A8FB0602DDF8A01501FB0621A9FB55
:1007400004230AFB043308FB071109FB0533801A55
:1007500061EB0301090441EA10410004DDF8A4350E
:10076000DDF8A8250CF06CFADDF8E815486006E025
:10077000DDF8E81500200860DDF8E8154860DDF8D0
:10078000E805D0E90012DDF8AC05504311EB20403C
:1007900048BF00200DF2BC5DBDE8F08F2DE9F04FA1
:1007A00089B01F4690460E46044605F067F808904B
:1007B000007B00281CBF1422022115D094F83A3087
:1007C00094F845C0012B1FD0002804BF0C480569D0
:1007D00024D00C480068438A408BC3EB0313B3FB5F
:1007E000F0F000FB00F519E008993C2291F8421066
:1007F00002292CBF03210F21E0E70000A8260110E9
:10080000E8860010A8870010FE4864250068438A27
:10081000408B6B43B3FBF0F000FB00F5FA4B94F810
:1008200095A00020A3F1320BA3F11409BAF1020F35
:1008300018BFBAF1010F32D10BEB0C0A0AF8010C08
:1008400009EB0C0A0AF8010C8AF80900DFF8BCA3CE
:10085000E2440AF8010C8AF8090003EB4C0A2AF872
:10086000020CAAF81200DFF8A8A386F87000E24490
:1008700084F870000AF8010CDFF898A3E2440AF843
:10088000010CDFF894A3E2440AF8010CDFF88CA312
:10089000E2440AF8010CA4F85880A4F85A70E34422
:1008A000DFF87CA3CDF804B01BF801BC0AEB0C1EEA
:1008B0000EEB4B0ACDF800B02AF8108CAAF8907015
:1008C00094F895A0BAF1020F00F004814FF0000AED
:1008D000CDF810A0CDF808A0DDF800A00AF1070AB5
:1008E0000AF0070A0EEB4A0A3AF810BCBAF890A0D0
:1008F000A8EB0B08A7EB0A0AC24F3F68B7F818B07D
:100900000BFB08F8B7F810B098FBFBFBB7F81A80A0
:100910007F8A08FB0AF898FBF7F70397BBF1000FF3
:1009200006DD03EB4C074FF0020827F8020C18E035
:1009300006DA03EB4C074FF0010827F8020C10E031
:10094000B24F674417F8018C03EB4C0737F802AC41
:10095000BAF1640F05D20AF1010A27F802AC0127A7
:100960000497039F002F06DD03EB4C0A4FF00407AA
:10097000AAF8120019E006DA03EB4C0A4FF003075D
:10098000AAF8120011E0A14F03EB4C0E6744BEF829
:1009900012A07F7ABAF1640F07D20AF1010AAEF809
:1009A00012A04FF0010ACDF808A0DFF860A2E244DF
:1009B0001AF801ECBEF1000F4CD0C64524D103EB70
:1009C0004C0B3BF802BC934509EB0C0B40D8CDF81F
:1009D00014B01BF801BCBBF1640F3BD2DDF810E092
:1009E000BEF1000F36D10BF1010BDDF814E00BF076
:1009F000FF0BBBF10A0F0EF801BC2BD3DFF810B2CE
:100A0000E3440BF8010C25E009EB0C0ECDF814E0E3
:100A10001EF801ECBEF1050F13D2DFF8F4E1E64455
:100A2000CDF810E01EF801ECBEF1640F0ED2BBF160
:100A30000A0F0BDB0EF1010BDDF810E00EF801BC24
:100A400004E0DFF8CCB1E3440BF8010CDDF814B09E
:100A50000BF8010C9AF809B0BBF1000F36D0BB457A
:100A60001CD103EB4C035B8A934284BF09EB0C025D
:100A700050722BD809EB0C035A7A642A26D2DDF87F
:100A800008B0BBF1000F21D1521CD2B25A720A2A0F
:100A90001CD3604A624402F8010C17E009EB0C0217
:100AA000537A052B5B4B634436BF13F801BC03F844
:100AB000010CBBF1640F08D2DDF80CE0BEF10A0FA7
:100AC000A4BF0BF1010B03F801BC50720AF8018CB2
:100AD0008AF80970009A019B521CD2B203F8012CCB
:100AE0004FF0010B082A09D3019A02F8010C96F87D
:100AF0007020002A08BF86F870B006E096F87020D3
:100B0000002A08BF84F870007AD0454E00231A46A8
:100B100006EB0C1707EB4206521C36F8106C92B22B
:100B20003344082AF6D34FEAD30800231A46EA468C
:100B300007EB420636F8106CA6EB080676434AF837
:100B40002260521C92B23344082AF1D34FEAD30EEA
:100B5000344E00231A4606EB0C1707EB4206521CD4
:100B600036F8106C92B23344082AF6D34FEAD30A0F
:100B700000231A46E84607EB420636F8106CA6EB4F
:100B80000A06764348F82260521C92B23344082A7F
:100B9000F1D3DA080326754528BF954208D309EB3F
:100BA0000C0212F8013C082B9CBF527A082A0ED97D
:100BB000194984F87060614401F8010C17496144D7
:100BC00001F801BC94F8701003293CD018E0124AD7
:100BD000624412F8013CC82B3CBF5B1C02F8013C8C
:100BE0000E4B634413F8013C012B06D112F8012C83
:100BF0008A4298BF84F8706025D9022184F8701069
:100C0000034911E0A8870010A62801107E280110D2
:100C1000CE280110D8280110E2280110D42201109A
:100C200034270110D4270110614401F8010CFE495A
:100C3000614401F8010C94F8700003281EBF0428D9
:100C400009B0BDE8F08F089880F89AB509B0BDE802
:100C5000F08F2DE9F007F54CDDE9077C24680E885C
:100C6000658A648BC5EB0515AD00B5FBF4F81D88EE
:100C70003B8890F895701488032F45D190F8457003
:100C8000DFF8AC9309EB470737F802ACBAF1050F70
:100C90003AD2BAF1000F1AD0A1F800C0E11A1380BD
:100CA0000029B8BF494241459CBFBDE8F0077047E5
:100CB00065451CBFBDE8F0077047052190F8450069
:100CC00009EB400020F8021CBDE8F00770474FF028
:100CD000010A27F802ACAE4208BF002705D0E71A88
:100CE0003F04A6EB050A97FBFAF77E43A1F800C084
:100CF000A4EB2646002FA4EB03011CBF0CFB07F35B
:100D000006EB23431380CBE7A1F800C0BDE8F00752
:100D100070472DE9F74F98B019980088ADF83C005E
:100D200019984088ADF8340004F0A8FD0090189898
:100D300090F8454090F89500022804BF204600F046
:100D4000ECFFBC48BF4A2044139010F8015CBA483D
:100D5000BD4B204400F8015CB84800EB4408001D7E
:100D600038F8021C00EB4400169020F8021CC8B2B0
:100D7000B34901EB040B1BF8011CF9B1691CC9B2A2
:100D8000282927D304EB840103EB011101EB450C67
:100D900031F8507C3CF8506CBE1B02EB840747F8DE
:100DA000046CBCF850C0B1F85010A1EB0C0C02F16F
:100DB000080101EB840141F804CC26E002EB840C2D
:100DC00000214CF8041CDFF884C20CEB840C4CF8B6
:100DD000041C1AE004EB840C03EB0C1C0CEB41012B
:100DE00031F850CC31F8526CACEB060C02EB8406B7
:100DF00046F804CCB1F850C0B1F84E10ACEB010C81
:100E0000924901EB840141F804CC04EB840103EB2B
:100E1000011606EB4501BDF83CC021F850CCBDF8E9
:100E20003430A1F85030C4EB041101EB410788497C
:100E3000272D01EBC70707EB4001A1F5805EAEF857
:100E400098CEA1F8683104BF01210BF8011CB3282A
:100E500004D180490120214401F8010C189890F830
:100E60009500022853D0002D1CBF681EC0B25FD071
:100E700006EB4000B0F8501030F8509CA3EB010195
:100E80001BF8013CACEB09000193002B57D0724BCF
:100E9000002803EB840C5CF8049CACBF034643427F
:100EA00009EB030A6D4B4CF804AC03EB84030029F7
:100EB00053F804ECB4BFC1F100098946F14402EBD8
:100EC000840243F8049C52F8042C002AB8BF524212
:100ED000AAEB02024CF8042C5C4A02EB840252F8A2
:100EE000042C002AB8BF5242A9EB020243F8042C9A
:100EF0004E4A1268138B5843138A90FBF3F9508BB8
:100F00004843518A90FBF1FA0198002830D05448A8
:100F100002212044129000F8011C52482044039002
:100F200000F8011C189890F87000032849D145E09A
:100F30001BF8010C01280CBF2720284698E7464AD9
:100F4000002802EB840252F804CCB4BF43420346AB
:100F5000634442F8043C414A002902EB840252F8FF
:100F600004CCB4BF4B420B46634442F8043CBFE799
:100F70003D48B9F1000F00EB440030F8022CB4BF3B
:100F8000C9F1000149468A4207DAB9F1000FACBF46
:100F90004946C9F1000120F8021C4288BAF1000F4D
:100FA000B4BFCAF1000151468A42B0DABAF1000F6B
:100FB000ACBF5146CAF100014180A8E704F038FDFA
:100FC00068B1204600F0A9FE1998BDF83C10818058
:100FD0001998BDF83410C1801BB0BDE8F08F1BF824
:100FE00001BCBBF1010F05D0BBF1000F40D1681C63
:100FF00007283DD3B9F1280FD8BFBAF1280F09DC73
:10100000194800EB440030F8021C28299CBF408896
:1010100028282ED90098007B002829D01299032077
:1010200001F8010C039921E0D8280110A8870010CD
:10103000EC280110EA860010EC860010FC860010F7
:10104000EE8600100C870010F41B011014870010AE
:10105000341D0110F0860010248700102C8700102A
:10106000E01B0110EA1B01101C87001001F8010CA5
:10107000A4E0BDF83C00ADF83800BDF83400ADF890
:101080003000FF484FF0000900EB840050F8041CCA
:10109000FC4800EB840050F8040C8142C8BF4FF0BC
:1010A0000109A6F15002002004900590069006F177
:1010B000500329464FF0280E0790089009900A9097
:1010C0000B90BBF1000F14BF4FF01E0A01F1010A93
:1010D000BAF1050F69D94FFA81FC0CF1010080B219
:1010E000282828BF0020BBF1000F44D032F810B0F0
:1010F000CDF810B033F810000590BCF1140048BFD3
:10110000283032F810C0CDF818C033F8100007901E
:101110000DF1400B0AF0FF00CDF800E0CDE9010B26
:101120004846FFF7C3F90890BDF83C001490BDF89D
:1011300034001590D4480068418A428BC1EB0111FC
:10114000B1FBF2F10991418A428BC1EB0111B1FB74
:10115000F2F10A91418A408B01EB81014900B1FB18
:10116000F0F00B90B9F1000F04AA14D015A910A843
:1011700000F016FE13E0B2F800C0CDF810C0B3F8CE
:1011800000C020F00100CDF814C032F800C0CDF846
:1011900018C0185ABBE714A910A800F05DFE1499F6
:1011A000ADF83C101599ADF83410012820D01299F3
:1011B000002001F8010C039901F8010C1398139910
:1011C00010F8010C401CC0B201F8010C282803D310
:1011D0001399002001F8010C38F8020C401C80B271
:1011E00028F8020CB42824BF002028F8020CEBE6F3
:1011F000A648C1681A9881427DD91698CB46A7F5B2
:10120000B47210F8021CA24807F5B473204416907B
:1012100010F801CC0020B4240490059006900790AB
:10122000089009900A900B90BCF1000F14BF4FF08A
:10123000AA0901F10109B9F1050F67D94FFA81FA3D
:101240000AF1010080B2B42828BF0020BCF1000FD1
:10125000944640D03CF810C0CDF810C033F81000D0
:101260000590BAF15A0048BFB43032F810C0CDF83A
:1012700018C033F81000079009F0FF00CDE90040D6
:101280000DF1400CCDF808C05846FFF70FF9089053
:10129000BDF838001490BDF8300015907A48006809
:1012A000418A428BC900B1FBF2F10991418A428B1C
:1012B000C900B1FBF2F10A91418A408BC900B1FB30
:1012C000F0F00B90BBF1000F04AA15D015A910A8DF
:1012D00000F066FD14E0BCF800C0CDF810C0B3F813
:1012E00000C020F00100CDF814C032F800C0CDF8E5
:1012F00018C0185ABFE738E014A910A800F0ACFDD8
:101300001499ADF838101599ADF83010012834D083
:10131000681CC4B2C4F1280906EB440A4FEA49022A
:10132000AAF150019346A7F5B4700BF084FC0AF1C2
:1013300050015A4607F5B4700BF07DFC07EB4907E6
:101340006400A7F5B470A6F1500122460BF073FCBF
:1013500007F5B47006F1500122460BF06CFC1699AB
:10136000002001F8010C28F8025C1299012001F814
:10137000010C039901F8010C20E7BDF83800BDF815
:101380003C1008444008ADF83C00BDF83000BDF802
:10139000341008444008ADF83400E6E72DE9F04F7A
:1013A0008FB0044600F094FD049000F094FD0A9084
:1013B00001200B9004F07EFA804604F05FFA099059
:1013C00094F8455004F05AFA94F84590002101270A
:1013D0008DF819108DF818708DF81770017B2A4E52
:1013E00000291CBF017D012918D03068016FC1F3AD
:1013F000C0428DF81420C1F340418DF81510006FE4
:10140000C0F380408DF81600FDF745FD02287AD024
:10141000FDF741FD012876D000F0E9B8316891F878
:101420007020C2F3C0038DF81430C2F340028DF86F
:10143000152091F87010C1F380018DF81610007D11
:1014400001287BD004F05EFA10F4817F77D0224629
:1014500049460120FEF716FB0B48D0F800C09CF867
:10146000700010F0010F00F0478394F84600B4F8C4
:1014700050A0ADF808A0B4F85260ADF80A6009E0D9
:10148000248700102C870010A8870010E886001021
:10149000F086001000EB400101EB001008EBC000EB
:1014A000089094F8952094F84500F849022A1CBF4A
:1014B00094F85F20012A00EB40007CD001EB800211
:1014C00032F80A3C22F8083C32F80C1C22F80A1CBC
:1014D00022F80CAC32F8049C22F8029C32F8068CFC
:1014E00022F8048C22F8066C1FFA8AF262F30F00CD
:1014F00061F31F408A4284BF61F30F0062F31F4013
:10150000010C994200E05BE088BF63F31F4081B2A9
:10151000020C914284BF62F30F0061F31F404FEA57
:10152000104A66F30F0068F31F40464584BF68F316
:101530000F0066F31F40010C494501E024E027E05D
:1015400088BF69F31F4081B2020C914284BF62F3ED
:101550000F0061F31F40060C9DF81400ADF80CA0BD
:10156000ADF80E60012801BF94F893000028ADF893
:1015700008A0ADF80A6094F8950002281CBF94F802
:101580005F00012846D0C5E022464946032061E7B6
:10159000FDF781FC02280FD0FDF77DFC01280BD060
:1015A00004F05CFA80B104F01DFA08280CD0224641
:1015B000494600204EE71EE08DF814708DF8167035
:1015C00022464946042045E794F83A000128EED126
:1015D0003068016FC1F3C0428DF81420C1F340415F
:1015E0008DF81510006FC0F380408DF8160022466C
:1015F000494602202EE701EB800020F808AC20F8D5
:101600000AAC20F80CAC20F8026C20F8046C20F82E
:10161000066CA1E7BCF87A000D90BCF87860FDF785
:101620003AFC022803D0FDF736FC012801D140F630
:10163000991697480022284400F8012C95480192F9
:10164000284400F8017C9448174600EB45100C90A4
:10165000924800EB45100790914800EB4510009030
:101660000799002001EB071E009901EB071B0C995D
:1016700001EB071900210EEBC0030BEBC00C09EBCB
:10168000C00803EB810A4AF8202C0CEB810A4AF8C7
:10169000202C08EB810A491C09B24AF8202C0229A7
:1016A000EFDB401C00B20228E4DB781C07B2022FFB
:1016B000D6DB019A0798DFF8ECE100EB021ADDE9CE
:1016C0000002002100EB0219774A002002EBC1085A
:1016D0000AEBC10C09EBC1070EEBC103814204D137
:1016E0000D9A43F8202048F8206053F820200CEB96
:1016F000800B02EB820252004BF8202C07EB800B90
:10170000401C00B24BF8202C0228E7DB481C01B239
:101710000229D9DBBDF8082000212046FEF76EFD26
:101720000646BDF80A2001212046FEF767FD002E7F
:10173000B8BF00260028B8BF00205C4F3968B1F957
:101740001020531EB342B8BF1E46B1F912104A1EF4
:101750008242B8BF1046B2B283B24D48ADF80C20F9
:1017600041190A30ADF80E30284411F801CC10F8B8
:10177000016C01F8016C00F801CC9DF816000128FD
:1017800019BF94F893000128ADF80820ADF80A308D
:1017900020460899FFF702F80898B4F85030B0F8DE
:1017A0005020991A48BFD11AB4F85220B0F85230DC
:1017B000D01A48BF981A494300FB0016022D9CBF5F
:1017C0009DF8170001281DD1324602A92046FFF7D7
:1017D000A0FA0998007BA8B93548284410F8010CF4
:1017E000012807D070B93348284410F8010C401C78
:1017F000282807D9BDF80C00ADF80800BDF80E0088
:10180000ADF80A002C492D4A2944002011F8011C8A
:1018100011B1012905D009E0511911F8011C29B9AC
:1018200005E0501910F8010C012800D001200090AB
:101830000998334602A990F842202046FEF7D2FAD2
:101840009DF81500012804BF94F89300002810D0DB
:10185000BDF80800A4F85400BDF80A00A4F856002A
:1018600004F0E6F8012804BF94F88D0001282FD178
:1018700026E0BDF80C00ADF80800BDF80E10ADF87C
:101880000A10A4F85400BDF80E00E7E7BC260110CA
:10189000A8260110B226011068250110E8220110C7
:1018A000282401103487001044870010A8870010F6
:1018B000EE860010EC860010E01B0110EA1B011000
:1018C000B4F85000A4F85400B4F85200A4F856003C
:1018D0009DF81900012805D1099890F8421020467A
:1018E00000F015F90B98D8B3B4F85400ADF808001F
:1018F000B4F85600ADF80A0003F0DCFF804600F0B3
:10190000E7FA064600F0E7FA054694F8460000EBD1
:10191000400101EB0010396808EBC000B1F81280FB
:10192000B1F81090BDF80810ADF82010BDF80A10FD
:10193000ADF81C10B0F85410ADF82C10B0F85600EB
:10194000ADF8300000F05EFBF0B3BDF82000B0420F
:1019500038BF3046ADF82000BDF81C10A94200E0A9
:101960001BE038BF2946ADF81C10A9EB0602531E38
:101970008342B8BF1846ADF82000A8EB0500421E10
:101980008A42B8BF1146ADF81C10BDF82000ADF872
:101990000C00BDF81C00ADF80E009DF818000128E1
:1019A0007ED0BDF80800049ABDF80A109042B8BF76
:1019B00010460A9A9142B8BF11463B68049AB3F99F
:1019C00010C0ACEB020200E013E0A2F1010C844570
:1019D000B8BF6046B3F912300A9A9A1A531E8B4266
:1019E000B8BF1946A4F85400A4F856100FB0BDE8CB
:1019F000F08F94F8950002281CBF94F85F0001282E
:101A00001DD16078FE4A58B139688B795B1E9842C7
:101A10001CBF2078002803D0C979491E884207D10D
:101A200094F84500052102EB400020F8021C06E076
:101A300094F84510002002EB410121F8020CBDF89A
:101A40002000B04208D20CA8CDE900060BAB07AAD3
:101A500008A92046FFF7FDF8BDF81C00A84208D2EF
:101A60000BA8CDE900050CAB08AA07A92046FFF793
:101A7000F0F8A9EB0600BDF82010401E884209DAF4
:101A800080B20CA9CDE900100BAB07AA08A920462B
:101A9000FFF7DFF8A8EB0500BDF81C10401E00E0C2
:101AA0000DE08842BFF671AF80B20BA9CDE90010FE
:101AB0000CAB08AA07A92046FFF7CBF865E794F816
:101AC00095000522CF4902281FBF94F85F00012826
:101AD00094F84500405C08BF94F83D0094F83D3010
:101AE0004FF0040C0CFB003090FBF2F094F8452012
:101AF000505484F83D0054E7B4F85000A4F8540062
:101B0000B4F85200A4F856000FB0BDE8F08F2DE9EC
:101B1000F04F90F84510DFF8F0B282B04FF6FF7E3C
:101B2000012910D00BF11C004FF0FF3101804180E2
:101B3000001DA0F800E0A0F802E000208BF80000F3
:101B400002B0BDE8F08FB149B0F854A0DFF8C0C2D0
:101B500009680A8B01920AFB02F30A8A009293FB3E
:101B6000F2F2B0F85690B1F81A804F8A09FB08F3E8
:101B700093FBF7F190F89540BCF80030BCF802C038
:101B8000022C47D09BF80060002E00F0BE80A14CD4
:101B9000022EB4F900B077D2019C03FB04F5009C3F
:101BA00095FBF4F90CFB08F494FBF7FAB2EB09048B
:101BB00048BFA9EB0204B1EB0A0548BFAAEB010537
:101BC000142CB8BF142D64DAF34562D04A45924A0A
:101BD00082FB04424FEA6204A4EBE272D4BF9A1A79
:101BE0001A448C4B51458C491A8081FB05214FEAE0
:101BF0006102A2EBE171C3BF6144864A5180ACEB44
:101C00000102DCBF83494A8082490A88A0F8542037
